:100000005446495300010000A46A0200198BABA3B7
:1000100009300126181120144E38413009300200F1
:10002000181120144E3841300930010418112014E1
:100030004E384130030000000000000000000000C6
:100040005446435300200000DC4E02000000000034
:1000500000000210012100002521000041220000C3
:10006000292100002B2100002D2100003D2100004E
:100070003D2100003D2100003D2100002F21000016
:10008000312100003D2100003321000049590000CA
:100090002F5A0000372100003D21000001BB001055
:1000A00037210000D53D0000DB3D00003D21000070
:1000B0003D2100007F550000994C0000E13D00000B
:1000C000C1520000372100003D2100003D21000009
:1000D0000000000000000000000000000000000020
:1000E0000000000000000000000000000000000010
:1000F0000000000000000000000000000000000000
:1001000000000000000000000000000000000000EF
:1001100000000000000000000000000000000000DF
:1001200000000000000000000000000000000000CF
:1001300000000000000000000000000000000000BF
:1001400000000000000000000000000000000000AF
:1001500000F003F800F020F8FEE70D480168890878
:100160008900002001C101C101C101C17047000027
:100170006CF00010FEE7FEE7FEE7FEE7FEE7FEE7B5
:10018000FEE7FEE7FEE703480047FEE7FEE7000064
:10019000202100003D21000000F002F800F068F886
:1001A0000AA090E8000C82448344AAF10107DA45D2
:1001B00001D100F05DF8AFF2090EBAE80F0013F0BC
:1001C000010F18BFFB1A43F001031847D05B010071
:1001D000105C01000A444FF0000C10F8013B13F0D2
:1001E000070408BF10F8014B1D1108BF10F8015B90
:1001F000641E05D010F8016B641E01F8016BF9D183
:1002000013F0080F1EBF10F8014BAD1C0C1B09D1D9
:100210006D1E58BF01F801CBFAD505E014F8016B4B
:1002200001F8016B6D1EF9D59142D6D370470000DD
:10023000103A24BF78C878C1FAD8520724BF30C812
:1002400030C144BF04680C607047000000230024E4
:1002500000250026103A28BF78C1FBD8520728BFD6
:1002600030C148BF0B6070471FB51FBD10B510BD32
:10027000DFF80CD0FFF7F8FF05F056FA14F08EFD0A
:100280000000021003B4FFF7F1FF03BC14F08EFD71
:100290001EF0040F0CBFEFF30880EFF309800AF0A3
:1002A0006BBD000008B5002103200B460A460091F3
:1002B00012F0B8FE08BD38B5F64C002525816581E1
:1002C000A58112F080FEE061FF20A071F24814F0D9
:1002D00035FF0120E0716561257003202B462A4619
:1002E0002946009512F09EFE012038BD38B5E94D33
:1002F0000228AC7922460DD0052810D0A24208BFB2
:1003000038BD0020034602462146009012F08AFEC6
:10031000AC7138BD022914BF01240224EEE7022982
:1003200014BF64246524E9E738B513460A464FF044
:10033000010C002401466046009412F073FE38BDA3
:10034000D449012048707047D24840787047D1495D
:100350000020487070472DE9F04104460127002530
:1003600003F00700CB4E8846012804BF0020B0816F
:1003700046D0022844D1B08904280BD2002818BFE7
:10038000B06902D112F03CFFB06110F8011B21707E
:10039000B0612EE0062808D212F034FFB189C1F115
:1003A0000501C900C840207023E0082808D212F0D7
:1003B0002DFFB189C1F10701C900C840207018E0C4
:1003C0000C2808D212F0FFFDB189C1F10B01C90060
:1003D000C84020700DE00E2808D212F0F6FDB18959
:1003E000C1F10D01C900C840207002E0FF2020705B
:1003F0000027B089401C80B2B0810E2828BF01259B
:1004000088F800503846BDE8F08130B403F00700AA
:100410000024DFF880C201280BD06046BCF80C3005
:100420000089022B0CD2120242EA1020ACF808001C
:1004300010E0ACF80840ACF80A40ACF80C400CE016
:100440001844851EB5F5806F04DADCF81C5028448A
:1004500000F8022C581CACF80C000C7030BC0020CA
:100460007047F0B40746002003F00704894D0646A4
:10047000012C04BFAE812E6125D0DFF818C2022CFA
:10048000BCF80AC003D013F0070F0DD01BE0AA89F7
:100490000CEB0203B3F5806F15D2E869C05C3870CD
:1004A000501CA88101200EE0120242EA1C226A813F
:1004B0002B69012B05D1B2F5806F24BF40F2FF32CA
:1004C0006A815A1C2A610E70F0BC704738B503F07F
:1004D000070000240D4601280AD16E4821460B462C
:1004E00084810481448102200A46009412F09AFD1E
:1004F0002C70002038BD30B50C0068A183B00968AD
:100500004FF00002029108BF03250AD0217802AB08
:100510005D5C002D18BF022D41D0012D7ED0032D32
:100520000DD10F2101700321417042808280C28071
:10053000028142818281817B21F001018173002D42
:100540001EBF012D03B030BD05F0FCF805281CBF0F
:1005500003B030BD0AF0A7FC042804BF03B030BDCF
:10056000002D0CBFC020C1208DF8000060788DF8F0
:10057000010060880123000A8DF80200A0788DF840
:100580000300A0880622000A8DF8040020798DF867
:100590000500694607200DF0A9FE03B030BD617863
:1005A00000EB011202F8101C617800EB011101F858
:1005B0000F5C6278618800EB021222F80E1C6278F0
:1005C000A18800EB021222F80C1C6278A17900EBE2
:1005D000021222F80A1C6278217A00EB021222F839
:1005E000081C6278617A00EB021222F8061C62781D
:1005F000217B00EB021222F8041CE17905296178C5
:1006000000EB011010F8021C0EBF41F0010121F0B7
:10061000010100F8021C92D132E0FFE7617800EBA3
:10062000011303F8101C6378012100EB031303F896
:100630000F1C6378618800EB031323F80E1C6378AA
:10064000A18800EB031323F80C1C617800EB011167
:1006500021F80A2C617800EB011121F8082C61784F
:1006600000EB011121F8062C617800EB011121F853
:10067000042C617800EB011010F8021C21F001013C
:1006800000F8021C5BE703490020887070470148AE
:10069000807870470004011008080110030002016F
:1006A0007549012088707047744A11547047724828
:1006B00000B5C06983B04FF00001407810F0020F20
:1006C0000AD000918DF8041001230522694600200C
:1006D0000DF043FE03B000BD10F0040F12D0012056
:1006E0008DF800008DF801108DF802108DF80310C0
:1006F0008DF8041003460522694600200DF02DFEFA
:1007000003B000BD10F0080F12D002208DF80000D9
:100710008DF801108DF802108DF803108DF804107B
:1007200001230522694600200DF017FE03B000BD2D
:1007300003B001230022632107205DF804EB0DF0D4
:10074000A5BD026812F0C00F10D04B4812F0400F48
:1007500004BF0021017004D0012101704169491CCE
:1007600041610123002106200DF090BD01230022EC
:10077000632107200DF08ABD70473F49002818BF4C
:100780000120C87170473C48C07970473A48C0782A
:100790007047002818BF01203749C8707047364994
:1007A0000871704734480079002818BF012070474D
:1007B000014600200729324A04BF02F14000704779
:1007C000082904BF2E487047092908BF02F180009C
:1007D000704710B44FF0000C294C072808BF04F1F3
:1007E000400C08D0082808BFDFF894C003D00928BF
:1007F00008BF04F1800C4FF00000ABB1002A9CBF91
:1008000010BC70473CF91030141A01EB440434F961
:10081000024C234403EBD3735B102CF81030401CC4
:100820008242EFD810BC7047002A9CBF10BC7047B2
:10083000131A01EB430333F8023C2CF81030401C30
:100840008242F5D810BC70470B480078002818BFCA
:100850000120704708484069704707494861704760
:10086000002818BF012004494871704702484079A8
:10087000002818BF0120704700040110080801106B
:10088000120801107047FE48D0F8C00000F00100C7
:10089000704770B5FA4C05000AD001F041FA38B93A
:1008A000D4F8C00010F0010F1CBF0020A06005D1DB
:1008B0000120A060002D08BF002000D00120206290
:1008C000002D18BF70BDD4F8D410D4F8D00011F0AA
:1008D000010F18BF11F0600F24D0D4F8B02222F419
:1008E0008032C4F8B02241F0610242F0FF22C4F825
:1008F000D42040F0610242F0FF22C4F8D02021F061
:100900006102C4F8D42020F06102C4F8D020D4F8E9
:10091000B02242F48032C4F8B022C4F8D410C4F833
:10092000D00070BD10F0010F18BF10F0600FD4D1CF
:1009300070BDD348006A002818BF01207047C0006E
:1009400000F1804000F5A04041637047C00000F115
:10095000804000F5A040006B00F4807070471021CB
:10096000C00000F1804000F5A04041637047C449D9
:10097000D1F8402160F30D22C1F840217047C048F2
:10098000D0F84001C0F3052070470207520DC0F3B4
:10099000031002EB401000F1804000F5A040002958
:1009A000D0F8401114BF41F0010121F00101C0F85D
:1009B000401170470107490DC0F3031001EB4010CF
:1009C00000F1804000F5A040D0F8400100F00100A7
:1009D0007047AB4900230B6202680A6042684A60B4
:1009E00082688A60C268CA60426A0A64826A4A642B
:1009F00002698A614269CA61426B0A66826B0A6750
:100A0000C26B4A67026C8A67426CC1F88020826CB4
:100A1000C1F88420C26CC1F88820026DC1F88C2016
:100A2000026EC1F89C20426EC1F8A020826EC1F80F
:100A3000A420C26EC1F8A820C26FC1F8C020D0F8AF
:100A40008020C1F8C420D0F88420C1F8C820D0F894
:100A50008820C1F8CC20D0F88C20C1F8D020D0F864
:100A60009C20C1F8E020D0F8A420C1F8F020D0F8F4
:100A7000A820C1F8F420D0F8AC20C1F8F820D0F8B4
:100A8000B020C1F8FC2021224A63CA63C2694A62CD
:100A9000C26A8A64026BCA64026FC1F8AC20D0F8E3
:100AA0009020C1F8D420D0F89420C1F8D820D0F8F4
:100AB000A020C1F8E420426FC1F8B020826FC1F8D5
:100AC000B420D0F8F821C1F88022D0F8FC21C1F878
:100AD0008422D0F80022C1F88822D0F80422C1F87C
:100AE0008C22D0F80822C1F89022D0F80C22C1F84C
:100AF0009422D0F81022C1F89822D0F81422C1F81C
:100B00009C22D0F8182222F48032C1F8B022D0F80A
:100B1000B420C1F80021D0F8B820C1F80421D0F8E1
:100B2000BC20C1F80821D0F8C020C1F80C21D0F8B1
:100B3000C420C1F81021D0F8C820C1F81421D0F881
:100B4000CC20C1F81821D0F8D020C1F81C21D0F851
:100B5000D420C1F82021D0F8D820C1F82421D0F821
:100B6000DC20C1F83021D0F8E020C1F84021D0F8D5
:100B7000E420C1F84421D0F8E820C1F84821D0F899
:100B8000F020C1F85021D0F8F420C1F85421D0F859
:100B9000F820C1F85821D0F8FC20C1F85C21D0F829
:100BA000EC20C1F84C21D0F82021C1F88021D0F8E8
:100BB0002421C1F88421D0F82821C1F88821D0F857
:100BC0002C21C1F88C21D0F83021C1F89021D0F827
:100BD0003421C1F89421D0F83821C1F89821D0F8F7
:100BE0003C21C1F89C21D0F84021C1F8A021D0F8C7
:100BF0004421C1F8A421D0F84821C1F8B021D0F88F
:100C00004C21C1F8C021D0F85021C1F8C421D0F83E
:100C10005421C1F8C821D0F85C21C1F8D021D0F806
:100C20006021C1F8D421D0F86421C1F8D821D0F8CE
:100C30006821C1F8DC21D0F86C21C1F8E021D0F89E
:100C40007021C1F8E421D0F87421C1F8E821D0F86E
:100C50007C21C1F8F021D0F88021C1F8F421D0F82E
:100C60008421C1F8F821D0F88821C1F8FC21D0F8FE
:100C70005821C1F8CC21D0F87821C1F8EC2101E04D
:100C800000500040D0F88C21C1F80022D0F890210B
:100C9000C1F80422D0F89421C1F80822D0F8982194
:100CA000C1F80C22D0F89C21C1F81022D0F8A02164
:100CB000C1F81422D0F8A421C1F81822D0F8A82134
:100CC000C1F81C22D0F8AC21C1F82022D0F8B02104
:100CD000C1F82422D0F8B421C1F83022D0F8B821CC
:100CE000C1F84022D0F8BC21C1F84422D0F8C0217C
:100CF000C1F84822D0F8C821C1F85022D0F8CC2140
:100D0000C1F85422D0F8D021C1F85822D0F8D4210B
:100D1000C1F85C22D0F8D821C1F86022D0F8DC21DB
:100D2000C1F86422D0F8E021C1F86822D0F8E821A7
:100D3000C1F87022D0F8EC21C1F87422D0F8F0216B
:100D4000C1F87822D0F8F421C1F87C22D0F8C4216F
:100D5000C1F84C22D0F8E421C1F86C22FE4A126896
:100D600032F0FF0C05D1D1F890C062F3030CC1F84A
:100D700090C0FA4A5370C36F13F0010F1CBF0123D8
:100D80005370D1F8C03023F00103C1F8C030D0F85F
:100D90008C3013F0010F03D0537843F002035370EB
:100DA000D1F8D03023F00103C1F8D030D0F8900052
:100DB00010F0010F03D0507840F004005070D1F8CB
:100DC000D40020F00100C1F8D4007047E348007857
:100DD0007047E24880787047E049C8707047DF4844
:100DE000C0787047DE4951F8C42F60F309020A60E9
:100DF0007047DB48D0F8C400C0F309007047D749FA
:100E000048607047D648C06870472DE9F047DFF862
:100E10004C93054615F4003F99F8010099F803102A
:100E200000EA010418BF24F0010415F4802F18BF54
:100E300024F0020415F4002F18BF24F0040415F464
:100E4000801F18BF24F00804DFF81483D8F8B0021C
:100E500020F48030C8F8B00214F00F0F59D0D9F840
:100E60000460D8F8B802002740F00100C8F8B802C2
:100E7000D8F8B80220F00100C8F8B802D8F8B002DB
:100E800040F48030C8F8B0024FF0630A0DE002F081
:100E9000ECFD5046D8F8B81211F0010F01D001272F
:100EA00003E0011EA0F10100F4DC301EA6F10106F2
:100EB00001DD002FEBD067B3D8F8C00014F0010FAC
:100EC0000CBF20F0010040F00100C8F8C000D8F8C5
:100ED000D00014F0020F14BF40F0010020F0010018
:100EE000C8F8D000D8F8D40014F0040F14BF40F0B4
:100EF000010020F00100C8F8D40089F80240012068
:100F000089F80000D8F8B00240F48030C8F8B00288
:100F100033E0D8F8C00020F00100C8F8C000D8F8CD
:100F2000D00020F00100C8F8D000D8F8D40020F09C
:100F30000100C8F8D400002089F80200ACB10220FA
:100F400089F80000D8F8B00240F48030C8F8B00248
:100F5000D8F8B80240F00100C8F8B802D8F8B802D2
:100F600020F00100C8F8B80207E0D8F8B01221F468
:100F70008031C8F8B01289F80000D8F8400115F0A7
:100F8000020F20F00D0018BF40F0010015F0080F0F
:100F900018BF40F0040015F0040F18BF40F008001F
:100FA000C8F8400115F0010F21D001F0A9F804465E
:100FB00001F0A9F80146D8F80C0000280EBF204621
:100FC000084621460028D8F8C00114BF40F00100AF
:100FD00020F00100C8F8C001D8F8E001002914BFD2
:100FE00040F0010020F00100C8F8E0010BE0D8F863
:100FF000C00120F00100C8F8C001D8F8E00120F0DD
:101000000100C8F8E00115F0200F18BF002417D028
:10101000204601F07FF800284FEA441000F180409C
:1010200000F5A040D0F8401214BF41F0010121F0BA
:101030000101C0F84012641C022CE9D3BDE8F0871E
:10104000D8F8400220F00100C8F84002D8F8600249
:1010500020F00100C8F86002BDE8F0872DE9F00338
:101060000246002011074C0DC2F3031104EB41119D
:1010700001F1804101F5A041D1F8401111F0010FBB
:1010800011D142F01001C1F3031104EB411101F140
:10109000804101F5A041D1F8401111F0010F04BFCA
:1010A000BDE8F0037047D60106F1804101F5A0418B
:1010B000D1F81C31C3F30809294BDB69D1F80011C1
:1010C00003F008071FFA81F8002142EA0113C3F375
:1010D000031304EB431303F1804303F5A043D3F858
:1010E000403113F0010F18D006EB411303F1804398
:1010F00003F5A043D3F844C1CCF3080517F1000C65
:101100001CBFD3F844C1CCF3023CD3F8403105FAFC
:101110000CFCC3F3054360441844491C0229D4D392
:1011200000FB08F0C9EB0911BDE8F00300EB41003A
:10113000704710B50120FFF791FF04460220FFF72A
:101140008DFF044400F0E7FB20444FF47A714843DC
:1011500047F2305106E00000E0FE030020040110D9
:1011600000500040B0FBF1F010BD2DE9F041FE4E03
:101170000546306810F01F0408BF01240120FFF766
:101180006DFF07460220FFF769FF074400F0C3FB2D
:101190003918F64F002D18BF00294DD0D6F8C000E1
:1011A000002210F0010F34D07820B0EB151F08D9C1
:1011B000D6F8CC0020F00F0040F00100C6F8CC00BB
:1011C0002CE0D6F8C400EA4BC0F309006043A0EB62
:1011D000001003EB4003E748A0FB05C04FEA502C8A
:1011E000B3FBF1F0102828BF0F20844598BF60465C
:1011F000002808BF012005D0012884BF00FB113260
:10120000B2FBF0F2D6F8CC3060F30303C6F8CC3072
:1012100004E0B7FBF5F0884288BF421AC4EB041023
:101220004000B2FBF0F0B0F5005F28BF41F6FF7060
:10123000726860F30C0272607068C0F30C00604367
:10124000C0EB001001EB4000B7FBF0F0BDE8F0810F
:10125000C548D0F8C01011F0010F07D0D0F8CC006D
:1012600000F00F00C0EB00108001704770B50168FE
:10127000406801F01F05C0F30C060120FFF7EEFEE9
:1012800004460220FFF7EAFE044400F044FB06FB9C
:1012900005F1C1EB011104EB41010844B349B1FB75
:1012A000F0F070BDB048D0F8CC0000F00F007047EF
:1012B000AD494A684B68C2F30C0260F30C034B6003
:1012C00010467047A8484068C0F30C007047C00142
:1012D00000F1804000F5A040D0F800014EF66021FA
:1012E00080B2B1FBF0F0401C4008704730B44EF6BD
:1012F000602331B1B3FBF1F1491C4A08B2F5804FCC
:1013000001D343F6FF72B3FBF2F1491C4D08C10152
:10131000530801F1804101F5A041002807BF981F43
:10132000A3F10C0CD1F8040180B218BFA2F1060C95
:101330002CF0010CD1F8004162F30F04C1F8004118
:10134000D1F8002163F31F42C1F80021D1F8042134
:1013500060F30F02C1F80421D1F810016CF30F0003
:10136000C1F81001284630BC7047C00100F1804030
:1013700000F5A040D0F80001000C7047C20102F156
:10138000804202F5A042D2F8003161F31F43C2F857
:101390000031002818BF70478A1F901F20F00101FC
:1013A0007148D0F8043162F30F03C0F80431D0F86B
:1013B000102161F30F02C0F8102170470107490D99
:1013C000C0F3031001EB401000F1804000F5A04095
:1013D000D0F84401C0F3080070470207520DC0F373
:1013E0000310654B02EB401000F1804000F5A04077
:1013F0009B58D0F84421CB1A61F30802C0F844216D
:10140000D0F844119B1E63F31841C0F84411704793
:101410005549C969594A11F0100F4FEA00714FEA56
:101420005151C0F3031001EB401000F1804000F572
:10143000A0405258D0F84401D2B2C0F3080008BF0F
:101440000022801A0004000C08BF01207047030925
:10145000DB0103EB810101F1405101F5C0410007BF
:10146000C00E0B6802FA00F01843086070470209CA
:10147000D20102EB810101F1405101F5C0410007A9
:101480000968C00E21FA00F000F00300704702075F
:10149000520DC0F3031002EB401000F1804000F544
:1014A000A040C0F84C1170470107490DC0F303106C
:1014B00001EB401000F1804000F5A040D0F84C0155
:1014C0007047294A0021D26912F0080F0DD0010798
:1014D000490DC0F3031001EB401000F1804000F50E
:1014E000A040D0F84401C0F30231084670471E4ABC
:1014F000D36943F00803D3610207520DC0F3031010
:1015000002EB401000F1804000F5A040D0F84421EB
:1015100061F30E32C0F844217047134A0021D269AA
:1015200012F0080F0DD00107490DC0F3031001EBB5
:10153000401000F1804000F5A040D0F84801C0F311
:101540000241084670470207520DC0F3031002EB38
:10155000401000F1804000F5A040D0F8482161F330
:101560001242C0F8482170470050004000389C1CCF
:101570001B81070089888888145100402051004051
:10158000042988BF704710B40023FD4CE26912F0B3
:10159000080F4FEA00724FEA5252C0F3031002EBF9
:1015A000401000EB04021CBFD2F84401C0F3023328
:1015B0000020D4F81CC01CF0080F1CBFD2F8480152
:1015C000C0F30240C91A0844042803DD081A011DAB
:1015D000042003E00028BCBF014400201944E36953
:1015E00043F00803E361D2F8443161F30E33C2F8EB
:1015F0004431D2F8481160F31241C2F8481110BCCE
:101600007047DF490028886914BF40F0080020F0C7
:10161000080088617047DA488069C0F3C0007047ED
:101620000207520DC0F3031002EB401000F180409E
:1016300000F5A040D0F8482161F30F02C0F848211E
:1016400070470107490DC0F3031001EB401000F192
:10165000804000F5A040D0F8480180B27047C84AE9
:10166000D2F8CC10022903D110F0010F18BF704737
:10167000D2F8400110F0010F08BF7047D2F84801BE
:10168000D2F844110304C1F302311B0C14BF00292A
:1016900070474FF6FF714840C2F848017047B84A9A
:1016A0000021D26912F0080F0DD00107490DC0F3D7
:1016B000031001EB401000F1804000F5A040D0F88D
:1016C0004801C0F30051084670470120704710B42C
:1016D000022ADDF804C026BF921E52080022022B07
:1016E00026BF9B1E5B080023A64CA4FB0C4C4FEAB4
:1016F0001C144FEA007C4FEA5C5CC0F303100CEB57
:10170000401000F1804000F5A040D0F854C161F3D2
:101710001B6C62F3134C63F30B2C64F3070CC0F8DF
:1017200054C110BC704770B40407640DC0F30310BB
:1017300004EB401000F1804000F5A040DDF80CC043
:10174000D0F854010029C0F30366C0F30345C0F389
:101750000324C0B218BF0E6012B16900891C116069
:1017600013B16100891C1960BCF1000F04BF70BC8B
:10177000704700EB80008000CCF8000070BC704720
:1017800070B491B000224FF480456C10EC4601E03B
:10179000082A05D2531C03EB8303B5FBF3F304E0E3
:1017A000D31F03EB8303B4FBF3F35B1A48BF5B4225
:1017B0004CF82230521C102AEAD30026009B01214B
:1017C0005CF821209A42BCBF13460E46491C1029E2
:1017D000F6D30107490DC0F3031001EB401000F1EF
:1017E000804101F5A041D1F85801D1F8582100F00D
:1017F0000F0066F30302C1F85821082807D2401CE5
:1018000000EB8000B5FBF0F011B070BC7047C01F5A
:1018100000EB8000B4FBF0F011B070BC7047010722
:10182000490DC0F3031001EB401000F1804000F5BA
:10183000A040D0F8580100F00F00082834BF401C29
:10184000C01F00EB800034BF4FF480414FF40051C3
:10185000B1FBF0F0704710F00F0F08BF70470007A2
:10186000400D00F1804000F5A0400029D0F824117F
:101870000CBF21F4803141F48031C0F8241170474D
:10188000002110F00F0F0BD00007400D00F1804039
:1018900000F5A040D0F8240110F4803F18BF0121CA
:1018A00008467047364AD2F8AC0011F0010FD2F862
:1018B000AC10C0F3C00014BF41F0080121F00801D2
:1018C000C2F8AC1070472E4A5067916770472C4998
:1018D0000028D1F8AC0014BF40F0020020F0020054
:1018E000C1F8AC00704726490028D1F8AC0014BFFD
:1018F00040F0010020F00100C1F8AC007047204822
:10190000D0F8DC0070471E49C1F8E00070471C4861
:10191000D0F89800704770B4194E0020D6F84011E6
:1019200011F0010F04BF70BC704711F0040FD6F81E
:101930001C3101F00805D6F800C1C3F308031FFAF3
:101940008CF4D6F844C1CCF3080C18BFC1F307409F
:10195000F269C1F3052112F008021CBFD6F8442138
:10196000C2F30232002D18BF491C0CFA02F201FB2F
:101970000200604370BCC3EB031100EB41007047F1
:1019800000500040CDCCCCCCFEF7D3BF10B5FEF755
:10199000D0FF012818BF10BD0020FEF77AFF2121DB
:1019A0000020FEF7CCFF2121BDE810400120FEF70A
:1019B000C6BF10B5FEF766FFFEF7BBFF01280AD1D0
:1019C0000020FEF766FF21210020FEF7B8FF21214D
:1019D0000120FEF7B4FF0121052001F06CFB01217D
:1019E000052001F068FBFC490020087110BD10B50E
:1019F0004FF4066001F0B5FBBDE810404FF40660FF
:101A000001F0A0BBF44A0146107B002818BF01205A
:101A1000002918BF012111737047EF4A516A5062C3
:101A200008467047EC490020C872887048707047BB
:101A3000E9490020C8728870487070470007C00EDE
:101A4000E64A801E02EBC0104FF4807213F0B4B966
:101A500070B50646FEF793FFE14D0446C6B1A201FC
:101A60003146284613F0A8F905EB841000210160E7
:101A700041608160C160016141618161C161016258
:101A800041628162C162016341638163C16370BD70
:101A9000800100F140012846BDE8704013F091B983
:101AA00010B5CD4CE061FFF7B0F9FFF78FF9A169F0
:101AB0006FF30F01A161A269C1B242EA0121A161E4
:101AC000022818BF10BDA06940F00100A06110BD40
:101AD000C4488168C44A114381600168521C1143A3
:101AE000016000F0D4BD2DE9F047BE4A0D46064620
:101AF0009368BD48184390601068BC490843106063
:101B000000F0C5FD0024002D6FD00020FEF7C1FEBF
:101B1000286820B1FEF75DFF0020FEF7BAFE3046D0
:101B2000FFF7BEFF0020FEF745FF002852D0D5F892
:101B30000480FEF724FFDFF8A89201260746B8F1DB
:101B4000000F1ED0BA014146484613F035F909EBA3
:101B50008710046044608460C460046144618461EF
:101B6000C461046244628462C46204634463846343
:101B7000C4639F48E96859B14FF4807213F01CF9AF
:101B800021E0800100F14001484613F01AF9F0E726
:101B9000984F4FF4807113F014F900203956002942
:101BA0000EDB0A09D20102EB800202F1405202F57B
:101BB000C0420907C90E136806FA01F11943116002
:101BC000401C2028EAD38C48696949B14FF48072DF
:101BD00013F0F2F80120FEF7EDFE804E50B905E05B
:101BE0004FF4807113F0EDF8F4E719E01120FEF7DF
:101BF000E1FE30B1A96821B130464FF4807213F094
:101C0000DBF80220FEF7D6FE18B91220FEF7D2FE4E
:101C100030B1296921B179484FF4807213F0CCF8C2
:101C20006D48C472847044704462017B002101736A
:101C30004FF4066001F095FABDE8F0474FF40660F6
:101C400001F080BA10B50020FEF723FE00F00CFD75
:101C50006148C078002808BF10BD6248016821F0C3
:101C6000030141F00D7141F080510160816821F064
:101C7000020141F00D7141F08051816010BD4FF4BF
:101C8000066001F064BA10B54FF4066001F05FFA27
:101C9000FEF74FFE01280AD10020FEF7FAFD2121B0
:101CA0000020FEF74CFE21210120FEF748FE54489B
:101CB000D0F8B01221F48031C0F8B0120020FEF745
:101CC000E8FD00F0D1FC4448C078002808BF10BDF2
:101CD0004448016821F0030141F00D7141F0805149
:101CE0000160816821F0020141F00D7141F08051E5
:101CF000816010BD10B501F02FFA10F0600018BF20
:101D0000012010BD3448C06970473348806970476E
:101D100072B631498A6922EA0000886162B670476A
:101D20002D480078002818BF0120704770B5FEF7D5
:101D300000FE002818BF70BD0024274DEC72AC7067
:101D40006C7021212046FEF7FAFD21210120FEF7CB
:101D5000F6FD2C70BDE870400120FEF79ABD70B50D
:101D60000446FEF7E6FD002818BF70BD00211A4D9D
:101D7000E972A970697021210020FEF7E0FD2121A0
:101D80000120FEF7DCFD022C3CBF0120FEF7E7FD41
:101D9000012028702C62BDE87040FEF77ABD10B5B6
:101DA000FEF7C7FD002818BF10BD00200A4CE072E6
:101DB000A07060702121FEF7C2FD21210120FEF7F5
:101DC000BEFD0120FEF7CBFD012020702062BDE8A2
:101DD0001040FEF75EBD00002804011040480030AE
:101DE0000040003000800040020034120300341232
:101DF00000600030D40801100080003040490030FD
:101E0000005000400020FEF744BDFF4900208870CC
:101E100048700120FEF73DBDFB4988627047FA48D3
:101E2000806A7047002000F068BB012000F065BBAD
:101E300010B5FFF764FD0446FFF765FDF348044263
:101E400008BF10BDF048816941F0040181610E2195
:101E500001EAD43104F001020A43816962F31F41AF
:101E60008161EB48016841F02001016010BD00284C
:101E700018BF0120E449C8707047E6487047E6483B
:101E80007047E148C06A7047DF484179C2799142A2
:101E900014BF006B406B7047DB48406B70472DE907
:101EA000F00FDC4E4FF0000C88B006F14007E14621
:101EB0004FF0FF3806F80C8007F80C900CF1010C7D
:101EC000BCF1200FF6DB4FF0000C002807DD12F804
:101ED0000C4006F80C400CF1010C6045F7DC0024C6
:101EE00022464FF0010A00280EDD16F902C0BCF1AF
:101EF000000F06DBBCF1200F3CBF0AFA0CFC4CEAD9
:101F00000404521C8242F0DB002294466D460AFA19
:101F100002FB1BEA040F1ABF05F802C00CF1010C0A
:101F200005F80280521C202AF1DB0022002810DD77
:101F300016F902C0BCF1000F08DBBCF1200F3ABF5C
:101F400015F80CC007F802C007F80280521C824244
:101F5000EEDBAD4C00220028C4F82C9008DD17F908
:101F600002C0944501D0E76202E0521C8242F6DBD7
:101F7000AA4F0020A7F1600CA7F120060CF8008002
:101F800006F8009007F80090401C2028F6DB00209F
:101F9000002905DD1A5C0CF80020401C8142F9DCA8
:101FA0000022104600290BDD1CF90030002B04DB59
:101FB000202B3CBF0AFA03F31A43401C8842F3DB90
:101FC000002003460AFA00FB1BEA020F1ABF2B543B
:101FD0005B1C05F80080401C2028F3DB0020002952
:101FE0000ADD1CF90030002B03DB202B3CBFEB5C2F
:101FF0003B54401C8842F4DB0020C4F83490002994
:1020000007DD3B56834201D0676302E0401C8842F3
:10201000F7DB11F0010F18BF1F2009D00AFA00F3F7
:10202000134203D10AFA00F0024301E0401EF5D545
:10203000002003460AFA00F717421ABF2B545B1C14
:1020400005F80080401C2028F4DB002000290ADD70
:102050001CF90020002A03DB202A3CBFAA5C325472
:10206000401C8842F4DB0020C4F830900029DEBF19
:1020700008B0BDE8F00F70473256824204D02663A4
:1020800008B0BDE8F00F7047401C8842F4DB08B090
:10209000BDE8F00F7047624900EB401001EB801083
:1020A000704700EBC0005F4900EB400001EB80008F
:1020B0007047DFF854C1012B8CF805008CF806102E
:1020C00003D9401C20F0010011468CF807008CF861
:1020D000081000FB01F24FF6FF7101EA4202ACF872
:1020E000122001EA4000ACF8140070474648007A1C
:1020F00070474548C0797047434A507291727047A3
:102100004148807A70474048407A7047464A10708C
:10211000517070474449085C70472DE9F047DFF87B
:10212000E890044699F80C00002804BF99F80100D3
:1021300012F04CFE99F80B00002808BFBDE8F087AC
:102140004FF00008D9F81C0047464646454610F0B7
:10215000020F1CBFDFF8C88010F0040F05D0B9F8DB
:1021600012102F4A21F001018F1810F0010F18BF33
:102170002C4E10F0200F18BF2C4DD9F828002060ED
:10218000FEF727FE10F0010F06D0FFF78BF80228AC
:1021900028BF99F8020000D20020E760C4E90108D6
:1021A000C4E904650120BDE8F08717490020C87222
:1021B000704710B50446FEF7E2FB82012046BDE8F9
:1021C00010401B4912F0F8BD2DE9F041FEF7D7FB96
:1021D00004460020FFF768F90022002C84BF012587
:1021E00041F6F07635D900214FEA821C05FA01F359
:1021F000034228D04B080CEB830303F1405303F553
:102200008043CF071B6815E0280401100100070078
:1022100064040110D4080110F408011054090110DD
:1022200074090110B4110110350401108C12011051
:1022300000400030FF0EFB40C3F30C03B34202D951
:102240000020BDE8F081491C2029CFD3521CA242B6
:10225000C9D30120BDE8F0810B460007C00EC54977
:10226000801E01EBC0114FF48072184612F0A4BD1D
:102270002DE9F05F00F00F0670000025A0F1020BC1
:10228000012741F6F07846EA05194846FEF792FB29
:10229000002835D04846FFF714F907FA00F4022C5D
:1022A00088BF02244846FFF7FFF80022002C84BFB5
:1022B0000BEB05014FEAC11A22D900210AEB821962
:1022C00007FA01F3034215D04B0809EB830303F12E
:1022D000405303F580434FEAC17CD3F840384FEABE
:1022E000DC6C23FA0CF3C3F30C03434502D9002042
:1022F000BDE8F09F491C2029E2D3521CA242DCD346
:102300006D1C022DBFD30120BDE8F09F2DE9F05FC9
:102310000026994C4FF6FF7500280F4644D000F078
:102320000F01C0F3031001290EBF00210229BDE8EF
:10233000F09F022828BFBDE8F09F01EB0009FEF7DF
:10234000F8FA5FEA00081CBF0020FEF7A2FA00209E
:102350004FEAC919002209EB8011530801EB8303EE
:1023600003F1405CD307DB0E0CF5804C05FA03FB50
:10237000DCF840A807FA03F32AEA0B0A4AEA030347
:10238000521CCCF84038202AE7D3401C0228E1D365
:10239000B8F1000F08BFBDE8F09FA6706670BDE8F9
:1023A000F05F0120FEF775BAFEF7C3FA5FEA000896
:1023B0001CBF0020FEF76DFA0020002281015308A7
:1023C00001EB83034FEAC27C03F140534FEADC6C1C
:1023D00003F5804305FA0CFAD3F8009007FA0CFCD9
:1023E00029EA0A0949EA0C0C521CC3F800C0202A49
:1023F000E5D3401C2128E0D3B8F1000FCDD1BDE8D2
:10240000F09F10B5FFF704F85B49088210BD5A4AE7
:10241000C1B200F4F853128A914288BF11464FF0BE
:10242000640C01FB0CF1B1FBF2F11A0A02FB0C1176
:1024300010F4005F12BF08B2484200B2704710B5F6
:102440004FF480714D4C4E4812F0BBFC002001232C
:102450002156002910DB0A09D20102EB800202F1A9
:10246000405202F5C0420907C90ED2F800C003FA73
:1024700001F14CEA01011160401C2028E8D310BD95
:1024800010B53E4C4FF480713D4812F09AFC00208C
:1024900001232156002910DB0A09D20102EB800238
:1024A00002F1405202F5C0420907C90ED2F800C03D
:1024B00003FA01F14CEA01011160401C2028E8D325
:1024C000BDE810404FF424612E4812F07ABC2A482F
:1024D00010B5808B00F48170FFF7E2FA4FF4807141
:1024E000274812F06EFC4FF40461264812F069FC94
:1024F000BDE810400020FEF7DBBE70B51E4C05465F
:10250000A06A401CA062207850B1206A10B1206AF5
:10251000401E2062206A002804BF0020FEF7B9F99F
:1025200020212846FEF70BFA616A00291CBF2846C5
:102530008847FEF74BFC022815D11348D0F8B81293
:1025400011F0010F0FD0D0F8B81241F00101C0F81E
:10255000B812D0F8B81221F00101C0F8B812A06981
:1025600040F00200A0610948016841F020010160CB
:1025700070BD00004048003028040110D40801104C
:102580000060003000400030005000406404011042
:102590002DE9F0410027634D0126002808BF2E7069
:1025A0001FD001282F7018BF6F701AD0DFF8788104
:1025B000D8F800005D490843C8F8000029785C4C51
:1025C000002914BF4BF608305A48E06014BF5A483F
:1025D0004FF0BB70A0605948006830F0FF0206D190
:1025E00001E06E70E2E7E26860F30302E26051B17D
:1025F000A06840F01800A060012000F071F8A06809
:1026000040F48050A060012000F06AF8687818B1AA
:10261000E06840F03000E060D4F8B00040F0010025
:10262000C4F8B000012000F05BF8E6674FF4E0600A
:102630002061C4F888702878002818BFC4F8946016
:10264000E06820F03000E060A06820F48050A060D6
:10265000D8F8000020F0040040F00D7040F08050E9
:10266000C8F80000BDE8F0813148C16821F03001B0
:10267000C160816821F4805181602B48016821F09C
:10268000040141F00D7141F080510160704726480E
:102690000268264911430160224925480A783AB167
:1026A000826842F018028260826842F4805282603E
:1026B000497819B1C16841F03001C160D0F8B0105B
:1026C00041F00101C0F8B01070471D49C0B241EAA5
:1026D000002017490864704715491A480864704774
:1026E00082B040F24C42009013E000BF00BF00BF38
:1026F00000BF00BF00BF00BF00BF00BF00BF00BFE2
:1027000000BF00BF00BF00BF00BF0198411E019184
:10271000EBD20098411E009128BF0192F5D202B081
:102720007047000060040110008000400400341273
:102730000060004005F401002000BB00D0FE030053
:1027400013005FA000005FA0414840498161891CDF
:10275000C161491E4163026822F0030242F00D721A
:1027600042F080520260426922F0010242F00D7292
:1027700042F0805242610269114301613549816032
:102780003549C160354900200860704710B501F037
:1027900064F932480468002C08BF30BFFAD0002129
:1027A000016001F05EF9204610BD10B501F055F949
:1027B00026482A4B2649421C1C682CB10020186070
:1027C00001F04FF9204610BD72B648638A6120BF00
:1027D00088614A6362B6BFF36F8FBFF34F8FEBE739
:1027E0001B48016821F0030141F00D7141F0805157
:1027F00001601B49816001691A4A1143016130BFC0
:10280000704772B6114912484163C91CC161891EE3
:10281000816162B670470E480168134A1143016036
:1028200070470B48016821F0030141F00D7141F040
:1028300080510160704772B6044905488161891C66
:10284000C161491E416362B6704700000000341246
:10285000008000403C00341228003412640401104F
:1028600008003412010034120300341270470028AB
:1028700018BF01204FF4E021486070470022B2EBFE
:10288000D10F26D20368B3F1FF3F04BF4368B3F111
:10289000FF3F17D18368B3F1FF3F04BFC368B3F1B3
:1028A000FF3F0FD10369B3F1FF3F04BF4369B3F1A9
:1028B000FF3F07D18369B3F1FF3F04BFC369B3F1A1
:1028C000FF3F01D0002070472030521CB2EBD10FE7
:1028D000D8D30120704710B40023B3EBD20F30D20D
:1028E000D0F800C00C68A44522D1D0F804C04C68D0
:1028F000A4451DD1D0F808C08C68A44518D1D0F8E3
:102900000CC0CC68A44513D1D0F810C00C69A44504
:102910000ED1D0F814C04C69A44509D1D0F818C024
:102920008C69A44504D1D0F81CC0CC69A44502D060
:1029300010BC00207047203020315B1CB3EBD20F5D
:10294000CED310BC012070472DE9F041054601F0BF
:102950008CF8002021264FF4825784464FF4E02261
:102960001660C5F800C0116841F0040111601168DB
:1029700011F0040FFBD1176040232C460021D4F83E
:102980000080B8F1FF3F04BFD4F80480B8F1FF3FE6
:102990001DD1D4F80880B8F1FF3F04BFD4F80C80F3
:1029A000B8F1FF3F13D1D4F81080B8F1FF3F04BF56
:1029B000D4F81480B8F1FF3F09D1D4F81880B8F1E9
:1029C000FF3F04BFD4F81C80B8F1FF3F08D0C2F825
:1029D00000C0401CC0B20828C2D30220BDE8F0816C
:1029E000491C2034B1EBD30FC9D3C2F800C0012079
:1029F000BDE8F0812DE9F041054601F036F80020F0
:102A0000092684464FF4E0231E60C5F800C019680B
:102A100041F004011960196811F0040FFBD12C4634
:102A20004FF4806200212768B7F1FF3F04BF676859
:102A3000B7F1FF3F17D1A768B7F1FF3F04BFE768C1
:102A4000B7F1FF3F0FD12769B7F1FF3F04BF6769B7
:102A5000B7F1FF3F07D1A769B7F1FF3F04BFE769AF
:102A6000B7F1FF3F08D0C3F800C0401CC0B2032834
:102A7000CAD30220BDE8F081491C2034B1EBD20F4B
:102A8000D1D3C3F800C00120BDE8F0812DE9F05F8B
:102A90000F46804604264FF0020A4FF0000B4FF419
:102AA000E02900F0E2FF44463846C9F800A00F21B3
:102AB000B0E82C10A4E82C10491EF9D2D9F8000077
:102AC00040F00400C9F80000D9F8000010F0040F2D
:102AD00006D000BF00BFD9F8000010F0040FF8D1F5
:102AE000C9F800B0454638460F21D5E90023D5E99D
:102AF00002C4D0F800E0964504BF42689A4205D16E
:102B00008268624504BFC268A24208D0761E03D321
:102B10004046FFF719FFC4E70220BDE8F09F1030E0
:102B20001035491EE1D20120BDE8F09F70B50D4679
:102B3000044600F09AFF4FF480722146284612F0B6
:102B40003BF9012070BD2DE9F041C0B014460E469E
:102B5000054610F0FF0F23D025F0FF086F4600F068
:102B600084FF4FF480724146384612F025F9E8B2EE
:102B7000C0F58077A74288BF274668443A46314669
:102B800012F029F94046FFF7DFFE022843D06946DC
:102B90004046FFF77BFF022841D03D443E44E41B02
:102BA000B4F5807F19D34FF480723146684612F035
:102BB00012F92846FFF7C8FE02282CD0694628469D
:102BC000FFF764FF02282AD0A4F5807405F580750C
:102BD00006F58076B4F5807FE5D2C4B16F4600F08B
:102BE00044FF4FF480722946384612F0E5F8224639
:102BF0003146684612F0EFF82846FFF7A5FE022896
:102C000009D069462846FFF741FF022807D040B0A7
:102C10000120BDE8F08140B00A20BDE8F08140B05D
:102C20000B20BDE8F08100002E490860086100F02B
:102C300010B82C490860486100F00BB82949486772
:102C40007047284988677047264801210166016559
:102C500070474FF04022116B10F0010F18BF21F4A4
:102C6000404110F0020F1CBF21F4405141F480514B
:102C700010F0040F18BF21F4406110F0080F18BFC6
:102C800041F4407110F0100F18BF41F0C00110F076
:102C9000200F18BF41F0300110F0400F18BF41F075
:102CA0000C0110F0800F18BF41F0030141F4BE0188
:102CB00041F020411163D2F8901010F4807F1CBFC6
:102CC00021F0030141F0020110F4007F1CBF21F04C
:102CD0000C0040F0080141F4BE0040F02040C2F872
:102CE00090007047001000407047D0488268D0497B
:102CF0000A438260C2681143C1604169CD4A1143F1
:102D000041617047C948416921F0010141F00D71ED
:102D100041F080514161C16821F0400141F00D71E5
:102D200041F08051C160816821F0400141F00D7196
:102D300041F080518160704710B5BC4CA168BC481F
:102D40000143A160E1680843E0606069B949084354
:102D50006061B94843F63F71C160002181638164BD
:102D6000C0F8B01003210A2000F0A5F90A2000F0F5
:102D7000C5F9606920F0010040F00D7040F080500E
:102D80006061E06820F0400040F00D7040F080503D
:102D9000E060A06820F0400040F00D7040F08050EE
:102DA000A06010BDA44A1060516048439060704715
:102DB000A14A10605160484310F0010F18BF401C39
:102DC000906070479C49C1F8B00070479A4900284C
:102DD00018BF01208864704797498863C86840F02D
:102DE0000200C8607047DFF850C2CCF82000CCF871
:102DF0002410CCF82820CCF82C300120CCF830005E
:102E0000DCF8340010F0010F05D020BFDCF83400EE
:102E100010F0010FF9D110F0020018BF4FF0FF3091
:102E200070478548C16821F00201C160704782483F
:102E3000C16841F00101C16070477F4B186259625F
:102E40009A6201201864586C10F0010F04D020BF62
:102E5000586C10F0010FFAD110F0060018BF4FF0B7
:102E6000FF3070477448C16821F00101C1607047AC
:102E70007148C16841F00401C1607047027C017B68
:102E800002F03F0241EA02416B4A916501685162DA
:102E9000416891628168D16201211165516D11F023
:102EA000010F04D020BF516D11F0010FFAD1D36D85
:102EB0008382D36D1B0CC382136E0383136E1B0CB2
:102EC0004383536E8383526EC2F30E42C28311F06A
:102ED000020018BF4FF0FF3070475748C16821F01B
:102EE0000401C16070475448C16841F00801C160E5
:102EF0007047DFF844C1CCF87820CCF82000CCF83B
:102F00002430CCF828100120CCF87000DCF87400D4
:102F100010F0010F05D020BFDCF8740010F0010F95
:102F2000F9D110F0060018BF4FF0FF30704742484B
:102F3000C16821F00801C160704701684FEA314261
:102F40003D49C1F89C204068C1F8A000C86840F025
:102F50002000C860704701684FEA31423649C1F825
:102F60009C208088C1F8A000C86840F02000C8609C
:102F70007047314B18625A6299620120C3F894007D
:102F8000D3F8980010F0010F05D020BFD3F89800B7
:102F900010F0010FF9D110F0060018BF4FF0FF300C
:102FA0007047254A106251620120C2F89000D2F8A1
:102FB000980010F0010F05D020BFD2F8980010F053
:102FC000010FF9D110F0060018BF4FF0FF30704725
:102FD0001948C16821F02001C16070471648C168D6
:102FE00041F01001C1607047A3F1050C124BC3F80A
:102FF00088C018625A6299620120C3F88000D3F831
:10300000840010F0010F05D020BFD3F8840010F029
:10301000010FF9D110F0060018BF4FF0FF307047D4
:103020000548C16821F01001C16070470080004070
:103030004000341201003412009000401B4810B5CB
:10304000022140F8501F012101611021416241F22B
:103050000601416100218161042181639021416366
:10306000416B41F0010141634FF4817101610161E4
:10307000032000F043F80021032000F01CF800209A
:1030800010BD10B5032000F045F808484FF48071DA
:10309000016600210166102181670221416500203F
:1030A00010BD034900200870704700000030004048
:1030B00068040110704700F00303DA004FF0FF0CC2
:1030C0000CFA02F24FF0050C0CEBC30301FA03F308
:1030D00000F00C0101F1E021002807DAD1F8140D0D
:1030E00090431A401043C1F8140D7047D1F8000402
:1030F00090431A401043C1F80004704700F01F01CC
:10310000012202FA01F14009800000F1E020C0F83C
:103110000011704700F01F01012202FA01F140097D
:10312000800000F1E020C0F88011704700F01F011E
:10313000012202FA01F14009800000F1E020C0F80C
:10314000801270474FF0E021C1F8000170474FF046
:10315000E021C1F8800170474FF0E020D0F8000175
:1031600070474FF0E021C1F88002704708480068BE
:103170007047074A1168106008467047044A126891
:1031800000F1100352F8230042F8231070470000AA
:1031900008ED00E002210C20FFF78DBFB8488268DF
:1031A000B8490A438260C2681143C1607047B4489D
:1031B000816821F4805141F00D7141F080518160AE
:1031C000C16821F4805141F00D7141F08051C1601E
:1031D0007047AD4881B0016F11F4007FFBD1816E63
:1031E00011F0010F1CBFD0F88410009104D0D0F86A
:1031F0008410009A9142FAD0016F11F4007F04BF4D
:103200004CF27101016642F24131816601B07047B2
:103210009D4981B04FF40D528A660A6FCA66012833
:1032200098BF012005D9401EB0F5803F28BF4FF65A
:10323000FF7082B24FF05C5040EA022048664FF0C7
:103240001140C1F88000086F10F4007FFBD1886E38
:1032500010F0010F1CBFD1F88400009004D0D1F809
:103260008400009A9042FAD0086F10F4007F04BFE7
:103270004CF27100086642F24130886601B0704736
:10328000814881B0016F11F4007FFBD1816E11F094
:10329000010F1CBFD0F88410009104D0D0F8841026
:1032A000009A9142FAD04FF40D51816601B07047F7
:1032B0007348806810F4805008BF70477248806E71
:1032C00000F0010070477048406EC0F30F20704757
:1032D0006D48D0F88400704710B50C20FFF726FF2A
:1032E0000C20FFF70BFF68490220486710BD6649B4
:1032F00010B5032088670C20FFF70CFFBDE81040D5
:103300000C20FFF713BF614A116810600846704730
:103310005D4810B5016FC1665C480068002818BFA1
:1033200080475B48016841F48051016010BD5748F7
:1033300040687047524810B5826852490A4382601B
:10334000C2681143C1605049032088670C20FFF711
:10335000E1FE0C20FFF7EAFE00F07EF94D4B042061
:10336000C3F888004FF6FF70C3F88C0072B6603364
:10337000FFF74EFF4FF40070186062B610BDF8B54D
:1033800072B64148016F11F4007FFBD1816E11F0DC
:10339000010F1CBFD0F88410009104D0D0F8841025
:1033A000009A9142FAD04FF40D51816639494FF499
:1033B00000320A6662B6D1F80412314D002946D0B7
:1033C000324C4FF6FF73591AA160AA69D5F81CC098
:1033D00002F00F020CF00F0C6244121D01FA02F20F
:1033E000A2F5EA41DFF8B0C0313961452FD2D0F8FB
:1033F0008400191AE160B1F5803F28D2274B4FF0C5
:10340000000CA1FB03070CFB037301FB0C316346AB
:1034100011F0E6FC401C40082061B0F57A7F38BF0F
:103420004FF47A701E4B9968002908BF98605A685B
:103430001A609968C3E901108A421BD9824205D9F2
:10344000814201D9616002E0606000E0626000F0EA
:103450000FF9A86820F4805040F00D7040F08050C3
:10346000A860E86820F4805040F00D7040F0805073
:10347000E860F8BD8242E9D88142E5D8E2E7000081
:10348000008000400010341200C000406C040110A5
:103490006404011000A000402F6E16000087930303
:1034A000D01201100F4881680F4A114381600F4804
:1034B000016841F404710160001F016841F00401DA
:1034C0000160016841F0100101607047084908601F
:1034D0007047BFF34F8F084906480860BFF34F8F0E
:1034E000FEE70000008000400400341214ED00E00C
:1034F00008ED00E00400FA050CED00E024488168C6
:10350000244A114381601003416941F00101416186
:10351000016A21F00F0220490A4302621F4B8A1EF2
:10352000C3F8C420016570474FF04020006900F0E7
:10353000700070474FF04020194940F8301F19497A
:103540004160194901661949416670474FF04021B1
:103550004868174A904202BF496C002915487047D5
:103560004FF04022516B032821F00F0128BF0120AA
:1035700041EA8001084340F4BE0040F0204050631F
:1035800070474FF04020406B00F00F007047000084
:10359000008000400400341203005FA0006000407F
:1035A000C0845FA055995FA00A005FA000005FA0E3
:1035B00061A5650561B66505022824BF0020704736
:1035C000DE4B53F8202043F820101046704770B5AA
:1035D000DB4C206FD94D10F0010F05D00120E066C3
:1035E0002868002818BF8047206F10F0020F08BF1E
:1035F00070BD0220E0666868002808BF70BDBDE8A5
:1036000070400047CF4810B58268CF490A438260B6
:10361000C2681143C160CA4902220A6501230B66D0
:103620000323CB664A65816821F0800141F00D716A
:1036300041F080518160C16821F0800141F00D713D
:1036400041F08051C1600920FFF758FD0221BDE81B
:1036500010400920FFF72FBDBA488268BA490A43D3
:103660008260C2681143C160B54902200865704795
:10367000B34902204865B348816821F0800141F0D8
:103680000D7141F080518160C16821F0800141F0ED
:103690000D7141F08051C1607047AA488068C0F345
:1036A000C0107047A648016F11F4007F14BF4FF49B
:1036B00040714FF480710166704710B5A04CE06F07
:1036C00010F0020F4FF0010018BF0320606700F0F8
:1036D00068F99C498A69C96902F00F02D04001F07B
:1036E0000F01C8400521B0FBF1F04FF4057100094E
:1036F000C4F880109549A1FB00104009C4F884006B
:10370000206F10F4007F14BF4FF440704FF48070AE
:10371000206610BD8A48016F11F4807F14BF4FF4FA
:1037200040714FF4007101667047854B30B4DA6F19
:1037300012F0010F14BF032202225A6700EB40056A
:10374000C5EBC0104FF49674C1EBC0004C4300EBC6
:1037500080007F4904EB4010A1FB00107949002252
:103760004FF0020C8C69C008C96904F00F0401F025
:103770000F012144C8400521B0FBF1F0B0F5803FB6
:1037800005D3511C4008CAB2B0F5803FF9D242EAD5
:103790000C2141F01001C3F88810C3F88C00186F99
:1037A00010F4807F14BF4FF440704FF4007018661F
:1037B00030BC70476248016F11F4003F14BF4FF4F2
:1037C00040314FF48031016670475D48016F11F45C
:1037D000803F14BF4FF440314FF400310166704711
:1037E0005748006FC0F3002070475548006FC0F382
:1037F0004020704753498968C1F3C011002904BFB4
:10380000002070474E4900280CBFD1F80002D1F8C3
:10381000040270474B4B9A68C2F3C012002A04BFDF
:1038200000207047464A00280CBFD2F88000D2F82A
:103830008800C0F30A200CBFD2F88020D2F888207C
:1038400002F00F02D3F818C0DB690CF00F0C03F084
:103850000F0363441A449140012202EB40004843A5
:103860003C49A1FB0010000970473B49012008704A
:10387000704770B4334BC1EB011149009A69D3F81A
:103880001CC002F00F020CF00F0C6244121DD1405C
:1038900008BF012104D0B1F5803F28BF4FF6FF716A
:1038A0009A68C2F3C012002A1CBF70BC7047D3F8DC
:1038B00008C0254A4CEA020CC3F808C0D3F80CC073
:1038C0004CEA0202DA601E4A4FF0020CC2F850C005
:1038D0004FF4003414660425C2F88850C2F88C10E6
:1038E0001E4DD566C2F874C01D4902283CBF134E58
:1038F00046F820100021184801704FF4007111663D
:10390000017819B920BF01780029FBD014669567AA
:10391000D566C2F854C0986820F0800040F00D7061
:1039200040F080509860D86820F0800040F00D7022
:1039300040F08050D86070BC7047000084040110D3
:1039400000A0004000800040800034121F85EB5131
:10395000CDCCCCCC8988888880040110020002027A
:103960001B5800004FF0E0210020886108611F49CA
:103970004860704710B54FF0E02460610020A061FE
:103980000221401EFFF797FB0720206110BD4FF07A
:10399000E02100200861704714480188491C01801B
:1039A00070471248806870472DE9F0410F4C00279E
:1039B00005462780A0684FF47A71B0FBF1F04FF014
:1039C000E026401E7061B7610221C81EFFF773FB3D
:1039D000072030612188A942FCD33761BDE8F0811E
:1039E0000349484301498860704700008C04011076
:1039F00040420F00704770B505464FF40D50040665
:103A0000A0660320E066264860664CF271002066DE
:103A10002448C4F8800042F24630A066022100200B
:103A2000FFF749FB0020FFF769FB002D08BF70BDC1
:103A3000A06E42F241310843A06670BD012110B56D
:103A4000880781674FF40D5181660020FFF762FB04
:103A5000BDE810400020FFF769BB012081074867DF
:103A6000704701208107886770474CF27100810719
:103A7000086670470C4A11681060084670470A488B
:103A800008B5006818B18047002818BF08BD4CF27F
:103A9000710188070166016FC166006F009008BD63
:103AA00007383937009C1C919804011070B5FF4EFF
:103AB00000244FF4A061347074703471FC4811F02C
:103AC00080F94FF4A061FB4811F07BF9FA4DB46026
:103AD00074712C606C60AC60EC602C616C61AC61EA
:103AE000EC612C626C62AC62EC622C636C63AC6364
:103AF000EC632C646C64AC64EC642C656C65AC6544
:103B0000EC652C666C66AC66EC662C676C67AC6723
:103B1000EC67B471682105F1800011F052F9682159
:103B200005F1E80011F04DF9F460F471C5F8B84101
:103B3000C5F8BC41C5F8C041C5F8C441C5F8C84185
:103B4000C5F8CC41C5F8D041C5F8D441C5F8D84135
:103B5000C5F8DC41C5F8E041C5F8E441C5F8E841E5
:103B6000C5F8EC41C5F8F041C5F8F441C5F8F84195
:103B7000C5F8FC41C5F80042C5F80442C5F8084242
:103B8000C5F80C42C5F81042C5F81442C5F81842F1
:103B9000C5F81C42C5F82042C5F82442C5F82842A1
:103BA000C5F82C42C5F83042C5F83442C5F8384251
:103BB000C5F83C42C5F84042C5F84442C5F8484201
:103BC000C5F84C42C5F85042C5F85442C5F85842B1
:103BD000C5F85C42C5F86042C5F86442C5F8684261
:103BE000C5F86C42C5F87042C5F87442C5F8784211
:103BF000C5F87C42C5F88042C5F88442C5F88842C1
:103C0000C5F88C42C5F89042C5F89442C5F8984270
:103C1000C5F89C42C5F8A042C5F8A442C5F8A84220
:103C2000C5F8AC42C5F8B042C5F8B442346170BDC5
:103C30009E490020487070479C48407870479B48D8
:103C40004079002818BF012070479848C0790028A3
:103C500018BF0120704795488079002818BF0120BF
:103C6000704792480079002818BF01207047002152
:103C70009148C0F87812C0F87C12C0F88012C0F8E1
:103C80008412C0F88812C0F88C12C0F89012C0F8E4
:103C90009412C0F89812C0F89C12C0F8A012C0F894
:103CA000A412C0F8A812C0F8AC12C0F8B012C0F844
:103CB000B412704781487047814A014681481378A1
:103CC00052781A44520011F086B870B57C4A054605
:103CD000107851784218520014462946774811F05E
:103CE0007AF822462946784811F075F86F49012084
:103CF000C87170BD6D48006970476C48407800EB32
:103D0000800101EBC000714901EBC00070472DE953
:103D1000F041664D04466D496A786D4F02EB8200B2
:103D200000EBC2006B4E01EBC0033A7830782146BD
:103D300010444200184611F04EF86A78664902EBCA
:103D4000820000EBC20001EBC0033A7830782146D4
:103D500010444200184611F03EF80120A871BDE859
:103D6000F0815248C068704750485149407800EB94
:103D7000800001EB002070472DE9F0414B4E0746D3
:103D80003078002814BF55485548047814BF55486A
:103D90005548057804FB05F8FEF7A7FF294620469D
:103DA000FFF700F87078434C00EB800004EB002232
:103DB000A4F5A06101EB00203B460146FFF713F894
:103DC000FEF7A0FF70784FEA480200EB800004EB9A
:103DD0000020394610F0FFFF01203071BDE8F0816E
:103DE0002DE9F047314D044631496878DFF8EC8021
:103DF00000EB800001EB002C2878DFF8E490394ECE
:103E0000394F2146002815BF98F8002099F8002066
:103E100033783B7802FB03F04FEA4002604610F033
:103E2000DAFF6878234900EB800001EB002C28784A
:103E30002146002815BF98F8002099F80020337813
:103E40003B7802FB03F04FEA4002604610F0C3FFEC
:103E500001202871BDE8F08714488068704770B56C
:103E6000224C0546014622781348520010F0B3FF59
:103E70002278294652001E4810F0ADFF0B49012060
:103E8000487170BD2DE9F04FADF24C5DDFF81C902C
:103E90000120CDF82C0599F80400CDF8280599F8F3
:103EA0000500CDF8240599F8060023E09C040110D4
:103EB000DC120110DC170110DC260110942801101F
:103EC000DD04011014290110D42801105C27011011
:103ED000DA040110DB040110C4270110D80401101A
:103EE000D5040110D9040110D6040110DC0401101E
:103EF0001C270110CDF8200599F80700CDF81C0506
:103F000001F020FC8046FDF73FFDCDF84405FDF7AC
:103F100007FFCDF84005FDF7D5F9CDF83C05FCF7D6
:103F200058FF0446FCF752FF0646FDF72FFD99F8AF
:103F300002001E270025002804BF0420C9F818002D
:103F400008D0B8F1020F18BF0A200ED0C9F8180027
:103F500089F80250FDF77CF9083000094FF0010B99
:103F6000CDF83005022E0AD01EE010F03EFF10F40E
:103F7000817F14BF0F20C9F81870E7D1E8E7B8F1C6
:103F8000020F06D0B8F1050F08BFC9F8187009D0A4
:103F90000AE04FF47A7141434FF47A7091FBF0F0EC
:103FA000C9F8180089F802B0D9F818000428BCBF75
:103FB0000420C9F8180099F80200B9F81810000296
:103FC00040EA014040F001020023912107200AF05D
:103FD0005DF914F0010F05D0FDF7A8FE0020CDF823
:103FE0002C0504E00020FDF763F9FDF7D8FE10F082
:103FF00001FF00263746CDF8186505F035FE01288B
:104000001CD00DF5A060FEF788F8002800F0EE82C5
:104010000DF5A06006F011FD002089F80100D9F827
:104020001800C01E8642CABF874201250025DDF860
:104030000C05B8B3DDF8240528B133E00120CDF834
:10404000180500F0BDBA6846DDF80C1510F0D7FE73
:1040500082467DB1FE4C514620784200FD4810F06A
:10406000BAFE207851464200FB4810F0B4FE89F8B1
:1040700005B017E0FEF739FEF54C01212078FEF778
:1040800091FEF54A5346A2F140010846FEF7ABFE09
:10409000FEF738FE207851464200EF4810F09BFEB4
:1040A00089F805B0DDF80805002800F0CE80DDF8BD
:1040B000280500287ED199F80000DDF80845E0BB0E
:1040C000D9F808A0BAF1000F24D0E4480078CDF860
:1040D0003805E3480078CDF83405FEF706FEDDF834
:1040E0003415DDF83805FEF763FE214652460846D2
:1040F000FEF7A3FEFEF706FEDA480078022804BFAA
:10410000504606F07DF9D7480078092804BF2046BC
:1041100006F076F9D4480078012816D9DFF844A3D0
:104120009AF80000042804BF204606F069F92146E9
:10413000684610F069FE044600E006E09AF80000C8
:10414000052804BF204606F05BF9A5B399F80100E5
:1041500099F8002000EB8001C448002A00EB012000
:1041600021460CBFC24ABD4A137814BFBC4AC14A9B
:10417000127803FB02F24FEA420210F02CFE99F88B
:10418000010000EB8001BC4800EB012399F800001E
:104190002146002814BFB148B548007814BFB04A82
:1041A000B44A127800FB02F04FEA4002184610F0C1
:1041B00012FE01E049E002E089F804B038E0CDF8F1
:1041C000344599F80000002814BFA448A84890F886
:1041D00000A014BFA248A74804780AFB04F0CDF859
:1041E0003805FEF782FD21465046FEF7DBFD99F8C3
:1041F0000100A14C00EB800004EB0022A4F5A061BB
:1042000001EB00200146DDF83435FEF7ECFDFEF74A
:1042100079FDDDF83805DDF83415420099F8010024
:1042200000EB800004EB002010F0D5FD89F804B00D
:104230008C480078032808D199F8010000EB800130
:104240008A4800EB012006F0DBF8DDF810050028B5
:104250007DD0DDF82005002879D199F80000DDF83F
:10426000104548BBD9F80CA0BAF1000F24D0834800
:104270000178834800780844401C400801900220DF
:104280000090FEF732FDDDE90010FEF791FD2146BA
:1042900052460846FEF7D1FDFEF734FD7948007816
:1042A000022804BF504606F0AFF976480078092886
:1042B00004BF204606F0A8F94DB399F80100DFF8D5
:1042C000BCA100EB800101EBC0016F489AF800200F
:1042D00000EBC1036A4821460078104442001846AA
:1042E00010F079FD99F80100654A00EB800101EBBF
:1042F000C00166489AF80030127800EBC1001A44F9
:104300002146520010F067FD89F806B030E05B48A6
:10431000009401785A4800780C18FEF7E6FC601CFF
:1043200040080221FEF73EFD99F80100DFF85CA18C
:1043300000EB800101EBC000AAF168010AEBC002AA
:1043400001EBC0010846009BFEF74DFD00E01EE0BA
:10435000FEF7D8FC99F80100620000EB800101EB48
:10436000C0000AEBC000009910F035FD89F806B0D6
:104370004448007803280AD199F8010000EB800135
:1043800001EBC001404800EBC10006F03DF9DDF84B
:10439000140500285AD0DDF81C0530B1B8F1020F21
:1043A00018BFB8F1050F52D0FDE099F80000DDF814
:1043B000144540BBD9F810A0BAF1000F23D03448FF
:1043C000017840780844401C400801900220009089
:1043D000FEF78BFCDDE90010FEF7EAFC21465246B1
:1043E0000846FEF72AFDFEF78DFC2A4800780228D1
:1043F00004BF504606F027FA26480078092804BF73
:10440000204606F020FADFF888A09AF800009AF813
:1044100001100844401C42082146084610F0F9FCEF
:104420001C480078332804BF204606F00CFAADB3D0
:1044300025469AF800009AF80110084444002246E4
:104440002946154810F0C7FC224628E0ABE081E081
:10445000DC040110DC2601101C270110D804011017
:10446000D904011055050110D7040110DC12011008
:10447000D5040110D6040110DC170110DA04011074
:10448000DB0401105A0501105C270110C42701103C
:10449000DD0401105F0501109428011006E0294693
:1044A000FE4810F098FC89F807B025E09AF8000063
:1044B0009AF801104518FEF718FC681C4008022104
:1044C000FEF770FCF54A2346A2F140010846FEF7CC
:1044D0008AFCFEF717FC6A002146F04810F07BFCCE
:1044E00089F807B09AF800009AF8011008444200D1
:1044F0002146EB4810F06FFCEA480078032804BF1F
:10450000E94806F0A0F910F089FCE8490020C1F85C
:104510007802C1F87C02C1F88002C1F88402C1F8B7
:104520008802C1F88C02C1F89002C1F89402C1F867
:104530009802C1F89C02C1F8A002C1F8A402C1F817
:10454000A802C1F8AC02C1F8B002C1F8B40200F090
:10455000B8FE28E00021DDF8140510F064FCDDF859
:104560003005782828BF16F0010F1CD0D04C207AD7
:1045700058B10820FCF71CF9CE4A137852789918E4
:104580004A0001460820FBF7CFFEE07958B107202A
:10459000FCF70EF9C74A01460720137852781A44EF
:1045A0005200FBF7C1FEFDF700FED9F81800761C9B
:1045B0007F1C8642A8BF874211DBD9F8140070B176
:1045C000FDF7E4F9DDF83C05FCF772FEDDF8440583
:1045D00088B1DDF8400560B1FDF7E1FB0BE0DDF8E7
:1045E0002C05002818BFFDF7DAFB06E501F0F7F807
:1045F00003E5FDF79BFBDDF81805002804BF042048
:10460000C9F818000FD0DDF8280589F80400DDF896
:10461000240589F80500DDF8200589F80600DDF895
:104620001C0589F80700DDF81805B9F81810000214
:1046300040EA014200239121072009F027FEDDF81E
:1046400018050DF24C5DBDE8F08F70B50024FDF744
:1046500059FB994E054610F0020F0AD03079002818
:1046600008BF012415F0040F03D07079002808BF9B
:10467000012415F0010F07D001F064F8052803D0DC
:10468000B079002808BF012415F0200F03D0F0797D
:10469000002808BF01240020002C08BF70BD0020A6
:1046A0003070BDE87040FFF7EDBB38B505460F240C
:1046B00010F09BFB40B101F045F8022803D001F057
:1046C00041F8052800D10E242146284601F04FF973
:1046D000012804D1FFF7B9FF009001F0BBFA76483A
:1046E000017900291CBF8179002906D0C1790029F0
:1046F0001FBF40790028012038BD002038BDD4E715
:10470000704770B56C4D00242C716C71AC71FCF766
:10471000ADF8002818BFEC71BDE870400AF0A4BAEB
:1047200010B54FF4A061654810F04BFBBDE8104098
:104730004FF4A061624810F044BB62487047624881
:10474000017862480078484341005E4810F039BB68
:1047500070B506465C4804785C480578FEF7C5FAF3
:1047600029462046FEF724FB53485449407800EB85
:10477000800001EB002231465248FEF75EFBFEF757
:10478000C1FA53480078152818BF70BD4D48BDE8E0
:10479000704005F035BE002818BF01204649087159
:1047A000704710B5444C002804BFA06010BDDFF86E
:1047B00024C149490B7849490A7801465A435200B5
:1047C000604610F008FB4348A06010BD3749002048
:1047D000086048608860C860086148618861C86195
:1047E000086248628862C862086348638863C86375
:1047F000086448648864C864086548658865C86555
:10480000086648668866C866086748678867C86734
:10481000704726487047002818BF01202649487174
:10482000704710B568212E4810F0CBFABDE8104053
:1048300068212C4810F0C5BA002818BF01201E4975
:104840008871704710B51C4C002804BFE06010BD93
:1048500068220146244810F0BEFA2348E06010BDEB
:1048600012490020C1F8B801C1F8BC01C1F8C0016B
:10487000C1F8C401C1F8C801C1F8CC01C1F8D00128
:10488000C1F8D401C1F8D801C1F8DC01C1F8E001D8
:10489000C1F8E401C1F8E80128E00000D4280110C3
:1048A000142901105F05011094280110DC26011065
:1048B00008080110DD0401109C040110DC12011035
:1048C000DC170110DC1C0110D5040110D604011006
:1048D00055050110DC210110D8040110D904011084
:1048E0005C270110C42701102C280110C1F8EC012D
:1048F000C1F8F001C1F8F401C1F8F801C1F8FC01F8
:10490000C1F80002C1F80402C1F80802C1F80C02A3
:10491000C1F81002C1F81402C1F81802C1F81C0253
:10492000C1F82002C1F82402C1F82802C1F82C0203
:10493000C1F83002C1F83402C1F83802C1F83C02B3
:10494000C1F84002C1F84402C1F84802C1F84C0263
:10495000C1F85002C1F85402C1F85802C1F85C0213
:10496000C1F86002C1F86402C1F86802C1F86C02C3
:10497000C1F87002C1F87402C1F87802C1F87C0273
:10498000C1F88002C1F88402C1F88802C1F88C0223
:10499000C1F89002C1F89402C1F89802C1F89C02D3
:1049A000C1F8A002C1F8A402C1F8A802C1F8AC0283
:1049B000C1F8B002C1F8B4027047002818BF012046
:1049C000F949C871704710B5F74C002804BF206141
:1049D00010BDF6490A78497811444A000146F44866
:1049E00010F0F9F9F248206110BDEF48C0780028B6
:1049F00018BF01207047002818BF0120EA49C8707D
:104A00007047EC487047EC487047E84A0146EA486E
:104A1000137852781A44520010F0DDB930B44FF0D8
:104A2000000C029C634304BF30BC704732F91C4049
:104A300051F82C502C4440F82C400CF1010C6345EB
:104A4000F4D830BC7047002B08BF704710B4DDF8B5
:104A500004C0BCF1000F4FF0000C11D0002A9CBF25
:104A600010BC704751F82C4004EB5304B4FBF3F432
:104A700020F81C400CF1010C6245F3D810BC7047C3
:104A8000002A9CBF10BC704751F82C4094FBF3F4F3
:104A900020F81C400CF1010C6245F5D810BC7047A1
:104AA00070B5C14D002604462E716E71AE71FBF7D4
:104AB000DDFE002818BFEE710AF0D6F8002C14BFF6
:104AC000012000202870BDE87040FFF7DBB92DE918
:104AD000F04FA9B04FF4A061B84810F072F9682106
:104AE000B74810F06EF9B7480021C0F8B812C0F806
:104AF000BC12C0F8C012C0F8C412C0F8C812C0F886
:104B0000CC12C0F8D012C0F8D412C0F8D812C0F835
:104B1000DC12C0F8E012C0F8E412C0F8E812C0F8E5
:104B2000EC12C0F8F012C0F8F4128021684610F0C0
:104B300048F9FDF7E7F80446FCF726FF2890FDF753
:104B4000EFF82790FCF7BEFB2690FCF71FFF002034
:104B5000FCF7AEFBFDF723F90026354605F084F897
:104B6000012875D020A8FDF7D8FA00287DD020A80C
:104B700005F063FF14F0020F1CD09348DFF83CB23D
:104B8000DDF8889090F800809048DA460778FEF7C4
:104B9000ACF80120FEF71AF939464046FEF708F94D
:104BA000524649465846FEF748F90020FEF70EF9EE
:104BB000FEF7A8F814F0010F20D08548DFF800B206
:104BC0004FF0020801788348DA46DDF890900078CB
:104BD0000844401C4708FEF788F80120FEF7F6F865
:104BE00041463846FEF7E4F8524649465846FEF735
:104BF00024F90020FEF7EAF8FEF784F814F0200FFD
:104C00001CD06A496B46022791F800C04978259864
:104C10006144491C4FEA510C00211A465FEA4C08D6
:104C200018BF0CFB07FC09D030F9117052F8218035
:104C3000474443F82170491C8C45F5D8FDF7B5FA77
:104C4000761C102E05D2FDF7AAF887E700E00CE0ED
:104C50000125FCF79BFE2698FCF72AFB289848B113
:104C6000279828B1FDF79BF804E000F0B8FD75E740
:104C7000FDF75CF8002D59D1DFF82CC114F0020FBC
:104C80001BD051484D4E017850483746007801FB03
:104C900000F210200021002A88BF03460AD937F904
:104CA000118008EB5008B8FBF3F826F81180491C76
:104CB0008A42F4D84148CCF8080014F0010F19D00A
:104CC00043483F4B017843481E4600780A184FF08E
:104CD00010004FF000010AD036F9118008EB50089F
:104CE000B8FBF0F723F81170491C8A42F4D8344815
:104CF000CCF80C0014F0200F18D02C482C4B6C462C
:104D0000017840780A184FF010014FF000000AD0E7
:104D100054F8206006EB5106B6FBF1F623F810605C
:104D2000401C8242F4D82248CCF8100029B0284612
:104D3000BDE8F08F0120704727487047264800687B
:104D4000704725490A68B2F1FF3F15D0052804BF16
:104D5000C87A704742DC012804BF087970470228EE
:104D600004BF087A7047032804BF487A70470428B4
:104D700004BF887A704741E0052813D007DC01287A
:104D80003CD002281CBF032804280BD036E014288E
:104D900012BF15282D207047162804BF2820704701
:104DA00017282BD1002070479C040110DD0401104E
:104DB000942901101429011054290110DC2101103B
:104DC0002C280110DC260110D8040110D904011090
:104DD000DA040110DB04011000AE0200142804BF45
:104DE000087B7047152804BF487B7047162804BF0E
:104DF000887B7047172804BFC87B7047FF20704727
:104E000030B5C1B000244FF4807168460FF0D9FF6F
:104E1000FF22D14D511C684610F00AF8FF212246AE
:104E200061F307022D23214663F3070163F30F218A
:104E300028234BF6BB3063F3174164F31F61CDE9C0
:104E40000002CDE9024104942846FDF77DFD694644
:104E50002846FDF71BFE41B030BD2DE9FF4FDFF8BE
:104E6000F882C1B08346D8F800004E9F91468A462A
:104E70004446B0F1FF3F08BFFFF7C2FFD4E901107D
:104E80006BF307018B466AF30700449969F30F201F
:104E900061F317402568D4E9036467F31F60074690
:104EA000FF22511C68460FF0C3FF0297CDE903644F
:104EB000CDE9005B4046FDF747FD69464046FDF7FA
:104EC000E5FD012818BF002045B0BDE8F08F2DE9B1
:104ED000F74FDFF8849283460020D9F80060C0B015
:104EE0008A464C46B6F1FF3F04BF43B0BDE8F08FA1
:104EF000D4E902856768FF22511C6846D9F8104042
:104F00000FF096FF6BF3070542986AF30F2560F3E5
:104F10001745012060F31F65CDF80880CDE90354E3
:104F20004846CDE90067FDF70FFD69464846FDF7A5
:104F3000ADFD43B0BDE8F08F2DE9F04F8648874EB8
:104F400000250368C1B074422F461720FFF7F9FE11
:104F500084461420FFF7F5FE40B2B3F1FF3F04D0C2
:104F6000BCF1000F03D12D2801D0FFF749FF142019
:104F7000FFF7E7FE40B202901520FFF7E2FE4FFA7E
:104F800080F91620FFF7DDFE40B201901620FFF7F2
:104F9000D8FE404240B20090FCF7B4FEDFF8C0A15A
:104FA000834600208AF804008AF805008AF8060083
:104FB000FBF75CFC00281CBF00208AF8070009F002
:104FC00053FE00208AF80000FEF75CFF1BF0010F83
:104FD00004D00FF032FF012808BF01251BF0020F9B
:104FE0007ED060489AF80110604A90F800C05E4890
:104FF00001EB810102EB012200784FF0000800284C
:10500000C8BFACF1010A1EDD0021BAF1000F16DDA8
:1050100001F1010B01FB00830BFB008B32F8133015
:1050200032F81BB0A3EB0B031BB2002BB8BF5B42E3
:105030001BB2BB42C8BF1F46491C5145E8DB08F103
:1050400001088045E0DBB945B8BF45F002054FF0E7
:105050000008C146BCF1000FC8BFA0F1010A1BDD6A
:105060000021BAF1000F13DD09FB001332F813B071
:1050700002EB43035B88ABEB03031BB2002BB8BF0F
:105080005B421BB24345C8BF9846491C5145EBDB08
:1050900009F10109E145E3DB02994145B8BF45F05B
:1050A00004054FF00009BCF1000F13DD00230028B8
:1050B0000CDD09FB003132F91110B142C8BF0E46B8
:1050C000A142B8BF0C465B1C8342F2DB09F1010927
:1050D000E145EBDB0198B04204DB0098A04200E020
:1050E00002E001DD45F0080560421B4C08F0FF0BB3
:1050F00000F0FF08206807F0FF0A06F0FF09B0F192
:10510000FF3F08BFFFF77CFED4E901106BF30700F7
:105110006AF30F20266869F31740D4E9037465F336
:10512000070168F31F600D468046FF22511C684648
:105130000FF07EFECDF80880CDE90374064CCDE972
:1051400000652046FDF700FC69462046FDF79EFC01
:1051500041B0BDE8F08F000000AE0200F1D8FFFFC3
:105160009C040110D6040110D5040110DC120110BA
:10517000FF4920F07E4008617047FD480069704794
:10518000FB4880897047FA48C089704770470843D8
:1051900018BF7047F648006910F0807F1CBF0020E0
:1051A000107070472DE9FF5F8346F2480027DDF855
:1051B00038A005780398109EB9463C4650452CD03F
:1051C00006FB050E0F983BF91EC006FB05093BF9CF
:1051D0001900BCEB000348BFA0EB0C0306FB05A8BD
:1051E0003BF91840B4EB000C48BFA0EB040C03EBF8
:1051F0000C0004B231F91EC031F91900BCEB0003F8
:1052000048BFA0EB0C0331F918C0BCEB000148BF4C
:10521000A0EB0C0158180FFA80F9012A2DD04FF09D
:1052200001080FF00FFED449002C0A782EDD0F99EB
:1052300006FB05113BF911101431282926D90399D1
:1052400002EB0A0C11448C4520D9119B129D13448A
:105250002A448B421CBF8D1A15F1020F30F91150F0
:1052600000EB4106B6F90260A5EB060508D01E3535
:105270003C2D08D94FF0000808E0A1450CDD0AE0FC
:105280000A35142DF6D8491C8C45E2D8A14503DD1A
:10529000B8F1000F00D0012704B03846BDE8F09FF8
:1052A000B64A0280428000218280C180018153423F
:1052B00043818181C181018241828182C1820283D5
:1052C0007047AB49002048618021AD480FF079BD9F
:1052D000AC480021016041608160C16001614161B1
:1052E0008161C161016241628162C16201634163A6
:1052F0008163C1637047A3487047A34A0146A14830
:10530000137852781A4452000FF065BD2DE9F04F22
:1053100091B00C460546FFF776FB0646DFF864823F
:105320000FF095FD924F14203C23D7F814B00A22B9
:1053300084464FF00509BBF1000F09D10021002C74
:1053400006D935F811A028F811A0491C8C42F8D8CC
:105350000021002C0AD935F811A038F811E0AAEB89
:105360000E0A2DF811A0491C8C42F4D8CB4524BF5D
:105370000021002C22D9DFF80892C0F10008EA468B
:105380004FF0000B35F911009842B8BF49F821B031
:1053900011DB59F82100401C49F8210090420AD93C
:1053A0003AF91100404506DD604504DC36F811E0AD
:1053B000704426F81100491CA142E3D33046FFF7A0
:1053C00024FB786942F2107188423ABF401C786130
:1053D00079616D4829460278407810444200694856
:1053E0000FF0F9FC11B0BDE8F08F6148007800289B
:1053F00018BF0120704710B54FF4A06163480FF04B
:10540000E0FC4FF4A06162480FF0DBFC584900203B
:10541000087010BD70B504460FF01EFD55490123FC
:10542000062209784FF0090C02FB013230F91250C4
:10543000142DD8BF70BD00EB4202B2F90220142A2D
:10544000A8BF70BD0CFB013130F91120142AD8BF60
:1054500070BD00EB4100B0F902001428A8BF70BD78
:105460004FF0FF3020604248437170BD2DE9FF4F7F
:1054700085B09846DDE913A691460446DDF848B0AC
:1054800009F0D2FB09F001FC0025394F002840F05B
:10549000E48000F057F9052800F0DF800698CDE998
:1054A00002060A2004903B481E26007800903248ED
:1054B00000780190B88910B9787801281FD109F0D7
:1054C0001EFCE0B9BAF1010F19D0BBF1010F02D1F6
:1054D000F889C82813D8F889002804BFB88900289B
:1054E0000DD009F0BEFB01280BD0DDE90021002022
:1054F000521812D0029931F91010B14209DDFD7134
:105500001BE0052004900398012814BF28263226AA
:10551000EBE7401C80B28242ECD8386910F4803F3F
:105520000BD0F879401CC0B2F8710499884204D9B4
:10553000012078714FF0FF34FD7109F092FB0128D2
:1055400042D1BBF1000F40DCBAF1010F3DD0386908
:1055500010F4003F0AD0B879401CC0B2B8710A28D4
:1055600004D9012078714FF0FF34BD710A2013E097
:10557000B8040110D5040110DB040110F1D8FFFFBD
:10558000142A0110D4290110DD040110942F0110F8
:10559000942A0110DA04011001905F48002690F867
:1055A00000B05E4890F800A01E2000900FF059FC5B
:1055B00001460020AAF1010CBCF1000F17DD31F902
:1055C00010201E2A03DD3D7247E0BD71CEE701EBDE
:1055D0004003B3F90230002BB8BF002A03DAD21A15
:1055E000B242C8BF16B2401C80B26045E7DB31F959
:1055F00010001E28E7DC0AEB0B00431E534515DDA7
:1056000031F91A001E28DEDC01EB4A02B2F9022051
:10561000002AB8BF002803DA801AB042C8BF06B219
:105620000AF101001FFA80FA5345E9DC31F91A004A
:105630001E28C8DC386910F4002F0ED0009886426E
:10564000C1DD387A401CC0B238720199884204D951
:10565000012078714FF0FF343D72B4F1FF3F28D044
:10566000002C07BFF878012809B0BDE8F08FFD7065
:105670004FF4A0612A480FF0A4FB4FF4A061294821
:105680000FF09FFB3D7000F063F8042832D0B9F1B1
:10569000000F1CBF4846FEF7A3FBB8F1000F04BF84
:1056A00009B0BDE8F08F404609B0BDE8F04FFEF705
:1056B0002EBB787901281CBF09B0BDE8F08F4846A1
:1056C000FFF746F87D714FF4A06115480FF079FBA4
:1056D0004FF4A06113480FF074FB3D70B9F1000F57
:1056E0001CBF4846FEF77CFBB8F1000FDBD109B0C8
:1056F000BDE8F08FB9F1000F1CBF4846FEF73CFB38
:10570000B8F1000F04BF09B0BDE8F08F404609B002
:10571000BDE8F04F0FF0AABBDA040110DB04011062
:10572000942F0110942A011010B506F01DFB06F00D
:10573000C6FB002010BD0000F94988707047F8488A
:1057400080787047F64800787047F5484078704791
:10575000F3480078022805D005281CBF00207047B8
:1057600005F0A1BB09F060BAED490870704770B54B
:10577000EB4E04460D463078A04212D002281AD0D3
:10578000052814BF002005F08EFB44EA052132787D
:10579000002341EA024141EA00626121072008F04A
:1057A00075FD7570072C28BF70BDDFE804F0160783
:1057B0000B13160F160009F037FAE6E7284600F03B
:1057C00055FA0AE0284609F0D2FA06E0284605F024
:1057D0005FFB02E0284608F011FE347070BDD1492D
:1057E00000200968B1F8641011F4807F08BF704789
:1057F000FCF7CCBFCB4900200968B1F8641011F464
:10580000807F08BF7047FCF7D0BFC64900200968F9
:10581000B1F8641011F4007F08BF70470FF02BBB84
:10582000C04900200968B1F8641011F4806F08BF06
:1058300070470FF025BBBA49C87800281CBF401E2E
:10584000C870704770B5B849D1F8CC00B44C10F0AE
:10585000030F0AD040F4BE0040F02040C1F8C80059
:10586000E078002804BF0120E070B0488068AD4DAA
:1058700010F0020F296807D14FF04020406910F066
:10588000010F01D0E07840B1B1F86410002011F4AC
:10589000807F18BFFCF789FF07E0B1F86410002093
:1058A00011F4806F18BF0FF0EBFAA149084208BF4E
:1058B00070BD2968496E090CE17070BD10B572B6F3
:1058C000FEF7BCF8BDE81040FDF703BE10B5012897
:1058D00002D0022805D008E04FF42F30FDF734F84D
:1058E00003E04FF040219348086772B6FEF7A6F830
:1058F000BDE81040FDF7EDBD894900280A7918BFC1
:1059000001200871C0B2824208BF704700220028FF
:1059100018BF012200230121022008F0B7BC8048F3
:105920000079002818BF012070477D484069704702
:105930007B48006970477A480069002818BFC07A20
:105940007047774988617047754880697047744926
:10595000C86170477248C06970477248026802F5B2
:10596000C073118A508A02F5A072FCF798BA2DE92B
:10597000F04FDFF8AC9197B08A46C9F8140006F0F2
:1059800014F9C9F81000002800F0A48090F800C0B5
:1059900089F805C0417889F80610837804460CF12F
:1059A000010089F8073000F0FE0089F80800E2786D
:1059B00089F80920207989F80A00607989F80B00B4
:1059C00009F10D05A0792870E0796870207889F8D0
:1059D0000C006046FCF76DFB99F80B1099F80A0073
:1059E000FCF78AFB69782878FCF790FB694620462B
:1059F00006F004F9608AD9F8185000281CBF6843E3
:105A0000050BB4F81A80D9F81C60B8F1000F08BF74
:105A10004FF48058678C002F08BF4FF48057002048
:105A20001AF0040F18BF4FF485701AF0080F18BF52
:105A300040F004001AF0020F1CBF40F2012108439D
:105A40001AF0010F18BF40F48460616A6FF30F0A07
:105A500008406FF30F0108434AEA000A00981090CB
:105A600004981190089812900C9814900198139033
:105A70000798159010A95046FCF735F81AF0020F58
:105A800071D005F02EFC5FEA000B30D005F040FC31
:105A90006843050B59460020FBF728FC218A0029A2
:105AA0001CBF0020FBF799FC05F052FC7043000B73
:105AB0008030020A0820012101FA00F3134201D1CB
:105AC000401EF9D5061FA07B002818BFA0F1010BCE
:105AD00017D112E013480068B0F8640010F4807F1A
:105AE00018BFFCF762FE002017B0BDE8F08FB4F8D5
:105AF0000CB0BBF1000FCDD1D0E70020FBF7E1FCEB
:105B00008346E07B002814BF401EFBF706FD0BEB2D
:105B10000601042910DD711A0E1D042110E0000099
:105B2000D0040110400601100060004000800040D9
:105B300008000300AD2007B00029BCBF761A002181
:105B40000644042E03DD301FC540042604E0002E69
:105B500002DA7042854000260020FBF7C8FC31467F
:105B60000020FBF7F0FC1AF0010F23D0A18A0029D6
:105B70001CBF0120FBF7BAFB268B3EB1314601204A
:105B8000FBF72BFC31461120FBF727FCA67D3EB12D
:105B9000711E0120FBF7ABFC711E1120FBF7A7FC67
:105BA000E67D3EB1711E0120FBF7CDFC711E112078
:105BB000FBF7C9FC1AF0200F23D0A18B00291CBFD2
:105BC0000220FBF793FB268C3EB131460220FBF707
:105BD00004FC31461220FBF700FCA67F3EB1711E8B
:105BE0000220FBF784FC711E1220FBF780FCE67F8D
:105BF0003EB1711E0220FBF7A6FC711E1220FBF7BE
:105C0000A2FCE07A00281CBF0001FBF7AEFA029864
:105C100005F043FB039830B12B4699F8062099F81C
:105C200005100FF032F93A46414628460FF032F996
:105C30000598FEF7B6FD0998FEF704FE05F0DBFFB8
:105C400010F4005F1CBF0D98FEF7BDFE012017B0D9
:105C5000BDE8F08F10B5FCF716F805F026FB0249F9
:105C600000200861012010BDD0040110FE49087019
:105C70007047FD4800787047FC4810B4FC4A016842
:105C8000914218D14168B1F5907F14D80022D0F824
:105C900008C003461146B2EB9C0F24BF10BC7047EE
:105CA00053F82140491C2244B1EB9C0FF8D3002A41
:105CB00004BF10BC7047002010BC7047EB48FCF7D5
:105CC00043BE2DE9F041C0B0044605F04EFF40B19F
:105CD00081692162C16961624169A162C068E06253
:105CE00005E04FF0FF30E062A0626062206238257C
:105CF0000020C4E90250DE4F4FF49076C4E90076EC
:105D0000224601462B4652F820C0401C6144B0EBAD
:105D1000930FF8D3C1F10008FF22511C6846C4F864
:105D20000C800FF085F8CDF80C800097CDE9016567
:105D300010340DF110080FCC88E80F000FCC0DF1D6
:105D4000200888E80F00D4E90001C84CCDE90C0117
:105D50002046FCF7F9FD69462046FCF797FE01282E
:105D600018BF002040B0BDE8F081BF490120087095
:105D7000704770B50E4605461024FFF7D9FD15F0A3
:105D8000020F18BF052408D115F0010F18BF092410
:105D900003D115F0200F18BF0D243246102C28BF58
:105DA00070BD002A08BF70BD204490F9281020461D
:105DB000BDE8704005F055BFF0B5ADF6040D0446E2
:105DC000FFF7B6FD054614F0020F0AD06F46042611
:105DD0003846FCF7EEF995F92C103A46304605F0B6
:105DE00040FF14F0010F0BD06F4608263946012002
:105DF000FCF732FA95F930103A46304605F031FF9B
:105E000014F0200F04BF0DF6040DF0BD0C246E46F7
:105E100031460220FCF720FA95F93410324620462C
:105E200005F01FFF0DF6040DF0BD2DE9F34F8BB00B
:105E3000002007900868089008790290487901903E
:105E40008879B1F90890B1F90AA08A6904928A891F
:105E5000D1E90784C0F5807602EA00070B9809694A
:105E600010F0010F09914FF0000016D0009001983A
:105E7000002840F206810098012101FA00F20998F9
:105E8000104018BF01200390009A0499002001EBF4
:105E900082118346059100F0E3B8FBF716FC8346B8
:105EA000DDE901014843032101EB400020F003023A
:105EB000414620460EF08FFF5846FBF706FC01983E
:105EC0004FF0000B002840F2DC800122099802FA12
:105ED0000BF1084018BF01200021039004988C4664
:105EE00000EB8B1005904DE0012000FA01F20898BC
:105EF000024244D038F9020B039AA0EB0A000CF1DD
:105F0000010C002A0CBF09EB0004A9EB00044808AF
:105F1000059A069052F82000CA07D50E0090E84076
:105F200082B2C2F30420D3B212F4005F02D0002C7C
:105F300002DB03E0002C01DD9C1B00E09C19BC424D
:105F400005DD1F283ABF0024401C3C4606E0002C1B
:105F500004DA0028C6BF3C46401E002402F400526A
:105F600042EA00204FF6FF73009AAB4020439A4369
:105F7000A84042EA0003DDE9050240F82230491C4E
:105F8000202902D202988445AED301980BF1010B6F
:105F900083459AD375E0012101FA00F208990A427B
:105FA0005BD034F9021B039AA1EB0A010BF1010B40
:105FB000002A0CBF4944A9EB010138F9022BA2EBDE
:105FC0000A0214BFA9EB02024A440029B4BF4B42A3
:105FD0000B46002AB8BF52429A423ED9059B42085E
:105FE000069253F82220C3074FEAD36E0A9222FA90
:105FF0000EF293B2C3F3042203F0FF0C13F4005F1C
:1060000002D0002902DB04E0002902DD0CEB0605CA
:1060100001E0ACEB0605BD4205DD1F2A3ABF0025B5
:10602000521C3D4606E0002D04DA002AC6BF3D465C
:10603000521E002503F4005141EA022129434FF684
:10604000FF730A9A03FA0EF39A4301FA0EF142EA39
:106050000103DDE9051241F82230401C202802D25C
:1060600002998B4597D305E0F004011000AF0200C0
:106070005443524600980199401C00908842FFF416
:10608000FAAE0B98032826BF0120079007980DB0A1
:10609000BDE8F08F2DE9F04F8BB0002205920D790D
:1060A0004E7991F806C00C68CDF808C0B1F90830F7
:1060B000B1F90A2006928A690392D1F810C0CA6920
:1060C000CDF81CC08989DDF808C001EA0C07C0F1D1
:1060D00008010091F0B1081EC0F2D7804FF0000A0D
:1060E000002E7AD9012101FA00F004900098401E98
:1060F00001FA00F00A904FF00108079808FA0AF137
:10610000084018BF01200021019003988C4600EB45
:106110008A1BACE04FF0000A002E5ED94FF0010858
:10612000079808FA0AF1084018BF012000210190E1
:1061300003988C4600EB8A1B49E0012088402042EE
:1061400042D032F9028B06980CF1010CA8EB00004A
:10615000DDF80480B8F1000F0CBF03EB0008A3EBDF
:106160000008480808905BF820004FEAC1794FEA20
:10617000D969049020FA09F080B210F4005F0AD0C7
:10618000B8F1000F0FDA10F4F85018BFA0F58070C6
:1061900040F4005007E0B8F1000F04DD10F4F850AF
:1061A00018BFA0F5807040F080004FF6FF7EDDF84C
:1061B00010800EFA09FE28EA0E0800FA09F048EAF3
:1061C000000808984BF82080491C202901D2AC45D2
:1061D000B3D30AF1010AB245A0D34FE001208840B1
:1061E000204241D032F9028B06980CF1010CA8EB49
:1061F0000000DDF80480B8F1000F0CBF03EB0008CD
:10620000A3EB0008480809905BF820004FEAC17929
:106210004FEAD969089020FA09F080B210F4005FC3
:1062200003D0B8F1000F07DA02E0B8F1000F03DD88
:10623000DDF8108020EA0800DDF80080B8F1000FDA
:10624000C4BFDDF8288048EA00004FF6FF7EDDF885
:1062500020800EFA09FE28EA0E0800FA09F048EA42
:10626000000809984BF82080491C202901D2AC4530
:10627000B4D30AF1010AB245FFF43DAF00980028FB
:10628000C2BF05980BB0BDE8F08F4FF0000B002E99
:1062900045D90298C0F580700090029840F4807053
:1062A0000190039A0020014602EB8B1A31E0012293
:1062B0004FEA184C82404FEA0C4C224226D04FEA5B
:1062C0005009C2075AF82980D20E28FA02F39BB26D
:1062D000DDF800E003F0FF0C0CEB5E0EDDF804C00F
:1062E000491C0EEA0C0CBC4588BFBC4623F0FF03DA
:1062F00043EA0C034FF6FF7C0CFA02FC28EA0C0C74
:1063000003FA02F24CEA02024AF82920401C202833
:1063100001D2A942CBD30BF1010BB345C1D301206C
:1063200005900BB0BDE8F08F2DE9F04F89B0002249
:1063300002920A790F6804924A790092B1F9083002
:10634000B1F90A608A690592CA6909690391FE492F
:106350004969A0EB010CCCF1050881424AD84AD129
:1063600000984FF0000A002844D90121039801FA4F
:106370000AFC1CEA000018BF0120019005990020CA
:10638000844601EB8A1B2DE001218140394226D051
:1063900032F9021B019C891B4FEA19454FEA05455A
:1063A0000CF1010C002C0CBF5D185D1A4FEA500E69
:1063B000C1075BF82E90CC0E29FA04F189B2002DAA
:1063C000C8BF41F4005141F480514FF6FF75A5401C
:1063D00029EA0505A14045EA01044BF82E40401C7E
:1063E000202802D204998C45CED300980AF1010AE4
:1063F0008245BAD35BE0B8F1000F5DDB00984FF047
:106400000009002853D908F10800012101FA00FB16
:10641000401E01FA00F008900124039804FA09F1E3
:10642000084018BF01200021019005988C4600EB20
:10643000891A34E00120884038422DD032F9020B0D
:10644000019C801B0CF1010C002C0CBF1C181C1AA9
:10645000480807905AF82000CD07ED0E0690E84056
:1064600080B210F4005F02D0002C04DA01E0002CAE
:1064700001DD20EA0B00B8F1000FC4BF089C2043E7
:106480004FF6FF7E0EFA05FE069CA84024EA0E0495
:10649000044307984AF82040491C202902D2049856
:1064A0008445C7D3009809F101098145B4D3B8F1F7
:1064B000000F04BF01200290029809B0BDE8F08FE0
:1064C0002DE9F04FD7B08346002088464990489088
:1064D00072B6FBF717FC0646FDF7DFF848B1FDF78B
:1064E0007FF94990FDF766F9FDF77FF94890FDF7D0
:1064F0006CF9FBF7EDFAFBF747FA4D90FBF710FC50
:106500004C90FBF743FA0120FBF79BF852901120C7
:10651000FBF797F853900220FBF793F85090122066
:10652000FBF78FF85190FCF7C3FE4B90FCF7A8FEE9
:106530004FF49350FCF715FE62B6FBF76CF84A90E7
:106540000120FBF75EF80120FBF7BFF85490002014
:10655000FBF763FA4F900020FBF754FA4E900020AF
:10656000FAF7A6FE55900020044636AF47F82040C3
:10657000401C0628FAD3DFF8D49116F0020F4FF032
:10658000010505D04FF40461484636950EF019FC1C
:1065900016F0010F10D04FF400716D480EF011FC91
:1065A0000120FAF707FA002818BF38951120FAF7EA
:1065B00001FA002818BF399516F0200F10D04FF4BB
:1065C000007163480EF0FDFB0220FAF7F3F9002892
:1065D00018BF3A951220FAF7EDF9002818BF3B953D
:1065E000DFF870A1584E369850B30020FAF75CFFE0
:1065F00000909AF800008DF80400574800780128B0
:1066000094BF5648564800788DF805000020FBF7E7
:1066100046F8002818BF4FF0FF3004908DF8068030
:106620007088ADF80800ADF80A400020FAF7F0FED7
:10663000ADF80C004FF04050CDE906904948089065
:1066400037984FF0FF0838B30020FAF72DFF099074
:106650009AF800008DF828008DF829500D948DF8D7
:106660002A807088ADF82C00ADF82E400020FAF793
:10667000CFFEADF830009DF8050009EB80110F91B9
:106680009DF8041048434FF0405101EB4001109138
:10669000344901EB40001190DFF8CC90DFF8CCA03A
:1066A000389858B30120FAF7FFFE1290FAF7AAFBC8
:1066B00000280CBF9AF8000099F800008DF84C00F3
:1066C0000120FAF7FEFE05FA00F08DF84D000120DA
:1066D000FAF7B7FFC04316908DF84E80B088ADF83A
:1066E0005000ADF852400120FAF792FEADF8540088
:1066F000174818901E4819901E481A90399810B3E0
:106700001120FAF7D1FE1B90FAF77CFB00280CBF92
:1067100099F800009AF800008DF870001120FAF73F
:10672000D0FE05FA00F08DF871001120FAF789FF0C
:10673000C0431F908DF87280B088ADF87400ADF83A
:106740007640112018E021E0F004011000400030F4
:1067500040480030D8040110D7040110D6040110BD
:10676000D904011000200030DA040110DB0401100C
:106770004008003040280030FAF74AFEADF87800B3
:10678000FE482190FE482290FE482390DFF8F893BF
:106790003A9828B30220FAF787FE249099F800006F
:1067A0008DF894000220FAF78CFE05FA00F08DF8BF
:1067B00095000220FAF745FFC04328908DF8968097
:1067C000F088ADF89800ADF89A400220FAF720FE64
:1067D000ADF89C00ED482A90ED482B90ED482C90A8
:1067E0003B9828B31220FAF75FFE2D9099F801002C
:1067F0008DF8B8001220FAF764FE05FA00F08DF863
:10680000B9001220FAF71DFFC04331908DF8BA800D
:10681000F088ADF8BC00ADF8BE401220FAF7F8FDE4
:10682000ADF8C000DC483390DC483490DC4835904B
:106830009DF84D000224022809D9042805D99DF8A5
:106840004C10199800EB810019908DF84D409DF87F
:106850007100022809D9042805D99DF870102298E2
:1068600000EB810022908DF871400120FAF7E9FEDB
:106870004FF0553620B171000120FAF7D1FE16967F
:106880001120FAF7DEFE28B14FF0AA311120FAF7F5
:10689000C7FE1F969DF89500022809D9042805D93E
:1068A0009DF894102B9800EB81002B908DF895406B
:1068B0009DF8B900022809D9042805D99DF8B81017
:1068C000349800EB810034908DF8B9400220FAF73B
:1068D000B8FE28B14FF0AA310220FAF7A1FE28969F
:1068E0001220FAF7AEFE28B14FF0AA311220FAF7C3
:1068F00097FE3196BDF8520000F58060ADF8520069
:10690000BDF8760000F58060ADF87600BDF89A001D
:1069100000F58060ADF89A00BDF8BE0000F580601B
:10692000ADF8BE00FBF73BFA0026B246B14634464E
:10693000B04642AF03F098F901287BD0BAF1800F3E
:1069400078D83CA8FBF7E9FB00287BD03CA804F0F2
:1069500074F819F1010971D04FF0000948460AF1A5
:10696000010A012147F82010401C0628F9D3002C09
:1069700008BF00250CD0012C08BF00251AD0022C1E
:1069800008BF002528D0032C08BF012635D05EE0C3
:1069900036A850F8250048B105EBC501684600EB64
:1069A00081014046FFF7C0FC47F825006D1C062D0D
:1069B000EED322E036A850F8250048B105EBC5011A
:1069C000684600EB81014046FFF764FB47F825006D
:1069D0006D1C062DEED310E036A850F8250048B106
:1069E00005EBC501684600EB81014046FFF71DFA43
:1069F00047F825006D1C062DEED30121002057F825
:106A00002020CAB1401C0628F9D3A9B11F2C0ED2F0
:106A10000120641C00FA04F111EA0B0F07D1641C79
:106A2000032C9CBF00FA04F111EA0B0FF7D04FF0D2
:106A3000000803E00BE005E008F101083EB9FBF7B0
:106A4000AEF977E7FEF7D6FE002E3FF473AFFAF704
:106A50009DFF01205299FAF7E3FD11205399FAF7AF
:106A6000DFFD02205099FAF7DBFD12205199FAF769
:106A7000D7FD4A98FAF7C5FD5498FAF726FE4F98C5
:106A8000FAF7CBFF4E98FAF7BDFF5598FAF710FCCE
:106A90004D9830B14C9810B1FBF781F901E0FBF74C
:106AA00045F9FCF7FAFD48B14998002818BFFCF7F2
:106AB000F9FD4898002818BFFCF72CFE4B980028D9
:106AC00018BFFCF786FB002E0CBF0120002057B03A
:106AD000BDE8F08F2DE9F843074600200E46054635
:106AE000009092E0284605F060F800287ED00089EA
:106AF00000EA070424F0CC0030F47C4076D00F216B
:106B00002846FEF734FF00287ED0FBF7FBF80099FB
:106B1000002977D1FAF7C4FFFF210F20FFF7D0FC3F
:106B20000090FAF733FF009800286BD19EB114F063
:106B3000010F1CBF0220FFF73FF914F0100F1CBF1C
:106B40000120FFF739F914F4807F1CBF2020FFF7E4
:106B500033F9009830BB24F0990030F4794006D026
:106B6000FDF7B5FF0090FAF711FF0098D0B9CEB14C
:106B700014F0020F23D0FDF76FF914E0C048003085
:106B8000C00A0030C02A0030DD0401104049003046
:106B9000C00E0030C02E0030C0490030C0100030A0
:106BA000C03000302EE08046FEF7C2FE05235FEACB
:106BB000080204D090F92D10184605F052F814F090
:106BC000200F0DD0FDF7CDF88046FEF7B1FE09236A
:106BD0005FEA080204D090F93110184605F041F838
:106BE00014F4007F0ED0FDF785F800E00CE00446B9
:106BF000FEF79EFE0D23220004D090F935101846B2
:106C000005F02FF8FFF726F86D1C04F0CAFFA84224
:106C1000009803D900283FF465AF04E0002804BFC2
:106C20000120BDE8F8830020BDE8F883F0B5DD4E13
:106C300091B001243578FEF785FD012865D1DA4849
:106C40000068B0F93610B0F934000EF028F915F0EC
:106C5000020F4FF000072ED002A800F06EF907983F
:106C60002146401C079040F27770FFF733FF012860
:106C700003D1FEF75FF8012813D009980023401CC8
:106C80000990502006901A462121072007F0FEFAAD
:106C900000231A461946FE200097FEF7DEF802A8E8
:106CA00028E015F0080F14BFA220A1200690089834
:106CB000401C0890F3E715F0100F1DD0B0680328B2
:106CC00024BF0024B76005D2684600F036F90C985E
:106CD000401C0C9021464FF4E060FFF7FBFE08B12A
:106CE000C4B106E0002301222121072007F0CEFADB
:106CF00014B16846FEF7E5FF0020FDF702FD002312
:106D00002A464021072007F0C1FA11B0BDE8F04043
:106D100002F054BF04F06FFF20F4E04004F068FF7D
:106D2000EAE7A04A002804BF51807047012804BF49
:106D300091807047022808BFD180704701004FF052
:106D40000000984A04BFB2F902007047012904BF4D
:106D5000B2F904007047022908BFB2F90600704773
:106D600070B50126FEF788FF20B10069A12818BF81
:106D7000A22801D0002070BD002404F012FF0028DA
:106D800042D9204604F011FF00281EBF058925F0D6
:106D9000CC0030F47C4032D00F212046FEF7E7FDD6
:106DA00068B315F0010F0AD0FBF70EFA38B944F4B6
:106DB000807200232021072007F068FA002615F0D2
:106DC000100F0BD00120FBF753FA38B944F480526E
:106DD00000232021072007F059FA002615F4807FB0
:106DE0000BD00220FBF744FA38B944F48032002378
:106DF0002021072007F04AFA0026FEF72BFF641C2B
:106E000004F0CFFEA042BCD8304670BD00207047D1
:106E100000207047002818BF012062494870704761
:106E200060484078002818BF012070475D48C0685E
:106E3000704770B582B00D460446FEF780FC00280E
:106E400078D1584E3069002874D0707868230028B3
:106E500034D000207070B5F9000043F2B0614218E0
:106E600046F66D3C624529D3B5F90220101A4A1046
:106E70001044884222D9288869888DF80030030A96
:106E80008DF801308DF80200080A8DF804100322F5
:106E90008DF803008DF8052000230622694607209F
:106EA00007F024FA10210120FEF761FC0320B060F6
:106EB000F068401CF06002B0012070BDB4F9000021
:106EC00043F2BC41884229DDB4F9020088422CDD3E
:106ED000B0680022401CB06003282BD32088618852
:106EE0008DF80030030A8DF801308DF80200080A91
:106EF0008DF804108DF803008DF80520002306227C
:106F00006946072007F0F2F910210120FEF72FFC57
:106F1000F068401CF06002B0012070BD2349884237
:106F2000BCBFB4F902008842D2DB0020B06002B0DE
:106F300070BDFFE702B0002070BD10B50446FEF73B
:106F40009BFE80B1B0E80E10A4E80E10B0E80E1061
:106F5000A4E80E10B0E80E10A4E80E10D0E900105E
:106F6000C4E9001019E0FF22382120460DF060FF2F
:106F70000F4820604FF49070606038200021C4E911
:106F800002015020C4E90401481EE062A062A16130
:106F90006062C4E90710216361630648FBF7D4FC13
:106FA000012010BDF00401104006011050C9FFFF80
:106FB0005443524600AF020070470020704710B59E
:106FC00003F00700042808BFFEF778FC002010BD7E
:106FD00070B503F007020025F84CF94B012A02D0E6
:106FE000022A14D011E0052018709D60FCF7AEFA5B
:106FF0002268532111702268452151702268010ACC
:1070000091702168C87020680571002070BD1A78E1
:10701000052A13D19A68052A28BF104607D2D4F84A
:1070200000C01CF802C080F800C0501C9860052801
:1070300004D101209D60087003201870012070BDEC
:107040002DE9F04103F0070201260025DB4CDC4B63
:10705000012A02D0022A3BD037E0052018709D603B
:10706000FCF774FA2168AC270F702268010A51708E
:107070002168887004F04CFDDFF8488380B1D8F8AF
:10708000000004F033FE58B1D8F8000090F820005A
:1070900010F0020F04D020684770216843208870E8
:1070A0002068C6702068057104F032FD50B1D8F830
:1070B000000004F01BFE28B1D8F800002168007E13
:1070C000487102E02168FF2048710020BDE8F0818E
:1070D0001A78052A12D19A68062A28BF104607D2C4
:1070E000D4F800C01CF802C080F800C0501C9860A2
:1070F000062803D19D600E70032018700120BDE8A2
:10710000F08103F00702022A1CBF002070472022F2
:1071100002700120087070472DE9F041A84F0D461C
:10712000064613F0070F04D003F00700022808D02A
:1071300004E012F0040F1CBF0020B8700020BDE86E
:10714000F08102F035FD002814BF0124002402F074
:1071500032FD002814BF0222002242EA0403B8785C
:10716000002814BF0422002242EA030030700120EC
:107170002870BDE8F08170B503F0070C0026904C34
:107180008E4DBCF1010F0AD0204613F0070F007896
:107190000DD0BCF1040F08BF062818D029E0A66066
:1071A00028680670286846700520207021E00528B0
:1071B0001FD1A068022803D22B681A54401CA0607B
:1071C000022816D10120A6600870062010E0286869
:1071D000007855280BD128684078AC2818BFBC2807
:1071E00005D128680122411C062002F0C7FC0320BB
:1071F0002070002070BD70B503F0070200256F4CB1
:107200006F4B012A02D0022A24D021E005201870F9
:107210009D6002F088FC41F6E8710144B0F5283F1A
:1072200010D8CA78086862F31F60674A904208BFA6
:10723000002007D10A18236812791A54401C142818
:10724000F8D305E0002021680D54401C1428FAD31F
:10725000002070BD1A78052A13D19A68142A28BF15
:10726000104607D2D4F800C01CF802C080F800C055
:10727000501C9860142804D101209D6008700320E0
:107280001870012070BD70B503F0070200254B4C4B
:107290004B4B012A02D0022A3FD03CE00520187057
:1072A0009D6002F040FC41F6E8710144B0F5283FD2
:1072B0002BD8CA78086862F31F60434A904224D1F1
:1072C0002268087C10702268487C50702268887C94
:1072D00090702068CA7CC27020680A7A02712268A5
:1072E000487A50712268887A90712268C87AD07181
:1072F0002268087D10722268487D50722268887D5D
:107300009072C87D2168C87205E0002021680D5484
:10731000401C0C28FAD3002070BD1A78052A13D11E
:107320009A680C2A28BF104607D2D4F800C01CF86F
:1073300002C080F800C0501C98600C2804D10120C5
:107340009D60087003201870012070BD70B503F0B7
:1073500007020025194C1A4E012A02D0022A3FD0FA
:107360003CE004F002FC40B3D0E906212368C06889
:107370001A70D4F800C0130A8CF80130D4F800C099
:10738000130C120E8CF802302368DA702268117127
:1073900023680A0A5A7123680A0C090E9A71226836
:1073A000D171216808722268010A51722268010CA9
:1073B0009172010E2068C1720DE007E0287701008C
:1073C000100501104006011034CD12AB21680D5498
:1073D000401C0C28FAD305203070B560002070BD29
:1073E0003278052A10D1B2680C2A28BF104604D280
:1073F00023689B5C0370501CB0600C2804D10120F2
:10740000B560087003203070012070BD70B503F0C6
:1074100007020024F84DF94B012A02D0022A3ED07F
:107420003BE00520187000269C6002F07CFB00F514
:107430000051B0F5283F98BF11F0030F27D1F04A53
:107440000868904204BF0022104620D151F8203035
:10745000401C1A440728F9D302B1C6B128680A7C37
:1074600002702A68487C50702A68887C90702A686C
:10747000C87CD0702A68087D10712A68487D5071D8
:107480002A68887D9071C87D2968C87105E0002050
:1074900029680C54401C0828FAD3002070BD1A78C3
:1074A000052A13D19A68082A28BF104607D2D5F8B2
:1074B00000C01CF802C080F800C0501C986008286A
:1074C00004D101209C60087003201870012070BD59
:1074D0002DE9F04103F0070C0027C84E4FF00508D6
:1074E000BCF1010F0DD013F0070F0FD03246BCF1E5
:1074F000020F127810D0BCF1040F08BF062A26D064
:1075000058E086F800807770B76053E07270BD482D
:10751000B062062030704DE0052A15D1B268042A09
:1075200028BF104609D2C2F10303D6F828C0DB00F9
:107530002CFA03F30370501CB060042804D101201E
:10754000B7600870032030700120BDE8F0817078CA
:107550000125002410F0010F11D002F0E4FAB0F57B
:10756000283F23D86A030021B1EB900F07D252F8CD
:10757000043B491C1C44B1EB900FF8D3B5B17078B3
:1075800010F0020F0ED004F0F0FA78B182680021FA
:10759000B1EB920F06D250F8043B491C1C44B1EBEE
:1075A000920FF8D3002D18BFB46200D1B762777084
:1075B00086F800800020BDE8F081F0B503F0070CEC
:1075C00000268D4D8D4C83B0BCF1010F0ED013F011
:1075D000070F1DD0224603271278BCF1020F26D0D8
:1075E000BCF1040F08BF062A36D03CE002AA01A96C
:1075F000684602F02DFE0520207029680198087069
:10760000296800984870296802988870A6602AE066
:10761000A068032803D229680A54401CA0600228ED
:1076200021D306212170032808BFA6601BE0052A8C
:107630000FD1A268032A28BF104604D22B689B5C96
:107640000370501CA060032803D10120A6600870BD
:10765000277003B00120F0BD286882780178407857
:1076600002F0EBFD277003B00020F0BD08B503F079
:10767000070001280AD104F04BFA38B101208DF837
:107680000000024669460D2002F078FA002008BD8D
:1076900008B503F0070001280AD104F039FA38B11F
:1076A00000208DF80000012269460D2002F066FAE4
:1076B000002008BD08B503F00700012809D104F037
:1076C00027FA30B103208DF800000122694602F04C
:1076D00055FA002008BD0020704708B503F00700E8
:1076E00001280AD104F014FA38B10B208DF80000FB
:1076F00001226946032002F041FA002008BD1FB5AF
:1077000013F0070F0ED104F003FA58B19DF80800EA
:10771000F0280AD004F0FCF920B1012202A90920C6
:1077200002F02CFA04B0002010BDFEF7C7FAF9E70A
:1077300008B503F0070001280AD104F0E9F938B1CF
:1077400010208DF8000001226946032002F016FA8D
:10775000002008BD70B503F00700274C274D012815
:1077600008D013F0070F12D0042804BF2878062889
:1077700016D01FE00020A8602168087021684870BA
:10778000216888702168C8700520287012E0A868F8
:1077900004280FD221680A54401CA860062008E083
:1077A00004F0B6F930B104221046216802F0E6F97F
:1077B00003202870002070BD10B503F007000128D9
:1077C00004D103F00FFA0D4900200871002010BD0C
:1077D00070B5054603F007000C4601280AD013F0E7
:1077E000070F02D002280FD004E0012200211B2045
:1077F00002F0C4F9002070BD2877010010050110C7
:1078000054464953EFBEADDE03F0AFFB28700120B4
:107810002070F0E710B503F0070CFE4CBCF1010F2F
:1078200006D013F0070F09D0BCF1020F18D015E0F5
:107830000020A06006F021FDA0610FE0A0680028F4
:1078400004BF1002A06106D0012804D1A069104332
:10785000A06106F011FDA068401CA060002010BDD2
:10786000A26812B1012A04D007E0218B090A017035
:1078700003E0237E037001200870501CA0600120EB
:1078800010BD10B503F0070CE24CBCF1010F06D09F
:1078900013F0070F09D0BCF1020F18D015E000203B
:1078A000A06006F0EDFCA0610FE0A068002804BF16
:1078B0001002A06106D0012804D1A0691043A06184
:1078C00006F0E1FCA068401CA060002010BDA2688A
:1078D00012B1012A04D007E0218B090A017003E0EC
:1078E000237E037001200870501CA060012010BD91
:1078F00070B503F0070CC74D0E460446BCF1010FEE
:1079000006D013F0070F07D0BCF1020F18D015E016
:107910000020A860E86011E0A868002804BF1002F9
:10792000A86108D0012806D1A869104381B2A861D6
:10793000E8880DF0B9FAA868401CA860002070BD66
:10794000E86802280ED2E8880DF0B3FAEB6882B23C
:10795000002B04BF100A207004D0012B02D122702A
:1079600001203070E868401CE860012070BD10B450
:1079700003F0070CA74CBCF1010F08BF00200BD08F
:1079800013F0070F03D0BCF1020F09D005E0A06887
:10799000002808BFE280401CA06010BC0020704797
:1079A000A2681AB9A379037001200870501CA06066
:1079B00010BC012070472DE9F047064603F0070090
:1079C000944F8946012808BF002039D0DFF848824B
:1079D000924D13F0070F02D0022835D031E0B8687D
:1079E000002808BF7A7029D0012804BF1002B861AE
:1079F00024D0022822D1B8691043B8617E7884B2BD
:107A000004F086F8D0B1062E18D2DFE806F003069F
:107A1000090C1014A8F80E4010E0A8F80C400DE076
:107A2000286884860AE02868A0F80C4106E02868E7
:107A3000A0F8504002E02868A0F85240B868401C06
:107A4000B8600020BDE8F087F86802282CD297F8CB
:107A500001A0002404F05CF8D8B1BAF1060F18D2E6
:107A6000DFE80AF00306090C1014B8F80E4010E025
:107A7000B8F80C400DE02868848E0AE02868B0F859
:107A80000C4106E02868B0F8504002E02868B0F8E1
:107A90005240F868002804BF200A307004D0012842
:107AA00002D1347089F80000F868401CF8600120A9
:107AB000BDE8F0872DE9F0411C4615460E46074605
:107AC00004F026F880B1544814F0070F04D004F0F5
:107AD000070102290BD007E0002D1ABF90F86C00B7
:107AE000C00800200DF0EAF90020BDE8F08190F810
:107AF0006C00C008387001203070BDE8F0812DE9BD
:107B0000F0411C4615460F46064613F0070F08D1F4
:107B100003F0FEFF28B1022D3CBF28460DF0D3F93B
:107B200003E004F00700022802D00020BDE8F08145
:107B30000DF0CEF9307001203870BDE8F08170B5DD
:107B400003F007020026364C324D012A02D0022AE9
:107B500015D012E007F02BF921680870FDF7F2FD4F
:107B60002168487003F0BAFB21688870FDF7F0FDCA
:107B70002168C87005202870AE60002070BD2A788A
:107B8000052A10D1AA68042A28BF104604D2236807
:107B90009B5C0370501CA860042804D10120AE60D7
:107BA000087003202870012070BD70B503F0070233
:107BB0001B4C0025174E012A02D0022A5DD05AE044
:107BC000FEF75AF800283FD04169FF292CBFFF215A
:107BD000C9B2226811708169FF2934BFC9B2FF217F
:107BE00022685170C169FF2934BFC9B2FF212268E0
:107BF00091702268017CD170226890F82010117178
:107C0000018C2268090A5171016A2268090C91717C
:107C1000016A07E0100501103083011040060110D1
:107C2000287701002268090ED171016BFF2934BF4A
:107C3000C9B2FF2122681172406BFF2834BFC0B265
:107C4000FF202168487215E02068057020684570A3
:107C50002068857021685020C8702168FF20087155
:107C600021684871216888712168C871206805728F
:107C700020684572B560002070BDB2680A2A28BF2E
:107C8000104604D223689B5C0370501CB0600A2825
:107C900002D10120B5600870012070BD03F0070219
:107CA000FE4B4FF0000C012A08BFC3F808C001D0FA
:107CB000022A01D0002070479A68022A3DBF80F84E
:107CC00000C0501C98601046022803D10120C3F860
:107CD00008C00870012070472DE9F047064603F000
:107CE0000700EE4F8A464FF00008012808BFC7F88A
:107CF000088001D0022802D00020BDE8F087B868D3
:107D0000A0BB0024254601F00EFF014600F50050FF
:107D100018384FF400524FF04009B1F5283F20D8F1
:107D200090F803C003686CF31F63DFF874C3634506
:107D300017D1091FB4EB910F06D252F8043B641C13
:107D40005D40B4EB910FF8D3C17D406961F31F60D2
:107D5000A84206D103F0A4FE012804BF80203070A1
:107D600001D086F80090B868401CB860012803D1A3
:107D7000C7F808808AF800000120BDE8F0872DE9E7
:107D8000F04103F007020026C64CC44D012A02D080
:107D9000022A56D052E0FBF7D9FB0520287003F0E9
:107DA000B7FE002849D0C04F386803F09FFF002875
:107DB00043D00DF092F880460DF094F839680A7EB1
:107DC00012F0040F11D0C98A2268090A11703968AB
:107DD0002268897D517039682268898A090A917000
:107DE00039682268097DD17010E0898A2268090A01
:107DF000117039682268097D517039682268C98A12
:107E0000090A917039682268897DD17022684FEA29
:107E100018211171216881F805802268010A917189
:107E20002168C87138682268817C11722268017CDF
:107E30005172008B2168000A8872AE600020BDE894
:107E4000F0812A78052A10D1AA680B2A28BF10468B
:107E500004D223689B5C0370501CA8600B2804D1DB
:107E60000120AE600870032028700120BDE8F08179
:107E70002DE9F04703F0070200268A4D874B012ABF
:107E800002D0022A5DD059E00520187000249E60BF
:107E900001F049FE00F50053B0F5283F98BF13F0FC
:107EA000030F45D1814A1968914204BF002211464F
:107EB00008D153F821C0491C62440729F9D3002A8C
:107EC00008BF01249F7C93F8138084B341F6E871C6
:107ED0000144B0F5283F07D8CA78086862F31F60EC
:107EE0006F4A904208BF012491F8129091F813A0B4
:107EF000002C08BF002014D003F037FE29688069E9
:107F000081F80090296881F801A02A68010C000E10
:107F100091702968C87028680771286880F8058002
:107F20000CE029680E54401C0628FAD306E0FFE74F
:107F3000002029680E54401C0628FAD30020BDE812
:107F4000F0871A78052A13D19A68072A28BF1046A5
:107F500007D2D5F800C01CF802C080F800C0501C41
:107F60009860072804D101209E60087003201870D3
:107F70000120BDE8F08710B503F0070C474CBCF1B9
:107F8000010F06D013F0070F0AD0BCF1020F1AD070
:107F900017E00020A060E0600CF0A9FFA06110E0F5
:107FA000A068002804BF1002A06107D0012805D1F5
:107FB000A0691043A06180B20CF09EFFA068401C35
:107FC000A060002010BDE268022A0BD212B1012A83
:107FD00004D007E0218B090A017003E0237E0370BF
:107FE00001200870501CE060012010BD70B503F046
:107FF00007010026294D0446012908BFEE6201D081
:10800000022901D0002070BDE86A002804BF28487A
:108010000CF077FFE96A082928BF267002D22448AD
:10802000405C2070481CE862012070BD2DE9F041E1
:1080300003F007010026194D0746012908BFEE622B
:1080400001D0022902D00020BDE8F08195F82C0073
:1080500000F007042879204304D115480CF051FFA3
:1080600001202871052C28BF2E711148005D387041
:10807000E86A401CE8620120BDE8F08170B5044662
:1080800003F007000D4602281CBF002070BD0CF055
:108090003DFF20700120287070BD00001005011008
:1080A00034CD12AB287701004006011054464953E5
:1080B0004005011070B503F007020025F94C012AB4
:1080C00002D0022A12D00FE00520207000221146B3
:1080D0001046A56002F0BCF84FF6FF7101EA4000BF
:1080E000206102F0C8F86062002070BD2278052A85
:1080F00017D1D4F810C0A268624528BF104607D235
:1081000012F0010F1CBF637803700CD0501CA060EC
:10811000604506D10120A56008700320207002F0A0
:10812000B8F8012070BD666A22F00103F35A1E0AF6
:1081300006706370EAE770B503F007020025D94CBA
:10814000012A02D0022A11D00EE0D7480522006889
:10815000B0F91210B0F91000227008444000A56078
:10816000206102F006FA6062002070BD2278052AC4
:1081700017D1D4F810C0A268624528BF104607D2B4
:1081800012F0010F1CBF637803700CD0501CA0606C
:10819000604506D10120A56008700320207002F020
:1081A000F6F9012070BD666A22F00103F35A1E0A37
:1081B00006706370EAE770B503F007020025B94C5A
:1081C000012A02D0022A0AD007E0052020700620EA
:1081D000A560206102F00AFB6062002070BD227879
:1081E000052A17D1D4F810C0A268624528BF1046EE
:1081F00007D212F0010F1CBF637803700CD0501C23
:10820000A060604506D10120A560087003202070A1
:1082100002F0F6FA012070BD002A12BF012A636A3B
:108220005B8806D0022A13BF032A636A1B884FF6B5
:10823000FF731E0A06706370E1E77FB51C460E46A9
:10824000054613F0070F08D103F062FC28B10122A4
:1082500002A9232001F092FC03E004F007000228A9
:1082600002D004B0002070BD06F08AFE2870012004
:10827000307004B070BD7FB51C460E46054613F045
:10828000070F08D103F044FC28B1012202A92420E1
:1082900001F074FC03E004F00700022802D004B0EF
:1082A000002070BD06F072FE28700120307004B00E
:1082B00070BD7FB51C460E46054613F0070F08D16A
:1082C00003F026FC28B1012202A90C2001F056FC83
:1082D00003E004F00700022802D004B0002070BDC3
:1082E00006F065FD28700120307004B070BD7FB5C8
:1082F0001C460E46054613F0070F08D103F008FC94
:1083000028B1012202A90F2001F038FC03E004F09B
:108310000700022802D004B0002070BD03F089FAE3
:1083200000F00F0040F0100028700120307004B001
:1083300070BD2DE9F04103F0070C5A4D0E4607467B
:10834000BCF1010F07D0594C13F0070F07D0BCF157
:10835000020F1BD017E00020A860E86013E0A868B7
:1083600004283CBF21680A54032809D120682168E9
:108370000068C97800BA20F0FF000843FCF7F8FE57
:10838000A868401CA8600020BDE8F081E86870B9CA
:10839000FCF7F3FE216820F07E42100E0870216881
:1083A000100C48702168100A88702068C270EA6852
:1083B000042A06D22068032A805C387004BF01209A
:1083C0003070501CE8600120BDE8F0817FB51C468C
:1083D0000D46064613F0070F08D103F099FB28B1AC
:1083E000012202A9102001F0C9FB03E004F00700FC
:1083F000022802D004B0002070BD03F057FA00F04C
:108400000F0403F016FA64F31F1030700120287077
:1084100004B070BD10B503F00702224C012A02D04F
:10842000022A0DD00AE003F0F5FD0021E0610028EA
:108430001ABF4FF4056020622162A160002010BDC8
:10844000236AA2689A4228BF104607D2D4F81CC0FB
:108450001CF802C080F800C0501CA060984204BF05
:1084600001200870012010BD10B413F0070F4FF069
:10847000402C04D003F00702022A19D00FE0012A91
:1084800004BFDCF8140040F0010006D0002A04BF4D
:10849000DCF8140020F0010001D1CCF81400002019
:1084A00010BC70471005011040060110287701002C
:1084B000DCF81430002213F0010F18BF0122FD4B2D
:1084C000D3F83CC0FC4B1B68B3F8A430C3F30334AF
:1084D000012303FA04F41CEA040F18BF42F002025D
:1084E00002700B700120DBE770B514460E4605469E
:1084F00013F0070F04D003F00700022813D010E098
:10850000002C14BF0120002002F05EFB4CB14FF0A4
:108510004020016B21F4405141F4BE0141F0204163
:108520000163002070BD02F056FB002814BF012239
:1085300000222A700120307070BD2DE9F04103F057
:10854000070CDE4C0F468046BCF1010F12D0D94E0D
:1085500013F0070F4FF0030510D02046BCF1020FB7
:10856000027822D0BCF1040F02BFA0680128062ABD
:108570002FD032E005202070002014E0A06810B158
:10858000012804D00DE062700620207009E06078B8
:1085900000EA0201316320EA02017163FAF744FB49
:1085A0002570A068401CA06017E0A068012808BFE3
:1085B000062A03D16078FAF73CFB2570F06B88F847
:1085C000000001203870A068401CA0600120BDE8B8
:1085D000F0816078FAF72DFB25700020BDE8F0816E
:1085E00070B5044603F007000D4602281CBF0020AA
:1085F00070BDFDF794F9002814BF012200222270FB
:108600000120287070BD70B50D46044613F0070FA9
:1086100004D003F00700022805D002E0104606F05F
:10862000F5FA002070BD06F0F4FA207001202870E1
:1086300070BD70B50D46044613F0070F04D003F06B
:108640000700022805D002E01046F8F7C5FB00201D
:1086500070BDF8F7C4FB20700120287070BD70B5A4
:1086600003F00702954D0E460446012A04BF002080
:10867000A86001D0022A01D0002070BD0CF04BFC94
:10868000AA68002A04BF000A207004D0012A02D17F
:10869000207001203070501CA860012070BD70B5A2
:1086A000044603F007000D46022807D013F0070F19
:1086B00004BF1046FDF740F8002070BDFDF73FF8FD
:1086C00020700120287070BD70B5044603F00700CB
:1086D0007A4D0E46012804BF0020A86014D013F084
:1086E000070F02D0022811D00EE0A86874490428B0
:1086F0003CBF0B681A54401CA860042804D1042213
:108700000968132001F03AFA002070BD07F0DDF986
:10871000AA68002A04BF000E20700FD0012A08BFEB
:10872000000C06D0022A08BF000A02D0032A02D099
:1087300004E0207002E0207001203070501CA8601E
:10874000012070BD70B503F0070C5C4D0E46044669
:10875000BCF1010F04BF0020A86015D013F0070F73
:1087600003D0BCF1020F11D00EE0A86854490228D2
:108770003CBF0B681A54401CA860022804D1022296
:108780000968142001F0FAF9002070BD07F070F9B3
:10879000AA68002A04BF000A207004D0012A02D16E
:1087A000207001203070501CA860012070BD70B591
:1087B000044603F00700414D0E46012804BF002087
:1087C000A86014D013F0070F02D0022811D00EE0D9
:1087D000A8683B4904283CBF0B681A54401CA86099
:1087E000042804D104220968152001F0C7F90020EB
:1087F00070BD07F093F9AA68002A04BF000E20702C
:108800000FD0012A08BF000C06D0022A08BF000AB8
:1088100002D0032A02D004E0207002E02070012080
:108820003070501CA860012070BD70B5044603F084
:108830000700224D0E46012804BF0020A86037D053
:1088400013F0070F02D002283CD031E0A8681C4C7E
:10885000002804BF21680A7021680978012901D025
:1088600039B11BE0002818BF04283CBF21680A5416
:1088700014E007F06CF921680009487007F05DF911
:10888000C0F3032607F063F9216846EA00108870F8
:1088900007F053F92168C8700320A860A868401C3D
:1088A000A860042804D104221620216801F066F98A
:1088B000002070BD0010004040060110100501109E
:1088C0002877010007F04FF9AA68002A04BF000EBC
:1088D00020700FD0012A08BF000C06D0022A08BF62
:1088E000000A02D0032A02D004E0207002E02070C7
:1088F00001203070501CA8600120DAE710B503F0A9
:108900000702FE4C012A02D0022A27D024E003F0FD
:1089100081FB0023002804BFE36123621BD000F128
:108920005001E1614168B1F5887F90F820100CD3C7
:1089300090F8212001EB020C01FB02C190F82220EB
:1089400090F823001044084404E090F822000A182C
:1089500001FB00202062A360002010BD236AA268F2
:108960009A4228BF104607D2D4F81CC01CF802C097
:1089700080F800C0501CA060984204BF012008701D
:10898000012010BD03F00702012A02D0022A05D0FF
:1089900002E0DA490020886000207047012202705E
:1089A0000A701046704710B513F0070F04D003F09B
:1089B0000702022A05D002E0104601F077FC0020F1
:1089C00010BDCF4A127802700120087010BD10B59A
:1089D00013F0070F04D003F00702022A05D002E0CB
:1089E000104601F0F7FD002010BDC64A1278027053
:1089F0000120087010BD10B513F0070F04D003F06C
:108A00000702022A05D002E0104601F006FF00200E
:108A100010BDBD4A127802700120087010BD1FB54C
:108A200013F0070F07D103F073F820B1012202A958
:108A30000B2001F0A3F804B0002010BD70B503F0C6
:108A40000700AE4C1546012804BF0020A06024D0CA
:108A500013F0070F21D103F05BF8F0B1A068AB4E23
:108A600003283CBF31680D54401CA060032814D17A
:108A7000F9F72EF83068B0F8010045BAF8F784FF2E
:108A8000040018BFF9F7BEF9306829460078F8F7F6
:108A90002DFC002C18BFF9F7B8F9002070BD70B597
:108AA00003F00700954C1646012804BF0020A06083
:108AB00029D013F0070F26D103F02AF818B3A068C5
:108AC000924D02283CBF29680E54401CA060022829
:108AD00019D1F8F7FDFFF8F757FF040018BFF9F7B1
:108AE00091F92868007880B129684978F8F775FC11
:108AF00028684178007840F01000F8F76EFC002CF0
:108B000018BFF9F782F9002070BD2868417800206D
:108B1000F3E77FB51C460E46054613F0070F08D154
:108B200002F0F6FF28B1012202A91A2001F026F86E
:108B300003E004F00700022802D004B0002070BD5A
:108B400006F00FF9002814BF012200222A7001202C
:108B5000307004B070BD7FB51C460E46054613F05C
:108B6000070F08D102F0D4FF28B1012202A91C206E
:108B700001F004F803E004F00700022802D004B07A
:108B8000002070BD06F0D9F828700120307004B0C4
:108B900070BD2DE9F04103F0070C584C0E46074616
:108BA000BCF1010F07D0594D13F0070F07D0BCF1EE
:108BB000020F19D015E00020A060E06011E0A0686D
:108BC00003283CBF29680A54401CA060032808D130
:108BD0002868B0F8010040BA01B228680078FEF7B2
:108BE000A0F80020BDE8F081E268022A12D242B962
:108BF00028680078FEF7A2F82A68010A51702968EF
:108C000088702868E2681044012A4078387004BFF0
:108C100001203070E068401CE0600120BDE8F08178
:108C200070B503F00700354C1546012804BF00203D
:108C3000A06017D013F0070F14D102F069FF88B1BC
:108C4000A068324B03283CBF19680D54401CA0603B
:108C5000032807D11868B0F8010041BA18680078F5
:108C6000F9F754FB002070BD10B503F00702234C48
:108C7000012A02D0022A07D004E00020A060FAF7FF
:108C800056FBA061002010BDA268042A07D2C2F1E1
:108C90000303D4F818C0DB002CFA03F30370501C54
:108CA000A060042804BF01200870012010BD10B589
:108CB00003F00700012807D102F02AFF20B10022AB
:108CC0001146202000F05AFF002010BD2DE9F04190
:108CD00003F00705094E174688460446012D04BFD8
:108CE0000020B06027D013F0070F22D102F010FF50
:108CF000F8B1B068054B03280AE000001005011028
:108D0000550501105A0501105F0501102877010073
:108D10003CBF19680F54401CB06003280BD1186881
:108D200090F9022090F9011090F90000FCF7CFF8BB
:108D300001E0022D02D00020BDE8F081B06830B122
:108D4000012809D002280CD003280FD015E01420E8
:108D5000FBF7F7FF207010E01520FBF7F2FF207003
:108D60000BE01620FBF7EDFF207006E01720FBF765
:108D7000E8FF2070012088F80000B068401CB06057
:108D80000120BDE8F08170B50D46044613F0070FD1
:108D900004D003F00700022805D002E0F8490020C3
:108DA0008860002070BD0120FBF7CBFF2070012000
:108DB000287070BD70B503F0070C0026F14CF04D23
:108DC000BCF1010F06D013F0070F0CD0BCF1020F5D
:108DD0001FD01CE006F0A9F8AE6021680870216879
:108DE000000A487013E0A868022803D221680A54D8
:108DF000401CA86002280AD1AE602068007810F0FC
:108E0000010F04D002221D20216800F0B7FE0020CF
:108E100070BDAA68022A28BF104604D223689B5C52
:108E20000370501CA860022804D10120AE600870B5
:108E300003202870012070BD7FB51C460E460546F4
:108E400013F0070F08D102F063FE28B1012202A936
:108E5000272000F093FE03E004F00700022802D070
:108E600004B0002070BD0CF05BF828700120307059
:108E700004B070BD7FB51C460E46054613F0070FC3
:108E800008D102F045FE28B1012202A9222000F0FB
:108E900075FE03E004F00700022802D004B00020B1
:108EA00070BD0CF042F828700120307004B070BD25
:108EB00070B50D46044613F0070F04D003F0070009
:108EC000022805D002E01046FAF74AFB002070BDE8
:108ED000FAF757FB20700120287070BD7FB51C4643
:108EE0000E46054613F0070F08D102F011FE28B117
:108EF000012202A9262000F041FE03E004F0070051
:108F0000022802D004B0002070BD0CF013F82870C5
:108F10000120307004B070BD002070472DE9FF4182
:108F2000974E1C460F46054613F0070F1CD102F062
:108F3000EFFDC8B19DF80800002818BF012802D035
:108F4000022807D014E0F070012202A9082000F0E6
:108F500015FE0DE0F07004208DF80800012202A932
:108F6000082000F00BFE03E004F00700022803D005
:108F700004B00020BDE8F081F0782870012038703E
:108F800004B0BDE8F0817FB51C460D46064613F0DF
:108F9000070F08D102F0BCFD28B1012202A9082068
:108FA00000F0ECFD03E004F00700022802D004B05A
:108FB000002070BDFCF7C6FB801E05280ED2DFE83E
:108FC00000F0030709050B00002008E0012006E07F
:108FD000022004E0032002E0042000E0FF203070C3
:108FE0000120287004B070BD2DE9F0411C461746E1
:108FF0000E46054613F0070F0BD102F089FD40B174
:10900000384605F0FDFD00221146012000F0B6FDB6
:1090100003E004F00700022802D00020BDE8F08140
:1090200005F0F1FD287001203070BDE8F08110B529
:10903000104613F0070F08BF05F0A7FE002010BD73
:1090400010B5104613F0070F08BF05F0A5FE00206D
:1090500010BD70B5044603F007000D4602281CBF82
:10906000002070BD05F0A0FE20700120287070BDAA
:1090700003F0070230B4424B4FF0000C012A05D038
:10908000022A04BF1A78022A0BD01EE002201870B0
:109090003D48C3F808C06FF07F410068081A986126
:1090A00013E09A68042A28BF104606D29D69D400AE
:1090B00025FA04F40470501C9860042805D101209E
:1090C000C3F808C008700320187030BC0120704736
:1090D00013F0070F04BF2D4802700020704710B531
:1090E00003F007002649012804BF0020886013D040
:1090F00013F0070F10D18868224B04283CBFD3F827
:1091000000C00CF80020401C8860042804D1042210
:109110001220196800F032FD002010BD2DE9F04743
:109120008C4603F007010024154F1646012904BFA1
:10913000BC60FC606ED013F0070F154BDFF8548055
:1091400007D002293ED0042904BF3878062859D018
:1091500061E0BD68002D08BFFE6130D0012D06D052
:10916000D7F81090AC1E4C4521D2DCB914E0701C2D
:109170003861F9690844B0F5807F88BF3C611EE022
:109180001005011028770100900401102C04011033
:1091900000AA0200554E564D4FF480721946FB4806
:1091A0000BF00AFEFA49F869096820440E54601C65
:1091B000484504D1F548C0F8FC8006203870681C8A
:1091C000B86028E0FF2101703B69C3B1FA69F96812
:1091D0000A44B2F5807F10D2EE4D2D68454518BF88
:1091E000047004D102F5283292F8002A0270481C5B
:1091F000984204BF01208CF80000481CF860012050
:10920000BDE8F0871D461846F9F79EFBDF49284662
:10921000F9F73CFC3C700020BDE8F0870020704767
:1092200070B503F00700DC4C1546012804BF002090
:10923000A06014D013F0070F11D102F069FC70B1D7
:10924000A068D34902283CBF0A681554401CA0609E
:10925000022804D102220968052000F08FFC0020BA
:1092600070BD2DE9F041054603F00700C84CCA4E19
:109270000F4601280AD013F0070F14D002281BD084
:10928000042804BF3078062834D03FE00020B060C6
:109290002168087021684870216888702168C8704A
:1092A0000520307032E0B06804282FD221680A54BB
:1092B000401CB060062028E0B06860B905F093FC5F
:1092C000216808702268010A51702268010C000EA2
:1092D00091702168C870B06804283ABF2168095CA1
:1092E000FF21297024BF01213970401CB06001208A
:1092F000BDE8F08102F00CFC40B12068C178006844
:1093000061F31F6005F06AFC032030700020BDE8A7
:10931000F08170B503F007019F4C064601290BD080
:109320009B4D13F0070F0CD0022914D0042904BF61
:10933000207806281DD025E00020A06005202070A0
:1093400020E0A068B0F5807F1CD229680A54401C38
:10935000A060062015E0A06818B9002128680BF06D
:10936000EEFD2868A168405C3070481CA0600120B8
:1093700070BD02F0CDFB28B1A16828680BF0E4FDB8
:1093800003202070002070BD7FB51C460E460546A8
:1093900013F0070F08D102F0BBFB28B1012202A98C
:1093A000112000F0EBFB03E004F00700022802D0DC
:1093B00004B0002070BD0BF0CCFD2870012030708F
:1093C00004B070BD2DE9F041054603F00700704C74
:1093D000714E0F4601280AD013F0070F14D002284F
:1093E0001BD0042804BF3078062834D03FE000208A
:1093F000B060216808702168487021688870216811
:10940000C8700520307032E0B06804282FD221687F
:109410000A54401CB060062028E0B06860B90BF028
:109420009DFD216808702268010A51702268010CB4
:10943000000E91702168C870B06804283ABF216896
:10944000095CFF21297024BF01213970401CB060E4
:109450000120BDE8F08102F05BFB40B12068C178DB
:10946000006861F31F600BF07EFD03203070002068
:10947000BDE8F0817FB50D46044613F0070F04D018
:1094800003F00700022808D004E0012202A92820E6
:1094900000F074FB04B0002070BD0BF0D8FC20700D
:1094A0000120287004B070BD2DE9F041044603F09E
:1094B0000700394E0F46012804BF0020B06001D0DC
:1094C000022802D00020BDE8F081314DB06860B9BB
:1094D000FDF7ACFC2A68010E11702A68010C51706E
:1094E0002A68010A91702968C870B06804283ABFD8
:1094F0002968095CFF21217024BF01213970401CBB
:10950000B0600120BDE8F0812DE9F04103F00702D1
:10951000214D0E460446012A04BF0020A86001D058
:10952000022A02D00020BDE8F081194FA86830B9A6
:109530000BF01EFD3A68010A117039684870AA687C
:10954000022A3ABF3868805CFF20207024BF0120C7
:109550003070501CA8600120BDE8F0811FB513F0E9
:10956000070F04D1012202A91E2000F007FB04B05E
:10957000002010BD03F00700074901280ED013F0AA
:10958000070F04BF087801280ED01CE094340110A6
:1095900028770100FCAA02001005011001200870C4
:1095A0000020886048610DE08868042805D24B6976
:1095B000401C42EA03224A618860042803D1032048
:1095C00008704869C8610020704703F00700DFF8A1
:1095D00050C4012807D013F0070F04BF9CF8000007
:1095E000022809D01EE002208CF800000020CCF8F0
:1095F0000800CCF8180015E0DCF80800022808D2B2
:10960000DCF81810401C42EA0121CCF81810CCF804
:109610000800022806D1DCF81800CCF8200003204E
:109620008CF800000020704770B403F0070200259A
:10963000FB4C012A02D0022A06D002E00220207050
:10964000A56070BC002070472278022A1CD1D4F893
:1096500020C0A268624528BF10460ED212F0030F48
:1096600004D1E36953F8046BC4E90663237E0370F5
:10967000A069000AA061501CA060604504D10120CF
:10968000A56008700320207070BC0120704770B581
:1096900003F007000025E24C0E46012806D013F027
:1096A000070F04BF2078022805D02BE0022020708D
:1096B000A560A56126E0216AA068884219D2A16947
:1096C000090A41EA0262401CA26110F0030FA06087
:1096D0000FD1E069B0F5303F28BF026006D2B0F587
:1096E000005F03D30422CF49F9F72DFAE069001D8A
:1096F000E061216AA068884204D10120A560307031
:1097000003202070002070BD70B503F0070C002509
:10971000C34CBCF1010F08BFA56033D013F0070F95
:1097200003D0BCF1020F2FD02CE0052A08BFBE48A1
:1097300023D005DC12D2DFE802F01316191C1E003C
:10974000BA48102A006818D0112A08BFB84814D0A7
:10975000202A08BFB43010D0312A10D0656111E042
:109760004FF4005009E04FF42F3006E04FF41C3066
:1097700003E0B04801E04FF42C30606102E008F0F3
:10978000C9FA6061002070BDA268042A07D2C2F144
:109790000303D4F814C0DB002CFA03F30370501C4D
:1097A000A060042824BF01200870012070BD70B49F
:1097B00003F0070C9A4DBCF1010F07D09E4C13F03B
:1097C000070F07D0BCF1020F21D01DE00020A860D8
:1097D000E86019E0A86805283CBF21680A540428FD
:1097E00010D123682268D4F800C0D3F80130696929
:1097F00012781BBA9CF804C023F0FF0343EA0C0361
:1098000041F82230401CA86070BC00207047EB6813
:1098100073B1042B07D22268032B1A4452780270CA
:1098200004BF01200870581CE86070BC012070471C
:109830002268D5F814C012785CF8222026684FEA16
:10984000126C86F801C026684FEA124C86F802C0F6
:1098500026684FEA122C86F803C0D4F800C08CF8B2
:109860000420D8E710B503F00700012804D1002236
:1098700011460E2000F082F9002010BD2DE9F041C4
:1098800003F00704664E174688460546012C04BFC0
:109890000020B06017D013F0070F12D102F038F992
:1098A00078B1B068644902283CBF0A681754401C6C
:1098B000B060022807D102220968072000F05EF993
:1098C00001E0022C02D00020BDE8F081B26812B1A4
:1098D000012A04D009E0FBF735FF287005E0FBF70B
:1098E00037FF2870012088F80000B068401CB06085
:1098F0000120BDE8F08170B503F007000025484C59
:10990000012808D013F0070F0BD0042804BF2078DB
:10991000062825D02DE06561A5616570A5602570DC
:1099200027E0A068022807D2616942EA012161614B
:1099300061781144617010E0042807D2A16942EAFD
:109940000121A16161781144617006E0052804D20B
:1099500061788A4204BF06212170401CA06008E0A3
:10996000D4E9050101F042FA002804BF0120A070EB
:109970002570002070BD10B5294C13F0070F07D0DB
:1099800003F00700042804BF207806281FD028E031
:10999000A068022807D2616942EA01216161617809
:1099A0001144617010E0B0F5817F08D22249096846
:1099B000014401F8022C61781144617004E001BF98
:1099C00061788A4206212170401CA06009E01B4991
:1099D000606901F02DFA002804BF0120A07000206A
:1099E0002070002010BD03F0070CBCF1010F00D067
:1099F000C1E70B49002048614870886008707047D3
:109A000030B403F007050024DFF814C0012D17D08F
:109A100013F0070F1DD0022D4CD0042D64D07FE031
:109A2000100501102805011000AA020040060110CF
:109A30003083011000AF0200287701009434011038
:109A4000CCF81440CCF81840CCF808408CF8004012
:109A500066E0DCF8080002280BD2DCF8141042EAB9
:109A60000121CCF814109CF8011011448CF801105D
:109A700019E0042817D2DCF81810032842EA012163
:109A8000CCF818109CF801301A448CF801200AD147
:109A900006228CF80020DCF81420114304BF4FF498
:109AA0003071CCF818102849401CCCF82810CCF89C
:109AB000080035E0DCF80820042A28BF10460AD246
:109AC000C2F10303DCF82850DB0025FA03F303702E
:109AD000501CCCF80800042803D10120CCF8084021
:109AE000087030BC012070479CF80000062815D192
:109AF000DCF8140000220102DCF818000302104612
:109B0000B2EB930F06D251F8045B401C2A44B0EB31
:109B1000930FF8D3CCF828208CF80040CCF80840FC
:109B200030BC002070474FF42F300168880A424251
:109B300011EB822218BF401C404201EB8000C01C88
:109B400020F0030070470000EFBEADDEE9480022C0
:109B500002704270827002714271C270DFF898C365
:109B6000114601EB410300200CEB43031A54401C47
:109B70000628FBD3491C2029F3D370470BF0FDB90D
:109B80002DE9F04115460E460746F9F7E5FA00F0D3
:109B900008040820F9F7DBFA2A46314638460BF06C
:109BA000ECF905462046F9F7CDFA2846BDE8F081E4
:109BB000D04880787047CF4840787047CD49002022
:109BC00048707047CB490820887170472DE9F041F3
:109BD0000026F8F79AF8044610F00F053ED0284604
:109BE000F8F796F8012D18D0FBF7B2FD44EA0064AF
:109BF000002322460321072004F048FB14F0060F3F
:109C00002CD00126FBF79EFD054605F00DF8074612
:109C1000022D18D0052D09D020E0FBF793FDB549A2
:109C20008A79904218BF8871DED1E7E714F0020FFD
:109C30000CD00120FAF765FD0120F6F711FE002097
:109C4000F6F7A7FD02E00120FAF75BFD022F05D031
:109C5000022D4FF0020004D001F01AF93046BDE8A1
:109C6000F08105F084F8F9E72DE9F84F0027F9F7BE
:109C7000FCFEFBF767FD022804D101F098FD0028E7
:109C800018BF0127FFF7A2FF002818BF0127DFF840
:109C9000649299F80200002800F08082D9F8080048
:109CA0006D464FF0FF34002640B1D9F8082000235C
:109CB0000121084604F0EAFAC9F80860F9F74CFAFD
:109CC00000F0080A0820F9F742FA99F80300DFF8D3
:109CD00028B200B399F8050000EB4001401CC0B267
:109CE0000BEB410189F80500202828BF89F80560A1
:109CF00099F80300401E89F803004C7891F8008021
:109D00000020002C05DD0A1892782A54401C844259
:109D1000F9DC0E704E705046F9F714FA002CC0F2C0
:109D20002D8208F0FF000024292880F0E481DFE87C
:109D300000F0D02A15222D3C1949F650D08D93D130
:109D4000F598B2B8F4F3F2F1F0D0D0D0FCEEEDEC2F
:109D5000EBD0EAD0E9E8E7D0E6E5E0000020FAF74A
:109D6000D0FC10E09DF80000AC280CBF01200220C0
:109D7000FBF7ACFD07E09DF800100120FBF7F7FCB6
:109D8000012089F80100012400F0B5B99DF8031005
:109D9000009861F31F6002F037F901210320FBF7FF
:109DA000E6FC012089F80100EDE7BDF8000040BAAB
:109DB00004F01CFF02210320FBF7D9FC012089F8E5
:109DC0000100E0E79DF801109DF80000FBF7CFFCD3
:109DD000D9E74FF0010A89F801A099F8000088BB83
:109DE000F7F788FF70B39DF8005089F800A0FBF7E3
:109DF000A9FC012808BF002515F0040F18BFFDF7C6
:109E000005F815F0020F07D0FF210F20FCF758FBD3
:109E1000FAF75DFE45F0010515F0010F10D0FBF7D4
:109E200091FC022802D104F0FFFE48B1FBF78AFC46
:109E3000052802D101F037F810B10020FAF730FE02
:109E400089F8006089F8016000F055B99DF80000BC
:109E5000401E01F0E3FA96E79DF8000004F0AAFF27
:109E600091E79DF8000010F00F0F0BD0012001F0DA
:109E700008FD9DF80000102100F00F0001F0DDFC4E
:109E800000F039B9002001F0FCFC9DF80000002131
:109E900000F00F00F2E79DF8000001F0F8FC00F080
:109EA0002AB99DF8000018B1012809D000F023B9A3
:109EB00000200BF067F8002007F02EFF002006E0DE
:109EC00001200BF05FF8032007F026FF012007F0C8
:109ED00044FF10E19DF8000010B3FBF733FC0228AB
:109EE00018BF012404F04BFF01460220FBF73FFCA2
:109EF00001E1FCE04805011094350110F0E0EAE0D2
:109F0000CBE0C5E0CEE07AE033E02DE027E01BE0D7
:109F10000BE0A3E094E08DE074E065E03BE04CE012
:109F200000210620FBF723FC2DE79DF80000002808
:109F300018BF012004F00BFF9DF80000002818BF97
:109F4000012000F09BFFD6E0002000F097FF0021E9
:109F50000520FBF70CFC012001F002F8CBE09DF896
:109F6000000004F0DFFEC6E0BDF8000004F07FFF53
:109F700009E79DF8000020B101283FD0022805D054
:109F8000B9E04FF42F30F8F7DFFCB4E001F0E6FD64
:109F900000210420C6E7F9F7DFF800F008040820E4
:109FA000F9F7D5F899F80300002808BF89F802608E
:109FB0002046F9F7C7F80121B3E79DF80000012812
:109FC00004BF02210520ADD0022804BF00210320D8
:109FD000A8D0032804BF00210420A3D004281CBF5C
:109FE000022108469CD09DE79DF80300009A0023BB
:109FF00060F31F626221072004F048F97BE0FAF762
:10A000009BFFC0E69DF800009DF80110000140EAAA
:10A01000111005F03CFD9DF801109DF8020001F0C3
:10A020000F0140EA012005F038FD9DF8030005F01E
:10A0300040FD2AE0BDF8000040BA05F01CFD5AE0E2
:10A040009DF8000005F04DFD9DF8010005F053FD61
:10A05000BDF8020040BA05F058FD4CE09DF8000044
:10A0600005F068FD9DF801009DF80210000140EA2E
:10A07000111005F06FFD9DF802109DF8030001F02E
:10A080000F0140EA012005F05BFD05F099FD32E08B
:10A090009DF8000004F06FFF75E69DF8000004F0E5
:10A0A00072FF70E60AF041FF9DF8004004F03DFFAA
:10A0B000012C0AD0022C08BF40F0805005D0042C9F
:10A0C00014BF082C40F0005001D104F0AFFE204630
:10A0D0000AF05DFF57E69DF800000AF05DFF0AE018
:10A0E0009DF800000AF05DFF04F0D4FD03E09DF848
:10A0F00000000AF05BFF0CB101273FE0D9F808002F
:10A100006D464FF0FF3440B1D9F8082000230121FB
:10A11000084604F0BBF8C9F80860F9F71DF800F02C
:10A12000080A0820F9F713F899F8030000B399F822
:10A13000050000EB4001401CC0B20BEB410189F867
:10A140000500202828BF89F8056099F80300401E03
:10A1500089F803004C7891F800800020002C05DD80
:10A160000A1892782A54401C8442F9DC0E704E7012
:10A170005046F8F7E7FF002CBFF6D3ADF8F7ECFF39
:10A1800000F008040820F8F7E2FF99F8031000290E
:10A1900008BF89F802602046F8F7D4FF002F14BFEB
:10A1A00001200020BDE8F88F02460020022928BFC8
:10A1B00070473AB1012A0DD0022A04BFFA4800EBD9
:10A1C00081107047C1EBC10000EB4000F74901EB83
:10A1D0008010704701EB810000EBC100F44901EBF6
:10A1E000C000704770B5F8F7B7FF00F00806082008
:10A1F000F8F7ADFFEF4C00256078FF2806D24FF44A
:10A200002861EA480AF0DDFDA570E570A079FF2815
:10A2100005D2D021E6480AF0D4FDE5712572E07A36
:10A22000FF2805D28021E0480AF0CBFD2573657335
:10A230003046BDE87040F8F785BF00FB01F3B3F589
:10A24000287F88BF7047DB4B9A61C3E904017047E0
:10A25000DFF860C30028DCF8103018BF0360D54871
:10A260000029406918BF0860002A1CBFDCF81810DC
:10A27000116058437047CF48012101710078CB49E4
:10A2800080F00100C0EBC00000EB400001EB80104B
:10A290007047C8488278002132B1C27822B902786A
:10A2A00082F001020270817001717047C1491E285D
:10A2B0004A78487008BF002003D01F2808BF01203B
:10A2C00000D1087010467047BA480078B74980F04E
:10A2D0000100C0EBC00000EB400001EB80107047B4
:10A2E000F0B4B44E96F800C0B04CCCEBCC0C356951
:10A2F0000CEB4C0C04EB8C1C03FB05F40CEB440C3A
:10A300008D4234BF2C460C467669F31A934238BF0F
:10A310001A460026002A9CBFF0BC70470023002C80
:10A3200006D930F813702CF813705B1C9C42F8D8D7
:10A33000761C0CEB450C00EB41009642EED3F0BCD2
:10A3400070472DE9F0419B4F14468C4601467A78C0
:10A3500006981D468A4218BFBDE8F0810121F970B8
:10A36000012802D0022825D02AE038788F49C0EB96
:10A37000C0003E6900EB400001EB8011A64234BFF3
:10A38000324622467869A84238BF05460023002D90
:10A3900016D90020002A06D91CF8007021F8107088
:10A3A000401C8242F8D85B1C01EB4601A444AB423E
:10A3B000EFD305E000232A4621466046FFF790FFD1
:10A3C000BDE8F04100F091BB002808BF7047794913
:10A3D000794B4A7879491B78002A097818BF022AF4
:10A3E00005D0042A18BF092A01D0012278E7744A4F
:10A3F0001278012A84BF734A1378012200F08FBBC0
:10A400002DE9F04F6B4C83B00121E1706E49627809
:10A410006B4D0F7868496B4E112A91F800A032D02D
:10A420000EDC002A18BF022A1ED0042A18BF092AEF
:10A430001AD0A0B1002352463946FFF751FF0EE073
:10A44000122A18BF132A1ED0212A18BF222AF0D19F
:10A4500028B100230AF102023946FFF741FF03B099
:10A46000BDE8F04F00F041BB2978012903D95749D5
:10A4700096F800A00F780028F1D000235246394604
:10A4800000F04DFBEBE7F7F723FBF7F77DFA0090C1
:10A49000002818BFF7F7B6FC2878012888BF96F87F
:10A4A00000A0F7F72FFC10F0040F18BF0AF1010A03
:10A4B000474801906078A0F1110920783B49C0EB32
:10A4C000C00000EB400001EB80152069B84238BFA6
:10A4D00007466069504538BF8246F7F7D0FC83468F
:10A4E0000020F7F78EFF0026BAF1000F34DD0024BC
:10A4F000002FC4BF019800EB861826DD1BF904006D
:10A50000202824BF002025F814001BD200EBD071B6
:10A510004910C00758F82110C00E21FA00F081B28E
:10A520004FF0FF30B9F1000F1CD0B9F1010F08BF97
:10A53000C8B205D0B9F1020F04BF0846F7F767FFAC
:10A5400025F81400641CBC42D8DB1A48761C56451A
:10A55000006905EB4005CADB0098002818BFF7F733
:10A5600054FC7CE711F4005FC1F3042018BF4042A3
:10A57000E6E7104801214172407980F0010000EBCC
:10A58000800101EBC0000A4901EBC0007047094897
:10A59000C279002132B1027A22B9427982F00102F5
:10A5A0004271C17141727047A441011054360110CB
:10A5B000D440011054050110D6040110DC04011030
:10A5C000D7040110D9040110D5040110D8040110DA
:10A5D00000400030FA491E288A79887108BF00209F
:10A5E00003D01F2808BF012000D1487110467047D2
:10A5F000F348407980F0010000EB800101EBC000DE
:10A60000F04901EBC00070472DE9F04FEE4985B0ED
:10A61000012291F80080ED4991F80090E8490A7212
:10A620008979E84C11291CBF1229132936D0F8B1B9
:10A63000E349497901EB810202EBC10104EBC1025C
:10A64000002119EB080C18BFE14C11D02368B9F1B7
:10A65000000F5B8A03BF30F811500B4422F81350EF
:10A6600030F8113018BF22F81130491C8C45EDD854
:10A67000F8F772FD00F008050820F8F768FDD04CE7
:10A68000607A002818BF01217ED0E1712846F8F7D2
:10A6900059FD0020207205B0BDE8F08FF7F718FAD9
:10A6A000F7F772F90190002818BFF7F7ABFBC44821
:10A6B0008179A1F11105C1690091407900EB800118
:10A6C00001EBC00004EBC006F6F79CFBC14FC2498A
:10A6D0004FF0110A002804BF8B46012004D0BB466E
:10A6E00050460F464FF0010AF7F78BFEF7F7C5FB10
:10A6F00000240390B9F1000F29D90098800102903D
:10A7000003980057202824BF002026F814001BD2ED
:10A7100000EBD0720299521001EB8201C00751F890
:10A720000B10C00E21FA00F081B24FF0FF30002D67
:10A7300048D0012D08BFC8B204D0022D04BF08467E
:10A74000F7F765FE26F81400641C4C45D8D306EBD9
:10A7500049065046F7F755FEF7F791FB002482466D
:10A76000B8F1000F28D90098A3464FEA80191AF9CA
:10A770000400202828BF26F814B01AD200EBD071AC
:10A78000491009EB810100E02AE0C959C007C00E59
:10A7900021FA00F081B24FF0FF30D5B1012D08BF92
:10A7A000C8B204D0022D04BF0846F7F730FE26F8E1
:10A7B0001400641C4445DAD30198002818BFF7F749
:10A7C00024FB55E711F4005FC1F3042018BF404299
:10A7D000B8E711F4005FC1F3042018BF4042E6E778
:10A7E000607980F00100607100214EE7744801211A
:10A7F0008173807A794980F0010001EB8010704705
:10A800006F48027B002132B1427B22B9827A82F00A
:10A810000102827201738173704769491E28CA7AE6
:10A82000C87208BF002003D01F2808BF012000D134
:10A830008872104670476248807A684980F001004B
:10A8400001EB801070472DE9F04F5D4987B04FF064
:10A85000010B81F80DB0C97A604D614C11291CBF04
:10A86000122913292CD0A8B15549897A237805EBF0
:10A87000811294F801C0002113EB0C0F0AD030F8BC
:10A88000113022F81130237894F801C0491C634438
:10A890008B42F4D8F8F760FC00F008050820F8F7C0
:10A8A00056FC474CA07B002818BF84F80CB07FD022
:10A8B0002846F8F747FC0020607307B0BDE8F08F2A
:10A8C000F7F706F9F7F760F80490002818BFF7F7D4
:10A8D00099FA444806902078617800EB01083848DE
:10A8E000C17AA1F11109C1690591817A806905EBED
:10A8F000811A404538BF8046022000901220002572
:10A900002E4601906C465DF82600F7F77AFD54F864
:10A910002600F6F7C9FD0290002004460390069831
:10A92000059900EBC61000EB81172CE0E01704EB53
:10A93000D060421102A920F01F0051F82210201A05
:10A940000BFA00F001421DD004EBD470401007EB6D
:10A950008000E107D0F84009C90EC84081B24FF02D
:10A96000FF30B9F1000F1CD0B9F1010F08BFC8B218
:10A9700005D0B9F1020F04BF0846F7F748FD2AF8E1
:10A9800015006D1C641C4545B8BF202CCEDB761C21
:10A99000022EB7DB0498002818BFF7F736FA79E7DC
:10A9A00006E011F4005FC1F3042018BF4042E6E75F
:10A9B000A07A80F00100A0720021217378E70000E6
:10A9C00054050110D4400110DA040110DB04011019
:10A9D00040060110C048003040480030A44101103A
:10A9E000DD0401100040003070B50D466F490122B2
:10A9F000CA706F4A497816786E4A212914781EBFAA
:10AA00002229232970BD002818BF002D11D0002352
:10AA100022463146FFF764FC631C0122214628468A
:10AA2000FFF75EFC05EB4400A31C01223146FFF753
:10AA300057FCBDE8704000F058B870B55B4D044657
:10AA4000687868B9E06858B15B490978012994BF12
:10AA500058495A490B785A490122097800F05FF8A1
:10AA6000E87A112804BF0020FFF7EDFEE87A1228EB
:10AA700004BF0020FFF7E7FEE87A132804BF002098
:10AA8000FFF7E1FE6878002804BFA068FFF7B8FC74
:10AA90006878112804BF0020FFF7B2FC68781228FC
:10AAA00004BF0020FFF7ACFC6878132804BF002027
:10AAB000FFF7A6FC206920B1A979002908BFFFF79C
:10AAC000A3FDA879112804BF0020FFF79DFDA879F8
:10AAD000122804BF0020FFF797FDA879132818BF9C
:10AAE00070BD0020BDE870408EE570B5F8F734FB0E
:10AAF00000F008060820F8F72AFB2C4C20790025E6
:10AB0000002801BF207880F001002070A5701CBFD4
:10AB10000120A0703046F8F715FBE57070BD2DE9F7
:10AB2000F047994616460D460446F7F7ADF95FEA39
:10AB3000000C1DD01D490878224AC0EBC000D1F896
:10AB4000108000EB400002EB801009FB08F200EBE4
:10AB50004200454594BF2F4647464969A1EB09018C
:10AB6000B14238BF0E460021002E09D8BDE8F0875B
:10AB70004B46324629462046BDE8F047FFF7B0BBBA
:10AB80000023002F08D91CF9032034F8122020F8E4
:10AB900013205B1C9F42F6D8491C00EB480004EBD5
:10ABA0004504B142ECD3BDE8F08700005405011024
:10ABB000D5040110D6040110D7040110D9040110E6
:10ABC000DC040110543601106849002814BF00202D
:10ABD0000120087070476548007800280CBF0120EC
:10ABE000002070476148017879B14FF040214A69EF
:10ABF00042F001024A618A6912F0010F05D00A6B26
:10AC00005B4B22F440521A430A6300214160816089
:10AC1000C160016170475548017879B14FF040211A
:10AC20004A6942F001024A618A6912F0010F05D0B7
:10AC30000A6B4F4B22F440521A430A6300214160D1
:10AC40008160C1600161704770B50446F8F784FA0D
:10AC500000F008050820F8F77AFA444A454900232D
:10AC6000D06801EBC001401CD060B0F5807F28BFE8
:10AC7000D3602078087060784870A0788870E07899
:10AC8000C8702079087160794871A0798871E0797D
:10AC9000C8711069B0F5807F3CBF401C106116D3AD
:10ACA0001D20087001204870207888706078C87076
:10ACB000A0780871E0784871207988716079C8714E
:10ACC0009068401C9060B0F5807F28BF936050680A
:10ACD00040F001005060107888B14FF04020416989
:10ACE00021F001014161016B11F4405F07D0016B5C
:10ACF00021F4405141F4BE0141F020410163284656
:10AD0000F8F720FA012070BD00B50178427883B0D1
:10AD1000890141EA82018DF80010418809098DF806
:10AD20000110818809098DF80210817801F00F0265
:10AD3000017962F31F118DF80310017A8DF8041068
:10AD4000417A8DF805108179C27901F03F0102F056
:10AD50000C0241EA02118DF80610C07980018DF8CD
:10AD600007006846FFF770FF03B000BD74050110CF
:10AD700000205FA024420110194A002112684FF000
:10AD8000402312F0804F26D0164AD2F800C05FEA66
:10AD90001C4C04D011686FF30F0141F00101D2F88F
:10ADA00000C01CF47F4F0CD011684FF0020C01F46E
:10ADB0007F414CEA0121DFF830C0DCF800C0C3F865
:10ADC00074C0D2F800C01CF0FF0F04D01168032239
:10ADD000C9B242EA014199678069D867FEE700007D
:10ADE0002CED00E028ED00E038ED00E070B50E46F7
:10ADF0000446FAF7A7FC042811D1A4F51C705028CA
:10AE00000DD2A019A0F27120502808D225020024EA
:10AE1000002E04D92846F7F797FD012801D000201D
:10AE200070BD641C05F58075B442F3D3012070BD7C
:10AE300070B50D460446FAF785FC04280AD1A4F53E
:10AE40001C70502806D220022946F7F71FFE012861
:10AE500008BF70BD002070BD10B5074CFEF704FFA1
:10AE6000012808BF10BD206800F040FF002818BF6F
:10AE7000FAF7C0FCF2E7000040060110FE4A002885
:10AE8000516814BF41F0010021F00100506070478B
:10AE9000F94B59680A0E120721F07F4142EA00601F
:10AEA000084358607047F4484068C0F30360704737
:10AEB000F1484068000F7047EF4880697047EE49DD
:10AEC000012088617047EC49002088617047EA489A
:10AED00040697047E849012048617047E649002011
:10AEE000486170472DE9F041AEB0002707F0FDF84A
:10AEF0000646A02102A809F064FF002425464FF071
:10AF00000308305D10F0800F18D0601C8DF8A90088
:10AF10008DF8AF508DF8A880ADF8AC508DF8B050DA
:10AF2000ADF8AA508DF8AE508DF8B1508DF8B450F0
:10AF3000355501272AA902A8F5F7DDFA601CC4B22D
:10AF40000A2CDED3012F06D1102302AA06210120EC
:10AF5000009508F067F80AF02EF82EB0BDE8F081F1
:10AF6000C549FF220A70C8617047C348007870471E
:10AF7000C149C8627047C04908637047BE48006B4A
:10AF800070472DE9F04FDFF8F48287B0D8F8000061
:10AF9000B0F90E11B0F90C0109F081FFF5F773FB60
:10AFA0000120F9F7AEFB0AF00BF8D8F80000B24F19
:10AFB000D0F8F800C0F30344C0F30321C0F3033515
:10AFC0008C420DD10F2D0BD003F021FF20B109F0E1
:10AFD000ACFF082818BF2C46786BA04218BF7C63D2
:10AFE0002046F9F78CFB09F0F0FF002818BF06F0A7
:10AFF0001AFBFAF7A7FB05284ED1DFF884B24FF011
:10B00000000A4FF040297868C7F808A0C7F80CA0DC
:10B01000C0F30365C7F810A0D8F80000A900D0F865
:10B02000F80020FA01F101F00F04C0F30321C0F38E
:10B0300003368C420DD10F2E0BD003F0E8FE20B169
:10B0400009F073FF082818BF3446786BA04218BF78
:10B050007C632946052003F0A7F9002D00F0E68067
:10B06000022D27D0042D00F0E58078680A2D4FEAE4
:10B07000106120F07F404FEA017118BF41F000716C
:10B0800008437860FEF7F0FD012805D009F093FF32
:10B09000FAF758FB0528B6D0F9F732FB09F09AFF0A
:10B0A000FAF750FB02287CD007B00020BDE8F04F33
:10B0B000F5F76FBB0F2509F098FE002818BF0E2585
:10B0C000386B012805D1D8F80000D0F8F800C0F39B
:10B0D000036429462046FAF74AFC0028D2D009F03A
:10B0E0007EFF09F081FFF9F7B0FA040078D1386BE0
:10B0F000012841D00020F6F7DBF86248F6F78DFC16
:10B100000120F6F77FFCF8F749F85F48F8F7FBF8FD
:10B11000F8F7E2F8F8F70BF94100D8F80000B0F8BA
:10B120000621B1FBF2F1491CC1F34F01798090F87F
:10B130000801787058B1F8F7FAF8D8F80010400014
:10B14000B1F80411B0FBF1F0401CC0F34F01084608
:10B15000F8F75EF84D48C9F81800F6F7B9FCF6F7AD
:10B160001EFE787880B1401E10F0FF00787004BF9A
:10B170007888F8F74DF807E000231A469321072056
:10B1800003F084F8F6F7D2FD7868C0F3036529462A
:10B190000520F5F7ABF8FEF767FD012808D07868C1
:10B1A00000E04BE0C0F30360A84208BF002C1ED0B3
:10B1B000C9F818B0386B012804BF0020386308D0E4
:10B1C000F8F75EF8F8F793F80020F8F79CF8F7F72F
:10B1D000EEFFF6F77DFCF6F7D9FB0020F6F71DFC35
:10B1E00009F002FF09F005FFFAF734FD4AE7684667
:10B1F000F6F793FF70B16846FFF71FFC0198F8F768
:10B2000017FD684609F0FAFE0446F6F7CEFFFAF796
:10B2100012FBC0E7D8F80000406E10F0704F02D06B
:10B22000FAF7E8FAB7E7FAF70DFBB4E7204609F0BA
:10B23000EAFE27E7204603F0A1FF23E70120FBF702
:10B24000E9FDF5F707FB10B9F5F7FEFA58B1002054
:10B25000F5F706FB0020F5F700FB07B00120BDE87D
:10B26000F04FF5F796BA0120F5F7FAFA0020F5F756
:10B2700090FA07B00CE000008805011040060110AC
:10B2800000005FA00D9D00105995001007005FA001
:10B29000BDE8F04F09F0C2BD7047002808BF7047F5
:10B2A00080220146014809F087BD7047244A0110F9
:10B2B000704708283CBFFE49087070470020FC49D1
:10B2C00088604860FB48006890F88100082838BF13
:10B2D000087070470020F64948607047F4480078CD
:10B2E000704770B5F34D0024286890F86C0010F09A
:10B2F000020F0BD0FAF726FA022807D1EC4829688A
:10B30000007801EB8000B0F8840084B2204670BD64
:10B3100070B5E84D4FF48054286890F86C0010F038
:10B32000020F0DD0FAF70EFA022809D1E048296879
:10B33000007801EB8000D0F88400000CC0F3130407
:10B34000204670BDDA488078002818BF0120704779
:10B350002DE9F041FAF7F6F9022803D103F064FC75
:10B36000022803D04FF48050BDE8F0814FF480559F
:10B370002E4603F01CFDCF4F0446DFF834833868B7
:10B3800090F86C1011F0010F0ED0B0F87600D8F8DC
:10B3900008104042814207DC34B10020641EC8F826
:10B3A0000800204603F006FD396891F86C0010F0A3
:10B3B000040F18BF002C0AD0B1F87C00621E904028
:10B3C000B1F87E20824238BF1046C0F31306D1F890
:10B3D000A40010F0020F1CBF98F80210002902D040
:10B3E000000CC0F31305B54298BF354609F0FDFCCB
:10B3F00010F4817F0FD0FAF798FA01463868B0F858
:10B400005800C0F3033081421CBF4FF40050B5F523
:10B41000005F38BF05462846BDE8F0812DE9F04FB2
:10B42000DFF890A287B0DAF8001091F86C2012F0E3
:10B43000020F0DD09E4A91F88090DFF87CB2177809
:10B44000002809DB484503D2B84218BF064643D15D
:10B4500007B00020BDE8F08F3E464FF0FF38F6F70A
:10B4600095FAF7F734F80025B9F1000F34D9DAF876
:10B470000000002400EB8500B0F8840081B2204673
:10B48000F5F734FFF6F78BFC6846F6F746FE002822
:10B4900066D0029878B1014688489BF80020007871
:10B4A0005043421E07D331F9020B0028B8BF404277
:10B4B0000444521EF7D2F6F778FEF6F767FA002337
:10B4C00022469221072002F0E1FEA04584BF2E46CD
:10B4D000A0466D1C4D45CAD3B74244D0082E3CBF90
:10B4E00073490E70DAF80000B0F8821039B300EB3F
:10B4F000870200EB8600B2F88420B0F8840092B294
:10B5000080B2801A484340F30F34F8F72DFC6C4B9F
:10B510009BF80020002193F800C002FB0CF2002AE7
:10B520000DD930F81120224420F811209BF800207A
:10B5300093F800C0491C02FB0CF28A42F1D84FF488
:10B54000800003F029FDDAF80000002300EB8600FC
:10B550008021B0F8840082B2072002F097FE09E053
:10B56000FAF748F990E703F022FC03283CBF401C9F
:10B5700003F020FC012007B0BDE8F08F4D484C4996
:10B580000068B0F87600424288688242BCBF401E24
:10B59000886070472DE9F04F91B093460E460446FF
:10B5A0004FF0000A03F003FCDFF80881404F05006C
:10B5B000D14610D109F02CFDD8F80010B1F8781060
:10B5C000884208D30120C7F8089003F0F3FB11B0BC
:10B5D0000120BDE8F08F002E1FDDB8680028B8BF3D
:10B5E000C7F8089007DBD8F80010B1F8741088424B
:10B5F000BCBF401CB860D8F80000B968B0F874004F
:10B60000884215DC032D13D2681CC7F8089003F09C
:10B61000D1FB11B00120BDE8F08F09D1D8F80000AE
:10B62000B0F876004142B8688842C4BF401EB86096
:10B63000B87850B1D8F8000090F8A40010F0040FCA
:10B640001EBF002011B0BDE8F08FD8F80000B0F99F
:10B6500072108C420EDD796821447960B0F86E007A
:10B66000884210DC4FF0FF30C7F80490FFF7D6FE99
:10B67000824608E07868002805DD002CD4BF01214F
:10B680002146401A7860DFF83C9099F800000728BE
:10B690003AD10D48594600784200684609F09BFBB4
:10B6A000ADF80040ADF80260ADF8045038890DE007
:10B6B0002006011040060110D5040110D904011024
:10B6C000D604011055050110DC040110ADF8060088
:10B6D000B888ADF80800D8F80000B0F87210ADF8DE
:10B6E0000A10B0F87410ADF80C10B0F86E10ADF888
:10B6F0000E10B0F87600ADF8100099F80000072899
:10B7000004BF6846FEF760FE504611B0BDE8F08FFA
:10B710003D4810B50068D0F8A40010F4807F06D032
:10B72000C0F30330012101FA00F0F7F782FA37493C
:10B7300000204870887010BD70B5344D0024A87882
:10B74000002814BF01260026687828B903F03EFBC4
:10B75000002808BF002100D001218E4225D00A1CFC
:10B7600018BF0122AA7028480068D0F8A43013F04E
:10B77000040F0ED021B1C3F30310082808D206E04D
:10B780000021A960696090F88100082800D2287023
:10B79000012413F0020F18BF0124002A18BF012250
:10B7A00000238221072002F071FD204670BD16495A
:10B7B00000200968D1F8A41011F4807F08BF7047F9
:10B7C000DFF848C09CF80120131C18BF012330B4D7
:10B7D0000F4CC1F30332E46B012505FA02F222405B
:10B7E00011F4007F01D00AB102E00AB1002100E0AB
:10B7F00001218B4204BF30BC7047081C18BF0120D8
:10B800008CF8010030BC97E74006011020060110BB
:10B8100000100040A148C079704710F5167FA8BFFE
:10B82000704701209D49C87170479C490020C8712C
:10B8300070479A4890F90100704770B5974E0446DA
:10B840000D4696F90100A04213D0F9F77BFF0228BC
:10B850000AD1B4F1FF3F07D0357044EA0522002336
:10B860006421072002F012FD7470002C04BF002038
:10B87000F071F9F767FF05281CBFB4F1FF3FB47002
:10B8800070BD8649C87070478448C07870470246CA
:10B8900000F00F0011210228A8BF70477F4B12094A
:10B8A000002818715A7108BF0021C6E77B4840790B
:10B8B00070477A480079704710B50446F9F760FC84
:10B8C0000146764A2046012982BF0021917110BDB0
:10B8D0009179142905D8491CC9B29171142938BF2E
:10B8E00010BD002010BD70B50C46054609F095FB53
:10B8F00000214FF0140C0DB30022401E00281DDD66
:10B9000035F91230002BB8BF5B429BB2634511D9A9
:10B910000221B3EBCC0F88BF032009D8B3EB8C0F07
:10B9200088BF022004D8B3EB4C0F8CBF012000204D
:10B93000207003E0521CD2B28242E1DB084670BDA7
:10B940002DE9F84F1D4692468046CCB2002709F0FB
:10B9500069FB009009F06BFBDFF840910646BB469F
:10B9600099F90100B0F1FF3F04BF99F802000128E6
:10B9700008D1F9F7E7FE052804D002240127CAF808
:10B9800000B069E054EA050006D0002C64D096F8B7
:10B99000E804012860D14DE0307B80B196F8420088
:10B9A00000281CBF02242746F1D196F8E80401289C
:10B9B00019BF96F8EA04012802240327E7D05D4660
:10B9C000D8F8148009F029FB002414220146B8F1AC
:10B9D000000F20D000204B1E002B1CDD38F910106A
:10B9E0000029B8BF494289B2914210D90224B1EB73
:10B9F000C20F88BF03250ED8B1EB820F88BF022586
:10BA000009D8B1EB420F8CBF01255D4603E0401C15
:10BA1000C0B29842E2DB002C18BF45F0A007B6D1B7
:10BA2000DAF800002C2817D2307B002818BF022437
:10BA300012D0ACE7F9F7A4FB012888BF89F806B05B
:10BA40000AD899F80600142805D8401CC0B289F815
:10BA50000600142800D3002499F80300012804BF2D
:10BA6000002C02240098007D012808BF002499F8CA
:10BA70000500012807D074B139460120FFF7DDFE2B
:10BA80002046BDE8F88F99F8040010F0FF0F14BFAE
:10BA900002240024F0D100210846EFE72C06011013
:10BAA00070B47E487E49002442681068884204BF12
:10BAB0005068B0F5087F25D19068B0F5605F21D857
:10BAC0007849D5688D4220D04FF0000C134661466E
:10BAD000BCEB900F07D253F8046B491C7440B1EBD8
:10BAE000900FF8D374B9116A79B10021B1EB900FBE
:10BAF00006D252F8043B491C9C44B1EB900FF8D39A
:10BB0000654502D070BC0020704770BC01207047B2
:10BB10006248007870476148406800F5407070479F
:10BB20005E48406800F58070704710B55B4C4FF47C
:10BB30001C306060FFF7B4FF70B1606800F5807082
:10BB400000F0D4F840B1606800F5407000F0DDF816
:10BB500010B10120207010BD002010BD4F49002001
:10BB600008704FF41C30F6F7EFBE4C48017841B135
:10BB700040684B4A0168914202BF4168B1F5087FB5
:10BB8000704700207047454B5B6803F5807318448D
:10BB9000F6F7D9BF414B5B6803F540731844F6F7DD
:10BBA000D2BF3E484068006970473C4949680A690D
:10BBB00082429CBF00207047C0EBC00001EBC00078
:10BBC00000F580607047354A526802EB80035B6A7B
:10BBD0001A44354B53F820C0403333F810000CEBB7
:10BBE0000003401E5B1E23EA000000FB012070479B
:10BBF0002A49886070472948806870472DE9F00F0E
:10BC0000264B0022DFF8A080D3E90145012708F187
:10BC100040069146831893F928C0BCF1000F18DB49
:10BC200007FA02F32B4214D0D3B204EB830A58F87C
:10BC300023B036F81330DAF824A09B445B1EABF136
:10BC4000010BA2442BEA030303FB0CA341F82230AF
:10BC500001E041F82290521C102ADBD3BDE8F00F1E
:10BC600070470029B8BF704730B494460B4A0F4C58
:10BC7000526802EB80035B6A13440B4A52F820209F
:10BC800034F810001418401E641E24EA000001FB62
:10BC9000003030BC6146F6F756BF00003406011094
:10BCA00054465053EFBEADDE2C7701006C77010097
:10BCB00010B5FFF73AFFA8B1FFF72DFF0146D022DC
:10BCC000174809F079F8FFF72BFF164C01464FF49F
:10BCD000E272206809F070F82068406DBDE81040FD
:10BCE00002F0EEBF0220F9F7F1FDE2E758B10E4A8B
:10BCF0000168914207D1406820F00F00B0F5107F35
:10BD000004BF012070470020704730B1006820F068
:10BD10000F00702804BF012070470020704700000A
:10BD2000308301104006011041505352AD4810B508
:10BD3000806810F0020F15D0F5F726FE90B1F5F7E8
:10BD4000E6FD0402F9F7FEFC44EA0044F9F700FDC1
:10BD500044EA00604EF2AF0108434FF04021C8674B
:10BD6000012010BD002010BD10B572B60120F6F7FD
:10BD7000EBFCF7F797FBF7F7C1FB4FF0FF30F7F756
:10BD8000E6F9994880234FF40052002152F821C06F
:10BD900040F821C0491CB1EB930FF7D3F7F7E9F94D
:10BDA000F7F728FEF7F74AFE9048F7F763FE012001
:10BDB000F7F721FEF6F75AFD1E20F7F711FEF7F709
:10BDC000B9FBF6F741FFF7F7CDFDF7F71BFCF7F7E7
:10BDD000E1F9F6F7B1FFF5F7ECFDFFF769FFF7F7CB
:10BDE00060F9F7F72BF9FDF7B1FEFBF7E5F8FEF781
:10BDF00012FF62B6F9F7B1FD7D4C206890F864003F
:10BE000000F00F00F6F7C4FB2068018BC1F3072296
:10BE1000418A008AFEF711FA2068806E000C02F059
:10BE200032FA744809F008F92068B0F90C0109F0F9
:10BE300008F9F4F740FAFFF73BFAF7F737FEF9F79E
:10BE400094FFFFF729FA09F001F9206890F8200023
:10BE500010F0010F04BF0021032003D002F08FFF78
:10BE600001460220F9F783FC4FF0402420690023AB
:10BE700000F070021946022002F008FA206910F062
:10BE8000200F17D0226F00230521072002F0FEF9B2
:10BE9000626F00230521072002F0F8F9A26F00234A
:10BEA0000521072002F0F2F9E26F002305210720A7
:10BEB00002F0ECF9FFF72CFC0020206710BD0224F3
:10BEC0004D4DFDF7D1FE012806D0F9F73BFC0328C4
:10BED00002D102F096FA58B3002D05DC02F04FFFB4
:10BEE00001460220F9F743FCDFF814914FF00108F6
:10BEF000424FDFF810A14FF04026A9F1030BF9F7EC
:10BF000021FC0546F9F724FC0146284602F04CFACC
:10BF1000F9F71EFC01462846F4F7E8F9FDF752FE52
:10BF2000072D5BD2DFE805F05A1D08272A192D00DE
:10BF30006D1E002DC5DCD1E7387850B9FAF710FF37
:10BF400038B900231A462021072002F09FF987F80C
:10BF5000008003F0F1FB0224D1E7FFF712F805247B
:10BF6000CDE7FAF763FEF9F7EDFB012804BF2046A1
:10BF7000F9F7FAFBC3E702F0E9FDC0E7FEF76CFF53
:10BF8000BDE7C6F81890F7F709F9F7F7A5F9F7F73D
:10BF9000CEF94000AAFB00104009401C4008F7F70A
:10BFA00037F9FDF761FE01280CD1F9F7CBFB062824
:10BFB00008D0F7F765F9F7F79AF9F7F7F8F8C6F840
:10BFC00018B09CE7F9F7C1FB0546F9F734FC15B149
:10BFD000F9F738FCE5E7F9F70DFCE2E70220F9F79D
:10BFE00075FC8CE70080004000860110DDDC00005D
:10BFF0004006011030830110FF700200440601105A
:10C0000003005FA0CDCCCCCCFE4908607047FD4951
:10C0100048607047FB4810B44068002808BF4FF4E0
:10C020002C30F94A016891421CD14168B1F5007F7A
:10C0300018D3836800228446B3F5056F88BF4FF498
:10C0400005630021B1EB930F24BF10BC70475CF86F
:10C050002140491C2244B1EB930FF8D3002A04BFBE
:10C0600010BC7047002010BC704770B50022C26041
:10C07000D0F808C0012113460446BCF5056F88BFFF
:10C080004FF4056C0022B2EB9C0F06D254F82250FC
:10C09000521C2B44B2EB9C0FF8D35A42C260D94ACF
:10C0A000127812F0800F07D14FF42C304FF4056254
:10C0B0002146F6F748FD014601290CBF012000206A
:10C0C00070BDFF2270B50025044605614FF4006184
:10C0D000503008F0ADFEA584E584E562A562656395
:10C0E0002563E563A56365642564E5640120A564B3
:10C0F00070BD2DE9F0414FF42C310446C24E086862
:10C10000B04218D14868B0F5007F14D38A68002384
:10C110000D46B2F5056F94BF94464FF4056C0020B0
:10C12000B0EB9C0F26D255F82070401C3B44B0EB7E
:10C130009C0FF8D3F3B1FF224FF40561204608F0BD
:10C1400077FE4FF40870C4E900604FF40560A0600A
:10C150000020E06084F8200084F8210084F82200A8
:10C1600084F8230020616061A061E0612046FFF750
:10C17000A8FF07E0B2F5056F88BF4FF405622046BF
:10C1800008F01AFE0120BDE8F08170B402684FF497
:10C1900008715160016801F1500291F821C091F8D5
:10C1A00020300CFB03F102EB41010022BCF1000F37
:10C1B00008D900EB4204521CB4F8F64021F8024BB7
:10C1C0009445F6D80022002B08D900EB4204521CFB
:10C1D000B4F8364121F8024B9342F6D804680022A5
:10C1E00094F82240002C0BD900EB4204521CB4F806
:10C1F000764321F8024B046894F822409442F3D825
:10C200000468002294F82340002C0BD900EB420470
:10C21000521CB4F8964321F8024B046894F823406A
:10C220009442F3D80022BCF1000F08D900EB42047D
:10C23000521CB4F8704021F8024B9445F6D8002205
:10C24000002B08D900EB4204521CB4F8B04021F88E
:10C25000024B9342F6D8B0F8F22021F8022BB0F846
:10C26000F42021F8022BB0F8F02021F8022B002452
:10C270000022BCF1000F88BF00EB841508D905EB44
:10C280004206521CB6F8766121F8026B9445F6D846
:10C290000022002B88BF00EB841508D905EB42066D
:10C2A000521CB6F8766221F8026B9342F6D8641CF1
:10C2B000042CDDD30023D0F800C000229CF822C05B
:10C2C000BCF1000F88BF00EB431C0BD90CEB420400
:10C2D000521CB4F8B64321F8024B046894F822408B
:10C2E0009442F3D8D0F800C000229CF823C0BCF1DF
:10C2F000000F88BF00EB431C0BD90CEB4204521C0F
:10C30000B4F8F64321F8024B046894F823409442B1
:10C31000F3D85B1C022BCED370BC70472DE9F74FCE
:10C3200088B000250A992C462E460968049101F12F
:10C3300050030999002984BF3449D1F800801CD9E1
:10C340000022002888BFB8F9CE700DD933F9021B3E
:10C350000029B4BFC1F1000C8C46BC45BCBF0D44E4
:10C36000641C521C8242F1D30999761C8E42E7D399
:10C37000002CC8BF95FBF4FA08DC4908414301EBE7
:10C380005002049901EB4201B1F950A00021029141
:10C3900001910499503100910021039109990029DC
:10C3A00075D91A49009E069609684FF0000B4FF0A8
:10C3B0000109B1F9C0E0D1F8B4105F46C1F30741FB
:10C3C000D846CDF814B00791002830D9B6F900202E
:10C3D0004FF0000C06999344634600280DD9B1F93B
:10C3E0000040A51A48BF151B7545B8BF0CF1010CDC
:10C3F00001EB49015B1C8342F1D307998C450AD3B9
:10C40000059905E04806011053454C4640060110C9
:10C4100011447F1C059108F1010806EB490680458F
:10C42000D4D3002FC4BF059991FBF7F101DC9BFB2E
:10C43000F0F1039B0A9A09B202EB4302A2F87010D2
:10C44000FE4A1268B2F9BA30AAEB030399420ADD38
:10C45000B2F9B82052448A4205DD019A1144019193
:10C460000299491C02910099099A01EB400100913F
:10C470000399491C0391914293D30299002906DD47
:10C48000DDE9011291FBF2F1019103E0FFE7514672
:10C49000CDF804A00A9AA2F8F210002102910391AB
:10C4A00004995031009100210491002868D9E34992
:10C4B000009F069709684FF0000B099EB1F9BCE098
:10C4C000D1F8B410D846090ED946CDF814B007916A
:10C4D000002E2BD9B7F900204FF0000C0699934499
:10C4E0006346002E0DD9B1F90040A51A48BF151BAF
:10C4F0007545B8BF0CF1010C01EB40015B1CB34268
:10C50000F1D307998C4504D3059908F1010811442A
:10C51000059109F1010907EB4007B145DAD3B8F1FC
:10C52000000FC4BF059991FBF8F101DC9BFBF6F10C
:10C53000049B0A9A09B202EB4302A2F8B010BF4A68
:10C540001268B2F9BA30AAEB030399420ADDB2F9D4
:10C55000B82052448A4205DD039A1144039102999E
:10C56000491C02910099891C00910499491C04916D
:10C5700081429CD302980028C4BF039991FBF0FA32
:10C580000A98A0F8F4A001980A99504400B200EB70
:10C59000D0704010A1F8F0000BB0BDE8F08F2DE98D
:10C5A000F04F146889B015460E460746A1F12008E1
:10C5B000202928BF4FF0FF3A05D24FF0010000FAC2
:10C5C00006F0A0F1010A38BF4FF0000B05D34FF081
:10C5D000010000FA08F0A0F1010B202F3DBF01205F
:10C5E000B840401E4FF0FF3038BF002207D3A7F1FC
:10C5F00020024FF0010101FA02F1A1F10102C6F19E
:10C600002009202E34BF20FA09F100FA08F1B240C7
:10C610001143B040CDE90001206920F4FE602061A3
:10C620008748007810F0010F7ED02A463146384600
:10C6300001F0D1F90020A8616861002F84BFDFF804
:10C64000FCE101221BD905EB4001B1F9B010002932
:10C65000B8BF494209B2DEF80030B3F9CC308B42A2
:10C660000ADD410905EB810100F01F0C4B6902FA5C
:10C670000CFC43EA0C034B61401CB842E3D300209E
:10C68000012F18BFA7F1010E3BD005EB4001B1F916
:10C69000B230B1F9B020991A48BFD11A09B2DFF807
:10C6A0009CC1DCF800C0BCF9C4C08C4526DAB5F9E1
:10C6B000F410B2EB010C48BFA1EB020C0FFA8CFC9A
:10C6C0005A1A48BFCA1A11B28C450BDB420905EB56
:10C6D000820100F01F0C01224B6902FA0CF21A438E
:10C6E0004A610BE0411C4B0905EB830201F01F0C72
:10C6F0000121536901FA0CF119435161401C704545
:10C70000C3D36969E869B14008432063A969286A0D
:10C71000B140014361636869202E34BF20FA09F0FB
:10C7200000FA08F0084300E000E060634448006855
:10C73000079010F0040F00F0BC8100202863E8622D
:10C74000002E88BFDFF8F4E01BD9DEF8002005EBEF
:10C750004001B1F97611B2F9D8308B4203DCB2F95D
:10C76000DA208A420ADA420905EB820100F01F0C46
:10C770000122CB6A02FA0CF21A43CA62401CB04290
:10C78000E3D30020A8626862002F88BFDFF8ACE026
:10C790001BD9DEF8002005EB4001B1F97612B2F9A1
:10C7A000D8308B4203DCB2F9DA208A420ADA420935
:10C7B00005EB820100F01F0C01224B6A02FA0CF219
:10C7C0001A434A62401CB842E3D300202864E8635D
:10C7D000002E88BFDFF864E01BD9DEF8002005EBEF
:10C7E0004001B1F9B611B2F9DC308B4203DCB2F989
:10C7F000DE208A420ADA420905EB820100F01F0CB2
:10C800000122CB6B02FA0CF21A43CA63401CB042FD
:10C81000E3D30020A8636863002F88BFDFF81CE023
:10C8200020D9DEF8002005EB4001B1F9B612B2F9CB
:10C83000DC308B4208DCB2F9DE2003E04006011058
:10C84000480601108A420ADA420905EB820100F02B
:10C850001F0C01224B6B02FA0CF21A434A63401C74
:10C86000B842DED300202865E864A8646864002E1E
:10C8700088BFDFF844E71CD9DEF8003005EB400143
:10C88000B1F9F611B3F9E0208A4203DCB3F9E220F2
:10C890008A420BDA410905EB810C00F01F030121EC
:10C8A000DCF84C2099401143CCF84C10401CB042AD
:10C8B000E2D30020002F88BFDFF8FCE61BD9DEF8AA
:10C8C000002005EB4001B1F9F612B2F9E0308B42DD
:10C8D00003DCB2F9E2208A420ADA420905EB82015E
:10C8E00000F01F0C01224B6C02FA0CF21A434A644E
:10C8F000401CB842E3D3696AE86AB14040EA010EDD
:10C90000C4F838E0A96A286BB1400843E063696A5B
:10C91000202E34BF21FA09F101FA08F141EA0000A2
:10C92000E0630590696BE86B01FA06F140EA0102E9
:10C930002264A96B286C01FA06F140EA01006064E8
:10C94000696B34BF21FA09F101FA08F141EA0001EB
:10C9500061646B6CE86C03FA06F340EA0300A064C0
:10C960000490AB6C286D03FA06F340EA0300E06420
:10C970006B6C34BF23FA09F303FA08F343EA0000AF
:10C98000E0640290059832EA0E0521EA000C4EEAB6
:10C9900005022564069240EA0C00C4F844C006EB88
:10C9A0000701039008BFBCF1000F42D000231A46D4
:10C9B0001846002988BF01273BD94FEA501804EBDD
:10C9C000880800F01F09D8F8408007FA09F918EA2A
:10C9D000090F03D0864294BF521C5B1C401C81424D
:10C9E000EBD8012B0FD105EA0A0040EA0E00A06344
:10C9F00005980CEA0B031843E06325EA0A0020645B
:10CA00002CEA0B006064012A13D1226C0098A36BFE
:10CA100010401843A063606C019BD4F83CC00340F5
:10CA200043EA0C03E363009B9A432264019A904318
:10CA30006064069A049830EA0202A264069840EA0A
:10CA4000020CDDE9020320EA0300E064039B43EAF1
:10CA5000000508BF002821D000231A4618460029E7
:10CA600088BF012717D94FEA501804EB880800F057
:10CA70001F09D8F8488007FA09F918EA090F03D006
:10CA8000864294BF521C5B1C401C8142EBD8002B99
:10CA900018BF002A02D10020A064E064079810F0BB
:10CAA000010F06D0206B20EA0C002063606BA843C6
:10CAB0006063206B0099084203D1626B01990A42BE
:10CAC00003D0216941F01001216110EA0A0F04BF6F
:10CAD000606B10EA0B0F03D0206940F0200020614A
:10CAE000A06B0099084203D1E26B01990A4203D07E
:10CAF000216941F04001216110EA0A0F04BFE06B97
:10CB000010EA0B0F03D0206940F080002061206CF8
:10CB10000099084203D1626C01990A4203D021694D
:10CB200041F48071216110EA0A0F04BF606C10EAC1
:10CB30000B0F03D0206940F400702061A06C002826
:10CB400004BFE06C002803D0206940F480602061BD
:10CB500009B00120BDE8F08F2DE9F04FB9B01646BD
:10CB60000D460446F4F712FFF4F74CF901004FF0BC
:10CB700011001DBF029001200390012108BFCDE9E3
:10CB80000210CDE93454F5F778F90022002D88BF62
:10CB900004A904D9835C8B54521C9542FAD8F5F74A
:10CBA0006EF90021002C88BF04AA07D9435C02EB70
:10CBB000010C491C8CF820308C42F7D8F5F7A2F80C
:10CBC0003890FE48007810F0200F5FD0F4F71AF983
:10CBD000FB4AFC4900280CBFCDE90012CDE9002139
:10CBE00006F1F600369040300025EA460DF1D809EE
:10CBF0000DF1D00B379002A85BF8257050F8250096
:10CC0000F5F7FFFB0024002F84BF04A800EB4518B4
:10CC10001AD918F90400202828BF00200DD25AF88C
:10CC2000251000EBD072521051F82210C007C00E30
:10CC300021FA00F080B2F5F7EAFB59F8251021F847
:10CC40001400641CBC42E4D36D1C022DD3D3DE4817
:10CC500004781D2C1AD100210A4614AD5BF822304D
:10CC60000020002B88BF59F822C007D93CF810706B
:10CC700025F81170401C491C8342F7D8521C022A27
:10CC8000ECD31D2C04BF2846FDF7BEFCCB4D287805
:10CC900010F00C0F00F09982F4F7B4F8CB49CC4AAD
:10CCA00000280CBFCDE91421CDE91412C948F4F7CE
:10CCB000F7FE0120F4F70BFB2D900120F4F755FB54
:10CCC0002C900120F4F7DCFD25900220F4F7D8FD2C
:10CCD00023900298F4F772FB24900398F4F76EFB0C
:10CCE00017900120F4F7EDFB2A901120F4F7E9FBEF
:10CCF00029900120F4F711FC28901120F4F70DFC85
:10CD0000279020A800901EAB1CAA1AA90298F4F73D
:10CD10000AFD21A800901FAB1DAA1BA90398F4F7D8
:10CD200002FD0298F4F77BFD22900298F4F777FD5C
:10CD3000A14C01902068B0F8E4100120F4F7D6FA75
:10CD400000210120F4F787FD00210220F4F783FD84
:10CD5000206890F8E6100298F4F73FFB206890F8FE
:10CD6000E6100398F4F739FB00210120F4F7BFFB2C
:10CD700000211120F4F7BBFB00210120F4F7E3FBB5
:10CD800000211120F4F7DFFB2068B0F8E8100298CA
:10CD9000F4F7F6FC2068B0F8E8100398F4F7F0FC1C
:10CDA00000210120F4F77EFD2B908448007810F0DC
:10CDB000040F00F0FE8025462868B0F8EC100091C2
:10CDC00090F8EB3090F8EA200B210298F4F77FFC02
:10CDD0002868B0F8EC10009190F8EB3090F8EA2059
:10CDE0000B210398F4F773FC00210120F4F75AFD9E
:10CDF0002EA800F0DBFD3299002234AC002054F85C
:10CE000022C0BCF1000F88BF06EB022308D931F81D
:10CE1000027B03EB4008401CA8F876718445F6D8E5
:10CE2000521C022AEAD30298F3F7C4FD1890039823
:10CE3000F3F7C0FD16900298F4F736FB269003989E
:10CE4000F4F732FB5C4D19902868B0F8EE100091B1
:10CE500090F8EB3090F8EA200B210298F4F737FCB9
:10CE60002868B0F8EE10009190F8EB3090F8EA20C6
:10CE70000B210398F4F72BFC002500210120F4F787
:10CE800011FD00210298F3F780FD00210398F3F7CC
:10CE90007CFD0DF10808012158F82500F3F775FD18
:10CEA00034A8002450F8257014A8002F50F825A0AD
:10CEB00030D904A800EB451906EB0528002119F824
:10CEC00004B00846F4F7FFFC012000FA0BF102A8B9
:10CED0008B4650F82500F4F7DAFA6FEA0B010920C7
:10CEE000F4F7F1FC0DF1B80BF4F759FFFCF7BCFEB9
:10CEF000012804D05846F5F710F900286CD0F4F753
:10CF000045FDBAF8000008EB4401641CA1F8B60125
:10CF1000BC42D3D300210846F4F7D5FC6D1C022D8A
:10CF2000ABD318990298F3F730FD16990398F3F7ED
:10CF30002CFD26990298F4F7AAFA19990398F4F7A8
:10CF4000A6FA1D4C2068B0F8F010009190F8EB3074
:10CF500090F8EA200B210298F4F7B9FB2068B0F8AA
:10CF6000F010009190F8EB3090F8EA200B21039834
:10CF7000F4F7ADFB01210846F4F794FC2EA800F06D
:10CF800015FD3299002234AC002054F822C0BCF1C7
:10CF9000000F88BF06EB022308D931F8025B03EBD0
:10CFA0004007401CA7F8F6518445F6D8521C022AC7
:10CFB000EAD30248007810E040060110480601104C
:10CFC000C0480030404800305A050110C00A003007
:10CFD0004008003001000E0046E010F0080F7CD041
:10CFE000F74D2868B0F8F210009190F8EB3090F807
:10CFF000EA200B210298F4F76AFB2868B0F8F210D7
:10D00000009190F8EB3090F8EA200B210398F4F7A8
:10D010005EFB00210B4634AF002057F821C0BCF165
:10D02000000F88BF06EB012206D902EB4004401C2A
:10D03000A4F836328445F8D8491C0229ECD3286874
:10D04000002490F82401B4EB400F7ADA286890F8B5
:10D050002401A042D4BF012100210120F4F722FCC9
:10D060002EAFF4F79CFE02E0F8F7C4FB3EE7FCF7B6
:10D07000FBFD012803D03846F5F74FF870B3F4F7FD
:10D0800085FC32994FF000090DF1D00E00225EF8B8
:10D0900029701046002F05D931F91030401C1A4470
:10D0A0008742F9D8B2FBF7F2781E18BF06EB092ABF
:10D0B00039D031F9103001EB400C3CF9028CB3EB64
:10D0C000080348BF5B4231F91080B8EB020831F920
:10D0D000108048BFA2EB080801E032E018E058BF1A
:10D0E000A8EB02083CF902BC3CF902CCBBEB020BFA
:10D0F0004CBFA2EB0C0CACEB020CE0450AEB400C75
:10D1000009DDBCF936824345C8BFACF8363208E0C9
:10D11000F8F770FBABE7BCF934829845B8BFACF8C0
:10D120003432401EC5D109F1010901EB4701B9F1C3
:10D13000020FABD32868641C90F82401B4EB400FB5
:10D1400084DB01202D99F4F7D1F801202C99F4F714
:10D1500015F901202599F4F77EFB02202399F4F7B5
:10D160007AFB24990298F4F738F917990398F4F7A1
:10D1700034F901202A99F4F7BAF911202999F4F722
:10D18000B6F901202899F4F7DEF911202799F4F770
:10D19000DAF9209800901E9B1C9A1A990298F4F7CD
:10D1A00096FA219800901F9B1D9A1B990398F4F7FB
:10D1B0008EFA22990298F4F7E3FA01990398F4F7AA
:10D1C000DFFA01202B99F4F76DFB3898F4F768FC2F
:10D1D00039B0BDE8F08F2DE9F04F7A4DADF24C4DEE
:10D1E000FF224FF4876168466C6807F021FE0094C7
:10D1F000288810F4804F1CBF2046FEF762FF6A4665
:10D20000009890F8203090F821C050300CFB03F1CA
:10D2100000EB41000021BCF1000F08D902EB4107EF
:10D2200030F8026B491CA7F8F6608C45F6D800214F
:10D23000002B08D902EB410730F8026B491CA7F814
:10D2400036618B42F6D81668002196F82260002ECF
:10D250000BD902EB410730F8026BA7F8766316682A
:10D26000491C96F822608E42F3D81668002196F881
:10D270002360002E0BD902EB410730F8026BA7F8B0
:10D2800096631668491C96F823608E42F3D80021F5
:10D29000BCF1000F08D902EB410730F8026B491CC2
:10D2A000A7F870608C45F6D80021002B08D902EB56
:10D2B000410730F8026B491CA7F8B0608B42F6D8E2
:10D2C00030F8021BA2F8F21030F8021BA2F8F4109A
:10D2D00030F8021BA2F8F01000260021BCF1000F6C
:10D2E00088BF02EB861708D907EB410930F8028B9B
:10D2F000491CA9F876818C45F6D80021002B88BFFF
:10D3000002EB861708D907EB410930F8028B491C5C
:10D31000A9F876828B42F6D8761C042EDDD300263F
:10D320001768002197F82270002F88BF02EB46177C
:10D330000CD907EB410930F8028BA9F8B683D2F873
:10D340000080491C98F822808845F2D8176800218F
:10D3500097F82370002F88BF02EB46170CD907EB14
:10D36000410930F8028BA9F8F683D2F80080491CF5
:10D3700098F823808845F2D8761C022ED0D36146D7
:10D380001846FEF7CBFF0F480126056815F4004F3D
:10D390007ED180460A486F460026006890F8B400A7
:10D3A00000F00F0901F033F801280DD00F21484695
:10D3B000F8F7DDFA012816D0002001F025F8B7E0D3
:10D3C000400601104806011000210846F4F78BFBC7
:10D3D000F3F7FFFC50B1FE48D0F8B01241F48031B1
:10D3E000C0F8B01202E0012001F00EF8F94890F800
:10D3F0000090F94890F800A0BAF1000F18BFB9F1F9
:10D40000000F7CD0009E002086F8209086F821A096
:10D4100086F8220086F82300F5F732F8F4F772FC5C
:10D420008346002015F0030F18BF4FF4817015F0EC
:10D43000200F1CBF40F20121084315F0100F1EBF42
:10D4400098F8001011F0210F40F4846060B10BEAED
:10D450000000F4F725FBFF210F20F9F731F8F4F76E
:10D4600095FA5846F4F71CFB15F0100F09D0DB496C
:10D470003A46087886F82200497886F8231000F0AA
:10D48000DBFC15F02C0F06D03A465146484600E02A
:10D490004EE0FFF761FB15F0030F46D00098CDF882
:10D4A0003C7400F15006CDF83804F4F7E8FC8346EC
:10D4B000F4F76CFA0020F4F7A4FF0027BAF1000F8C
:10D4C00024D900254FEA871817E01BF9050020280A
:10D4D00012D200EBD071491008EB810101F14051EB
:10D4E00001F58041C0070968C00E21FA00F080B242
:10D4F000F4F78DFF26F8020B6D1C4D4500E015E09A
:10D5000038BF202DE1D37F1C5745DAD3B4480078CB
:10D510001D2804D1DDF838045030FCF771FF514666
:10D520004846DDF83C24FEF7F9FE0126F4F7ABFB94
:10D5300094F82000CDF8400494F82100CDF844047C
:10D54000002E1FBFDDF840040028DDF84404002849
:10D5500004BF0DF24C4DBDE8F08FA2480068CDF835
:10D56000480410F0020F00F01081009DDDF84474B3
:10D57000DDF8402428696E4620F00F00286147F648
:10D58000FF706FEA0009CDF83804002005F150085B
:10D5900004900390029082460190002F51D90AFB1B
:10D5A00002F0012138F9103000209B46DC46CDF80E
:10D5B0003C04012A1AD90AFB021038F91000604510
:10D5C000C8BF84469842B8BF0346B0EB0B0E48BFB5
:10D5D000ABEB000E0FFA8EFBDDF83CE4F345C8BF61
:10D5E000CDF83CB48346491C9142E4D3CC45C8BF36
:10D5F000E146DDF838048342B8BFCDF83834BCEBDF
:10D60000030048BFA3EB0C0001B277480068B0F9F3
:10D61000C0308B4205DBB0F9C210DDF83C04884213
:10D620000BDD4FEA5A1006EB80000AF01F0C0121B7
:10D63000C36801FA0CF11943C1600AF1010ABA4545
:10D64000ADD34FF0000A002A4FD938F91A00002153
:10D6500083460123DC46CDF83C14012F1AD903FB85
:10D6600002A138F911106145C8BF8C468142B8BF8C
:10D670000846B1EB0B0E48BFABEB010E0FFA8EFB69
:10D68000DDF83CE4F345C8BFCDF83CB48B465B1CE9
:10D69000BB42E4D3CC45C8BFE146DDF8381488422C
:10D6A000B8BFCDF83804BCEB000148BFA0EB0C01BB
:10D6B00009B24D480068B0F9BC308B4205DBB0F9C7
:10D6C000BE10DDF83C0488420BDD4FEA5A1006EB31
:10D6D00080000AF01F0C0121436801FA0CF1194384
:10D6E00041600AF1010A9245AFD3F068002804BFF7
:10D6F0003069002803D0286940F00800286170686C
:10D70000002804BFB068002803D0286940F0040056
:10D7100028617168F068B9400843A862B16830694F
:10D72000B9400143E9627068202F39BFC7F1200278
:10D73000D040A7F1200290400843E862DDF83804A9
:10D74000A884A5F82690B6F9F010B9EB010048BFFF
:10D75000A1EB090024490968B1F9B820904203DD22
:10D76000286940F002002861B6F9F020DDF838049D
:10D77000101A44BFDDF83804801AB1F9BA10884293
:10D7800003DD286940F001002861DDF84804154DEB
:10D7900010F0050F06D06A46DDF84414DDF84004A9
:10D7A000FEF7FDFED5F8009019F0080F7DD0009A25
:10D7B000DDF840A4DDF8443411694FF0000B21F48A
:10D7C000C05111616846CDF860B059460EE00000C6
:10D7D00000500040D5040110D6040110DD040110F2
:10D7E000550501104806011040060110CDF85CB047
:10D7F000002B84BFDFF844E401261AD9DEF800705C
:10D8000000EB410CBCF936C2B7F9267167450DDA59
:10D810004FEA511C00EB8C0C01F01F08DCF85C7027
:10D8200006FA08F847EA0807CCF85C70491C9942E8
:10D83000E4D3C0F858B00021C0F854B0BAF1000FDA
:10D8400084BFFE4E01271AD9D6F8008000EB410CA8
:10D85000BCF936C3B8F92681E0450DDA4FEA511814
:10D8600000EB880C01F01F0BDCF8548007FA0BFB6F
:10D8700048EA0B08CCF85480491C5145E4D3916B1D
:10D88000D0F85CC041EA0C01D0F854C00CFA03FC9B
:10D8900041EA0C019163D16BD0F860C041EA0C0100
:10D8A000D0F858C00CFA03FC00E022E041EA0C0C6E
:10D8B000C2F83CC0416D202B39BFC3F12003D940D1
:10D8C000203B994041EA0C01D163416D002904BF1E
:10D8D000816D002903D0116941F400611161C16DAE
:10D8E000002904BF006E002803D0106940F4805066
:10D8F000106119F0100F18BF19F0050F06D094F839
:10D90000231094F822006A4600F079F9287810F084
:10D91000400F0FD16069401C60612069002814BF6E
:10D92000E069A06900F1010014BFE061A0616846F0
:10D93000FEF72BFC0020E060A36821460246A446C7
:10D94000B3F5056F88BF4FF405630020B0EB930F6C
:10D9500006D25CF82070401C3A44B0EB930FF8D329
:10D960005042C860287810F0800F05D14FF42C3059
:10D970004FF40562F5F7E7F841208DF83804207C74
:10D980008DF83904607C8DF83A04A07C8DF83B0456
:10D99000E07C8DF83C04002305220DF5876107200B
:10D9A00000F0A4FC0DF24C4DBDE8F08F70B50546BB
:10D9B0000024F4F7F4F9FCF757F9012804D02846BD
:10D9C000F4F7ABFB20B10124F3F7E0FF204670BD74
:10D9D000F7F710FFEFE72DE9F74F84B04FF000089D
:10D9E000C2F82080C2F81C80059B944E0127414656
:10D9F000002B1ED902EB4103B3F97030002BB8BFE6
:10DA00005B421BB2D6F800C0BCF9CCC09C450CDD13
:10DA10004B0902EB830301F01F04D3F81CC007FA83
:10DA200004F44CEA040CC3F81CC0059B491C994241
:10DA3000E0D30021012B1CBF059BA3F1010940D0BD
:10DA400002EB4103B3F97240B3F970C0B4EB0C03BD
:10DA500048BFACEB04031BB23568B5F9C6509D4214
:10DA60002CDAB2F9F230BCEB030548BFA3EB0C058E
:10DA70002DB2B4EB030C48BFA3EB040C0FFA8CF3EC
:10DA80009D420DDB4B0902EB830301F01F04D3F829
:10DA90001CC007FA04F44CEA040CC3F81CC00DE0E7
:10DAA0004B1C4FEA531C02EB8C0C03F01F03DCF8F9
:10DAB0001C4007FA03F32343CCF81C30491C4945AA
:10DAC000BED3316891F8CA30002B7DD091F8CB10CD
:10DAD00014688B4288BF19460023DDF814C0BCF1DE
:10DAE000000F84BF491C00916ED94FF0010EDDF884
:10DAF00000C04FF000090121CA46BCF1010F52D904
:10DB0000DFF838C103FB0005DCF800C0CDF80CC01D
:10DB1000BCF9CEC002950EFB0005019503FB001574
:10DB200004EB4505B5F95080B8F1000FB4BFC8F15A
:10DB300000054546AC4536DB0EFB001504EB4505FC
:10DB4000B5F95070002FB4BF7D423D46AC452ADB8D
:10DB5000029D6D1A04EB4505B5F94E60002EB4BF69
:10DB600075423546AC451EDB019D6D1A04EB45053B
:10DB7000B5F94E50002DB4BFC5F1000BAB46E345DF
:10DB800011DCA7EB0808039FB7F9C8704745B8BF79
:10DB900009F10109AD1BBD42C8BF0AF1010A491CC8
:10DBA000009DA942BAD3BAEB090148BFA9EB0A010B
:10DBB000DFF888C0DCF800C09CF8CAC061450FDB04
:10DBC000590902EB810100E015E003F01F064FF058
:10DBD000010CCD690CFA06FC45EA0C0CC1F81CC01E
:10DBE00005995B1C8B4206D2002B18BFA3F1010ED6
:10DBF0007FF47DAF79E707B00120BDE8F08F2DE914
:10DC0000F04F83B04FF0000C1368C2F864C0C2F844
:10DC100068C0C2F86CC0DFF828C04FF0010BDCF818
:10DC200000E0DFF818C01EF0010FDCF800C02ED0B5
:10DC30001C69002524F480342F4603E040060110BF
:10DC4000480601101C61CDE900015DF827A0002401
:10DC5000BAF1000F88BF02EB471915D909EB44064A
:10DC6000BCF9D480B6F97663B04503DCBCF9D68044
:10DC7000B04505DA566E0BFA05F846EA0806566610
:10DC8000641C6D1CA245E9D87F1C022FDDD31EF059
:10DC9000040F71D01C69002524F4C0241C612F4698
:10DCA000EE46CDE900015EF827A00024BAF1000F8E
:10DCB00088BF02EB871915D909EB4406BCF9D88057
:10DCC000B6F9B663B04503DCBCF9DA80B04505DAD5
:10DCD000966E0BFA05F846EA08069666641C6D1CFB
:10DCE000A245E9D87F1C022FDDD300252F46CDE9C0
:10DCF00000015EF827A00024BAF1000F88BF02EBF4
:10DD0000871915D909EB4406BCF9DC80B6F9D6634E
:10DD1000B04503DCBCF9DE80B04505DAD66E0BFAFF
:10DD200005F846EA0806D666641C6D1CA245E9D8CB
:10DD30007F1C022FDDD34418D2E91A5030EA050CBB
:10DD40004CEA0506C2F86CC013D000210846002C2E
:10DD50000FD90BFA00F71CEA070F18BF491C401C2B
:10DD6000A042F6D3012904D145EA0C0090660020B8
:10DD7000D066506EB043506693F8200093F821109F
:10DD80000844516ED9B1196941F480311961D2F852
:10DD900064C0196B0CFA00FC41EA0C011963516E66
:10DDA000202827BFA0F1200C01FA0CF1C0F1200CB3
:10DDB00021FA0CF1D3F834C041EA0C015963916E99
:10DDC000D9B1196941F400311961D2F868C0996B71
:10DDD0000CFA00FC41EA0C019963916E202827BFE0
:10DDE000A0F1200C01FA0CF1C0F1200C21FA0CF189
:10DDF000D3F83CC041EA0C01D963D16EC1B11969B5
:10DE000041F480211961D2F86CC0196C0CFA00FC45
:10DE100041EA0C011964D16E202827BF203801FA8D
:10DE200000F0C0F1200021FA00F0596C084358645A
:10DE300003B00120BDE8F08F2DE9F04FA7B01746E1
:10DE40000D460446F3F7A2FD02221C9212221D92F7
:10DE5000CDE90845F3F756FF1990FE480DF1380A51
:10DE60004FF0010B007810F0210F5BD0FA480A90B8
:10DE7000FA480B901C98F3F717FB0E901D98F3F7D8
:10DE800013FB00250F9008A850F825901CA850F807
:10DE90002500F4F7B6FA0024264607EB451817E0EC
:10DEA0005AF825000BFA04F1084210D00AA86108BC
:10DEB00050F8250050F82100E107C90EC84080B293
:10DEC000F4F7A5FA08EB4601761CA1F87603641C6A
:10DED0004E4538BF202CE3D36D1C022DD3D3E04830
:10DEE00005781D2D1ED100210A466C4608AE002083
:10DEF00056F822C0BCF1000F88BF07EB421309D9C6
:10DF000003EB4008401CB8F8768324F81180491CC4
:10DF10008445F5D8521C022AE9D31D2D04BF2046A2
:10DF2000FCF791FCCB48007810F0040F00F08C81D6
:10DF3000CC480C90CC480D900220F3F7C8F92690FD
:10DF40000220F3F712FA25900120F3F799FC2090B4
:10DF50000220F3F795FC1B901C98F3F72FFA16900C
:10DF60001D98F3F72BFA17900220F3F7AAFA2490E2
:10DF70001220F3F7A6FA21900220F3F7CEFA2290AE
:10DF80001220F3F7CAFA1F9006A8009004AB02AA69
:10DF90000AA91C98F3F7C7FB07A8009005AB03AAD2
:10DFA0000BA91D98F3F7BFFB1C98F3F738FC1E90E4
:10DFB0001D98F3F734FCAD4C01902068B0F8E410E4
:10DFC0000220F3F793F900210120F3F744FC00212C
:10DFD0000220F3F740FC206890F8E6101C98F3F755
:10DFE000FCF9206890F8E6101D98F3F7F6F9002187
:10DFF0000220F3F77CFA00211220F3F778FA0021CF
:10E000000220F3F7A0FA00211220F3F79CFA20680F
:10E01000B0F8E8101C98F3F7B3FB2068B0F8E810EC
:10E020001D98F3F7ADFB00210220F3F73BFC239092
:10E030002068B0F8EC10009190F8EB3090F8EA20EE
:10E040000B211C98F3F743FB2068B0F8EC1000910B
:10E0500090F8EB3090F8EA200B211D98F3F737FB8E
:10E0600000210220F3F71EFC10A8FFF79FFC159972
:10E07000002208AD002055F822C0BCF1000F88BF77
:10E0800007EB821308D931F8026B03EB4008401C00
:10E09000A8F8B6638445F6D8521C022AEAD31C9825
:10E0A000F2F788FC1A901D98F2F784FC18901C98DF
:10E0B000F3F7FAF90E901D98F3F7F6F90F90206830
:10E0C000B0F8EE10009190F8EB3090F8EA200B21B8
:10E0D0001C98F3F7FCFA2068B0F8EE10009190F865
:10E0E000EB3090F8EA200B211D98F3F7F0FA0024AA
:10E0F00000210220F3F7D6FB00211C98F2F745FC23
:10E1000000211D98F2F741FC0DF17008012158F82B
:10E110002400F2F73AFC08A8002550F824900CA837
:10E120002E4650F824A007EB84182EE00EA850F8D5
:10E130002410012000FA05FB11EA0B0F24D0002166
:10E140000846F3F7C0FB1CA8594650F82400F3F723
:10E150009EF96FEA0B010920F3F7B5FB0DF1400BB7
:10E16000F3F71DFEFBF780FD012804D05846F3F7B6
:10E17000D4FF00287DD0F3F709FCBAF8000008EBC3
:10E180004601761CA1F8D6036D1C4E4538BF202DE4
:10E19000CCD300210846F3F796FB641C022CA7D3CE
:10E1A0001A991C98F2F7F1FB18991D98F2F7EDFBFC
:10E1B0000E991C98F3F76BF90F991D98F3F767F90F
:10E1C00002202699F3F792F802202599F3F7D6F862
:10E1D00001202099F3F73FFB02201B99F3F73BFB4B
:10E1E00016991C98F3F7F9F817991D98F3F7F5F8B5
:10E1F00002202499F3F77BF912202199F3F777F99C
:10E2000002202299F3F79FF912201F99F3F79BF947
:10E2100006980090049B029A0A991C98F3F757FA03
:10E2200007980090059B039A0B991D98F3F74FFAF6
:10E230001E991C98F3F7A4FA01991D98F3F7A0FA18
:10E2400002202399F3F72EFB1998F3F729FC27B046
:10E25000BDE8F08F4806011040490030C049003049
:10E260005F050110C00E0030C010003040060110E4
:10E27000FFE7F7F7BFFA75E770474FF0FF307047D9
:10E280005D48406870475C494860704710B582B08F
:10E2900007280BD14FEA111C012404FA0CFC564C40
:10E2A00064681CEA040F04BF02B010BD9B0100F0BB
:10E2B0000F0043EA800040F001008DF800008DF867
:10E2C00001108DF80220100A8DF80300100C8DF853
:10E2D0000400100E8DF8050000208DF806008DF862
:10E2E0000700684606F0B7FE02B010BD10B582B058
:10E2F00007280DD191F800C001244FEA1C1C04FA34
:10E300000CFC3D4C64681CEA040F04BF02B010BD55
:10E310009B0100F00F0043EA800040F001008DF8FF
:10E320000000072A88BF072200206B46002A09D96F
:10E3300011F800C01C18401C84F801C09042F7D3AB
:10E34000072805D200211A18401C51700728FAD35B
:10E35000184606F080FE02B010BD10B59B0100F01B
:10E360000F0082B043EA800040F002008DF8000008
:10E37000072A88BF072200206B46002A09D911F816
:10E3800000C01C18401C84F801C09042F7D3072835
:10E3900005D200211A18401C51700728FAD31846DC
:10E3A00006F059FE02B010BD70B5134E40EA0125CB
:10E3B00002283488224618BF052803D1002918BF37
:10E3C000022900D12C46A24209D051B17088002305
:10E3D00044EA004290210720FFF758FF34807580FF
:10E3E00070BDF4F7A4FF44EA004200239021072007
:10E3F000FFF74CFFF2E7000050060110FD490870DE
:10E400007047FC4800787047FA4948707047F948EF
:10E41000407870472DE9F04FF748F64DADF6740D92
:10E4200000686978836D0229C3F303201AD06A68F3
:10E4300012F4007F1EBFC3F303310F29084612F008
:10E44000800F1EBFC3F303110F29084602F0070116
:10E45000F7F78DFA012814BF00200220687040F001
:10E460006F830DE000210846F3F73DFBF2F7B1FCA6
:10E4700030B1E248D0F8B01241F48031C0F8B012A7
:10E48000F3F740FCCDF82C08287910F0100F18BFD6
:10E49000F3F7D5FF287910F0080F03D1FF210F20E3
:10E4A000F8F70EF8D6484FF000080078CDF84C0881
:10E4B000D4480078CDF85008D3480478D348007881
:10E4C000CDF84808D24890F80090DDF850080028B0
:10E4D0001CBFDDF84C08002816D006F080FD06F0C1
:10E4E00083FD0020F6F75DF90020F6F7ABF9002078
:10E4F000F6F769FABF48007910F0100F0CD0012030
:10E50000F6F7CEFA01200BE0DDF84808002818BF26
:10E51000002CE2D100F014BB0020F6F7C1FA002075
:10E52000F6F7BEFAF2F755FC10F0010F04BF012018
:10E53000F2F7BEFEF3F7FAFB1E20FBF7B7FE002151
:10E540000846FBF731FECDF85C0801210020FBF7FF
:10E550002BFEDDF85028DDF84C188346002001FB27
:10E5600002FABAF1000F84BF47F6FF72D14308D90F
:10E57000DDF85C3823F810102BF81020401C824581
:10E58000F6D81E20FCF726F800210120FBF70CFE30
:10E59000064601210846FBF707FE0546DDF8481848
:10E5A000002067181CBF47F6FF71CA4306D026F843
:10E5B000102025F81010401C8742F8D81E20FCF7C8
:10E5C0002CF900210220FBF7EFFDCDF858080121BE
:10E5D0000220FBF7E9FDCDF85408002019EB0809EB
:10E5E0001CBF47F6FF73D9430AD0DDF8582822F83C
:10E5F0001010DDF8542822F81030401C8145F4D862
:10E600007C484FF000084088002840F2A181DDF8E6
:10E610004818781C491ECDF86C18DDF848184008D9
:10E620002144491ECDF8601809F101014908CDF8CF
:10E630006818CDF86408FBF717FB012800F0888103
:10E640000DF50360F3F769FD002800F07A81DDF82D
:10E650003408F5F7EDFADDF83808002853D006F055
:10E66000FBFB04466348007910F0100F0AD02046E7
:10E67000DDF8381806F0F4FC0190A04208BFDDF880
:10E68000384810E0002000230090019002901A46C4
:10E690001946DDF8380806F0E8FC01905548007985
:10E6A00010F0200F0BD1F5F75FFBDDF8502800923A
:10E6B00001462046DDF84C38019A06F0DBFC4D4857
:10E6C000808810F4804F1EBF01980028F5F788FB62
:10E6D000002C1CBF0020BAF1000F14D9DDF85C2813
:10E6E00034F9101032F910208A42BCBFDDF85C28E2
:10E6F00022F810103BF910208A42C8BF2BF81010E6
:10E70000401C8245EAD8DDF82C0810F0010F1CBF30
:10E71000DDF8400800286CD006F094FB044635482C
:10E72000007910F0400F07D000231A461946DDF893
:10E73000400806F0A4FC0DE0F5F7DFFA0222009293
:10E7400001462046DDF86438DDF8402806F092FCEA
:10E75000DDF840082749898811F4005F1CBF0028B4
:10E76000F5F7D5FA002C44D02248426812F4806FA5
:10E7700033D0DDF848180020012911D004EB400106
:10E7800034F910C0B1F90230B3EB0C0148BFACEB67
:10E79000030124F81010DDF86C18401C8842EDD3FA
:10E7A0004FF0000E24F810E0DDF86018401C88429D
:10E7B00011D204EB400134F910C0B1F90230B3EBCF
:10E7C0000C0148BFACEB030124F81010DDF8601811
:10E7D000401C8142EDD824F810E00020002F22D9FF
:10E7E00034F9101036F910308B42B8BF26F81010EB
:10E7F00010E04EE0580601104006011000500040A5
:10E80000D5040110D6040110DA040110DB04011054
:10E81000DD04011035F910308B42C8BF25F8101007
:10E82000401C8742DCD812F4806F32D0F14A08F1E4
:10E830000100A2FB00318908494201EB8101C1427C
:10E8400027D1A2FB08108008A2FB00210909494238
:10E8500001EB810100EB810000EB800101EBC001C5
:10E8600003A800EBC1010020002F84BF47F6FF7C06
:10E870006FEA0C020DD936F8103035F810401B1B2A
:10E8800021F8103026F8102025F810C0401C8742CF
:10E89000F1D8DDF82C0810F0200F1CBFDDF844087B
:10E8A000002849D006F0F0FB0446D348808810F4D5
:10E8B000807F13D0F5F7FEF9022200920146204630
:10E8C000DDF86838DDF8442806F0D4FBDDF84408AC
:10E8D000C949898811F4805F0FD109E00021DDF872
:10E8E000440806F0A0FAB8F1040F38BF0024EFE79F
:10E8F00018B1F5F7EAF9F5F7BAF9002C1CBF0020BA
:10E90000B9F1000F18D9DDF8582834F9101032F990
:10E9100010208A42BCBFDDF8582822F81010DDF81C
:10E92000542832F910208A42C4BFDDF8542822F856
:10E930001010401C8145E6D8F3F737FC08F10108B8
:10E9400001E0F6F757FFAC4840888045FFF473AE0E
:10E95000F3F71CF806F048FB06F04BFBA64C60886A
:10E96000804578D3DDF82C0810F0020F2AD0002261
:10E970004FF6FF731046BAF1000F10D9DDF85C189E
:10E980003BF910C031F91010A1EB0C019142C8BF46
:10E990000A469942B8BF0B46401C8245EED8422039
:10E9A0008DF80000100A8DF801008DF80220180A79
:10E9B0008DF803008DF804300023052269460720F6
:10E9C000FFF794FCDDF82C0810F0010F7DD0A08833
:10E9D00010F4806F51D08748A0FB08108308142BD7
:10E9E00088BF14234FF0000844464146002F84BFDF
:10E9F000981E009055D94FF0000CDFF800A247F6A2
:10EA0000FF7B6246002B12D902EB820000EBC20EA4
:10EA100003A800EBCE0030F9110084445045C8BF74
:10EA200082465845B8BF8346521C9A42ECD3002B0D
:10EA300004BF002026F811000ED09CFBF3F026F84E
:10EA40001100022B08D9ACEB0A00A0EB0B020098D6
:10EA500092FBF0F001E06AE0002025F8110036F9A1
:10EA60001100A042C8BF044635F911004045C8BF97
:10EA70008046491C8F42BED813E000244FF6FF7831
:10EA80002046002F0DD936F9101035F91020891ABB
:10EA9000A142C8BF0C464145B8BF8846401C8742CA
:10EAA000F1D843208DF80000200A8DF801008DF880
:10EAB00002404FEA18208DF803008DF804800023EF
:10EAC000052269460720FFF711FCDDF82C0810F03D
:10EAD000200F2CD000224FF6FF731046B9F1000F23
:10EAE00012D9DDF8581831F910C0DDF8541831F991
:10EAF0001010ACEB01019142C8BF0A469942B8BF61
:10EB00000B46401C8145ECD844208DF80000100ACB
:10EB10008DF801008DF80220180A8DF803008DF899
:10EB200004300023052269460720FFF7DFFBFF20A2
:10EB3000FBF7BCFBFF20FBF74DFDFF20FBF76DFE55
:10EB4000F3F7A1F80DF6740DBDE8F08F10B5ADF533
:10EB5000056D4FF0FF30FDF74BF8274C002060703B
:10EB6000F3F785F9FF224FF40561684606F060F976
:10EB70006846FDF7BEFA6846FDF749FAFBF774F8F8
:10EB8000012803D1F6F7DEFD03281BD1207810F011
:10EB9000010F07D0FEF71FFB207820F00100207046
:10EBA000FBF70CF8207810F0020F07D0FFF732FCCB
:10EBB000207820F002002070FBF700F8F6F7C2FD85
:10EBC000032808D00020FDF722FA0120F3F74FF9BF
:10EBD0000DF5056D10BDF6F70DFECFE7064948604F
:10EBE00000204870704704484068704702494880D8
:10EBF00070470000CDCCCCCC580601100080FFFF40
:10EC0000FD4908707047FC4800787047FA49C871A0
:10EC10007047F948C0797047F748406AB0F5B47F4B
:10EC20002CBF012000207047F34840787047F2491C
:10EC3000002280B1012818BF7047487802280CD004
:10EC4000042818BF486A06D0B0F5B47F84BF4FF4DB
:10EC5000B470486270474A627047486A401C486214
:10EC6000F2E7E548407A7047E348C17911F0010FB7
:10EC700018BF704710B5002141720846F6F73CFEF8
:10EC8000BDE810400020F5F7D7BDDB48008CC0F38D
:10EC900000207047D84910B5098C0020C1F300212D
:10ECA00051B106F03DF964280FBF4FF0C04001217B
:10ECB00001FA00F040F08040BDE8104006F0E9B9EC
:10ECC000CD4A10B5C0F3074381B293611162C0F31E
:10ECD0000360507090700020C1F30021D06151B1E9
:10ECE00006F01EF964280FBF4FF0C040012101FA61
:10ECF00000F040F08040BDE8104006F0CAB9BE48C0
:10ED000040797047BC4A0028116A14BF41F00200E4
:10ED100021F0020010627047B74890F82000C0F35D
:10ED200040007047B44A10F0010F106A14BF40F061
:10ED3000020020F0020010627047AF49002091F8F5
:10ED40002010C1F34001002918BF0120704700289E
:10ED5000A94A116A14BF41F0010021F001001062BC
:10ED60007047A54890F8200000F001007047A249C4
:10ED70004A788A70487070479F48807870479F48EB
:10ED80000068406DC0F303607047012181409A48DC
:10ED900082691140816170470121814096488269F2
:10EDA00022EA010181617047934880697047924867
:10EDB000C0697047904910B5CC69C861024600230C
:10EDC00081210720FFF762FA204610BD8A48008C97
:10EDD000C0F380207047884880797047864890F853
:10EDE0002000C0F380007047834890F82000C0F3F3
:10EDF000C00070478048008CC0F3402070477E48B8
:10EE000090F82000C0F3C0107047FCF79BBA7A4816
:10EE1000008CC0F3403070477748008CC0F3C020AE
:10EE200070477548008CC0F300307047724A10F08C
:10EE3000805F116A14BF41F4806121F4806110F099
:10EE4000005F14BF41F4005021F400501062FCF741
:10EE500073BC6948016A002011F4806F18BF4FF03D
:10EE6000805011F4005F18BF40F00050704770B53B
:10EE70006149044610F0040F0D6A284614BF40F49F
:10EE8000807020F4807014F0080F14BF40F40070FC
:10EE900020F4007014F0100F14BF40F4006020F450
:10EEA000006014F0400F14BF40F4805020F48050F4
:10EEB00014F0200F14BF40F0800020F080000862A2
:10EEC0000021C0F3002050B106F02AF864280FBFDB
:10EED0004FF0C041012101FA00F040F080410846A6
:10EEE00006F0D7F8C4F38000C5F30021884208BFBC
:10EEF00070BD05F07AFF04460120F5F702FC14F41A
:10EF0000807018BF012002F007FF3D4890F86C00A8
:10EF1000C00805F0D3FF14F4C06F08BF70BD02F045
:10EF200082FBBDE8704002F06EBB3348016A0020EE
:10EF300011F0040F18BF012011F0080F18BF40F0A6
:10EF4000020011F4807F18BF40F0040011F4007F2C
:10EF500018BF40F0080011F4006F18BF40F0100017
:10EF600011F4805F18BF40F0400011F0800F18BF0F
:10EF700040F02000704703283CBF1F49486170479C
:10EF80001D48007D70471C49487370471A48407BF4
:10EF900070471948006B704717498A6A10438862A6
:10EFA000704770B5144EB06A40F000740020B06233
:10EFB000356A15F0040F18BF44F0010415F0080F6E
:10EFC00018BF44F0020415F4807F18BF44F0040415
:10EFD00015F4007F18BF44F00804FCF7B3F90028CB
:10EFE00018BF44F0805415F4006F18BF44F01004AB
:10EFF00015F0800F06E000006006011040060110C9
:10F000003083011018BF44F0200415F4805F18BF4E
:10F0100044F0400415F4005F18BF44F00054F16957
:10F0200044EA0140002918BF40F0806070BDFE49ED
:10F03000C8627047FC4890F82C0000F0010070474F
:10F04000F94890F82C00C0F340007047F64890F85B
:10F050002C00C0F380007047002818BF0120F2493F
:10F06000C87270472DE9F047002586B02F46F6F7A5
:10F0700069FBEE49052808680CBF90F8F80090F885
:10F08000580000F00F063046FCF78FFDDFF898833C
:10F090004FF0000A4FF00109002808BF54460FD076
:10F0A000446A05F0A2FE10F4C06F08BF88F80AA0F9
:10F0B00006D014F0020F18BF24F0010488F80A905B
:10F0C00014F0010F14BF0220042040F40031304638
:10F0D000F6F74DFC002804BF06B0BDE8F08701201C
:10F0E000F2F7E6F8F2F75BFEFAF7BEFD012837D03B
:10F0F0006846F3F712F800282ED00198F4F798FD2F
:10F100000298B8B10146CA4805F0C8FFC84A904203
:10F1100009D0C84AC84B014612781B7852005A439E
:10F12000C34805F058FEC5480078492804BFC048C8
:10F13000FBF766F9049848B1C148C24900780978DC
:10F1400008444200C048049905F045FE88F80B9039
:10F15000F3F72BF8012703E0F6F74CFB002DC3D0A3
:10F16000F2F714FCF6F776FD06B03846BDE8F087F6
:10F17000AD48C07A002818BF012070472DE9F04340
:10F1800087B005460F24F6F7DDFA0646F6F7E0FAF3
:10F19000DFF894828146052E07D1FBF798FE002800
:10F1A00004BF002088F80B0002D098F80B0058B973
:10F1B000F6F7D0FB07464FF48050F6F7C8FBFFF791
:10F1C00051FF3846F6F7C3FB052E0CBF9F4FA04FEB
:10F1D00005F00BFE002818BF0E2421462846F6F73E
:10F1E000C6FB002804BF07B0BDE8F08305F0F7FEBA
:10F1F00005F0FAFEF5F729FA04001DD10125F2F712
:10F2000057F82846F2F7ABFDC8F83C50F4F792F8EF
:10F21000A5F10108FAF728FD012809D0F6F792FABE
:10F22000B04205D1F6F794FA484508BF002C0AD041
:10F23000F2F7ACFBF4F7A3F805F0DBFEF6F70AFDF6
:10F2400007B0BDE8F0836846F2F767FFC0B16846D3
:10F25000FBF7F3FB0198F4F7EBFC6846B84704466C
:10F26000F2F7A3FF002CD5D115B901984045D1D1B3
:10F27000F2F78AFB002804BF2846F2F770FDC9E7C1
:10F28000F6F7ADFAC6E72DE9F14F88B04FF0000967
:10F29000CDF81890CDF81490CDF81C90CDF81090C2
:10F2A000F6F750FA01906348C846CDF80880047814
:10F2B0006148DFF888B1474605789BF8000004FBF9
:10F2C00005FA462804BF0898FBF79AF808980899A9
:10F2D00000EB4A0005F0E2FE03909BF800004B288B
:10F2E00004BF0398FBF78CF80898234600EB8A06C6
:10F2F00000954F493046039A05F0BCFE9BF800008C
:10F30000492804BF4A48FBF77BF84C4800784C2852
:10F3100004BF3046FBF774F80198052845D106EB89
:10F32000440BDFF804E13BF9020C3BF9041CDEF866
:10F330005830014406EB840030F9022C30F9040CFB
:10F3400010440022012B11D1DEF850305B1ACEF8A8
:10F3500054300093DEF84830A0EB030CCEF84CC0DC
:10F36000009B1E2BC4BFBCF11E0F0122CEF8501013
:10F37000CEF848000120CEF85800002A18BFFBF74D
:10F38000ADFDB6F93C0010F10A0FBCBFB6F93E0066
:10F3900010F10A0F09DABBF93C000A28C1BFBBF91A
:10F3A0003E000A280120FBF7E3FD1F48807A039006
:10F3B000002834D00198052831D1601E21184FF063
:10F3C000180C36F8112006EB410131F8021C511AD5
:10F3D00036F8102006EB4000891A30F8020C084479
:10F3E00000B202903228C4BF4FF00109CDF810904E
:10F3F0000020002D13D96146A4453CBF00FB04C288
:10F4000006EB420308D200FB041B33F8022C491C14
:10F4100026F81B20A142F6D3401CA842EBD306EBF2
:10F420004A039E4616E000006006011040060110E7
:10F4300080860110D5040110D60401105505011075
:10F44000DB040110DA040110808C01101B92001003
:10F450000B9800104FF0000C002D22D90021601EE7
:10F4600013D006EB400B36F810203BF802BCA2EBA1
:10F470000B0212B2002AB8BF524212B223F8102077
:10F480008A42C8BF1146401EEBD1198006EB4406E4
:10F4900003EB44034145C8BF88460CF1010CAC4561
:10F4A000DCD3FE48B0F90E0000908045A4BF4FF0B9
:10F4B0000109CDF81890F44600260EEB4A03002D02
:10F4C0002DD90022601E02281BD9039931B1019960
:10F4D000052903D1162888BF00210AD80CEB40016A
:10F4E0003CF810B031F802EC31F8041CF3445944F4
:10F4F00009B223F810109142C8BF0A46401E0228E4
:10F50000E3D800201A80588098800CEB440C03EB61
:10F510004403BA42C8BF1746761CAE42D1D3DF4B74
:10F52000B3F910209742A4BF4FF00109CDF8149011
:10F53000B9F1000F14BF186C586C00F1010014BF32
:10F5400018645864D6480078FF284AD008990AEB16
:10F550008A00022621F81090DDF820C006990CEBF5
:10F560004000B9F1000F4180059981800499C18064
:10F5700007990181196C4FEAE17C01EB1C5C6FF388
:10F580000B0CA1EB0C014181596C4FEAE17C01EBC2
:10F590001C5C6FF30B0CA1EB0C018181A0F80E80B9
:10F5A00007820299418200998182C282B3F8541085
:10F5B0000183B3F84C10418305EB8500089900F1F5
:10F5C0000103224600960CBF4E204D20FAF7B9FEEB
:10F5D00005EB8500431C2246009647200899FAF760
:10F5E000B0FE09B04846BDE8F08FAE4870472DE93F
:10F5F000F84F8346A948AE490025B0F90E80AB48C4
:10F600000978A94C00782E46AA464718F2F77AFBEB
:10F610000090A848A4F168090078492804BF48462A
:10F62000FAF7F2FF0020002F09D93BF8101039F843
:10F630001020891A24F81010401C8742F5D8DFF8F2
:10F64000749299F800004C2804BF2046FAF7DCFFBA
:10F65000009810F4007FA7F1010012D000281CBF11
:10F660008E49B1F9103026D034F910100029B4BFFA
:10F670004A420A469A42BCBF0D44761C401EF3D152
:10F6800019E000281CBF8549B1F9103013D004EBF4
:10F69000400234F8101032F8022C891A09B224F80A
:10F6A00010100029B4BF4A420A469A42BCBF0D441A
:10F6B000761C401EEBD1002EC8BF95FBF6F52EB28E
:10F6C000268099F800004F2804BF2046FAF79CFFD7
:10F6D0000025781E0ED034F81010891B09B224F8CA
:10F6E00010100029B8BF494209B28D42B8BF0D467B
:10F6F000401EF0D1258005F078FB10F4817F18BF03
:10F700004FF00508454506DD99F800004FF0010A65
:10F710004D2807D103E099F800004E2802D1204679
:10F72000FAF772FF99F80000472804BF2046FAF75D
:10F730006BFF5046BDE8F88F2DE9F04F87B0FBF71F
:10F74000BDFD5D4C2068B0F93610B0F9340005F00D
:10F75000A6FB0120F4F7D5FFDFF840A19AF81800C6
:10F7600010F0100F06D0042000F00FF90F2818BF7A
:10F77000F4F7C5FFFF208AF808000021481EFCF7B7
:10F780005CF805F090FC05F020FC002818BF01F0A3
:10F790004AFFF5F7D7FF022808BF4FF0000B7BD1D7
:10F7A0009AF801604448CAF834B0CAF838B0006822
:10F7B000B100806D20FA01F101F00F04C0F30325C0
:10F7C000C0F30319C0F30338C0F30357AC4220D190
:10F7D0000F2F05D005F009FB10F4817F18BF3C46C0
:10F7E000AC420CD1B8F10F0F09D0BAF82000C0F329
:10F7F000403020B105F099FB082818BF4446AC42C0
:10F8000007D1B9F10F0F04D0F6F789F8002818BF17
:10F810004C4631460220FEF7C7FD052E7CD2DFE8BC
:10F8200006F074030303780026460F249AF801506B
:10F8300005F0DBFA002818BF0E2421463046F6F703
:10F8400096F8002868D005F0CAFB05F0CDFBF4F768
:10F85000FCFE040037D19AF8000000281CBF00010C
:10F86000F1F783FCF2F762FA8AF803B0F4F767FF66
:10F87000F5F7C1FD114F4FF0E026DFF84480FAF7AD
:10F88000F3F901281FD0F5F75DFF022802BF9AF8AF
:10F890000100A842002C15E04BE0000060060110BA
:10F8A00055050110808C0110E88C0110DB0401105B
:10F8B000DA0401105A050110400601102C04011051
:10F8C0009004011006D005F08FFB05F092FBF6F7CF
:10F8D000C1F921E06846F2F720FC98B16846FBF7D1
:10F8E000ACF80198F4F7A4F9684605F0E1FB04468A
:10F8F000387820B1B069C8F80000C6F810B0F2F747
:10F9000054FCBCE7F5F776FFB9E7204605F07BFB32
:10F9100002E02046FFF732FCFAF7A6F9012803D1EE
:10F92000F5F710FF022804D1F5F70CFF02283FF489
:10F9300037AF05F040FBF4F7E3FEFBF7BFFCF5F74C
:10F9400001FF05281CBF07B0BDE8F08F0120F7F7C5
:10F9500061FAF0F727FF40B10020F0F781FF07B010
:10F960000020BDE8F04FF0F778BF0120F0F778FFF6
:10F970000020F0F70EFF07B0BDE8F04F05F04EBADB
:10F980004A000146314805F026BA2DE9F0413049D8
:10F9900080000968896D21FA00F000F00F04C1F3BE
:10F9A0000325C1F30317C1F30336C1F30358AC4277
:10F9B0001FD1B8F10F0F05D005F017FA10F4817FB1
:10F9C00018BF4446AC420BD10F2E09D02148008C01
:10F9D000C0F3403020B105F0A8FA082818BF34461B
:10F9E000AC4206D10F2F04D0F5F799FF002818BFBD
:10F9F0003C462046BDE8F08110B581680446B1B1AF
:10FA0000154805F04BFB144A904209D0134A144B99
:10FA1000014612781B7852005A430F4805F0DBF973
:10FA200010480078492804BF0B48FAF7E9FC21691F
:10FA300041B10D480D4A0078127810444200034845
:10FA400005F0C9F903490120C87210BD808C01106E
:10FA5000400601106006011080860110D5040110D7
:10FA6000D604011055050110DB040110DA04011061
:10FA7000FE48408A7047FD49B0F5C87F488284BF80
:10FA80004FF4C87048827047F848808A7047F74939
:10FA900088827047F548C08A7047F44AF449D0829A
:10FAA0000968098B814238BFD1827047EF4840789E
:10FAB0007047EE490228487004D8888ACA8A824270
:10FAC00028BF7047002048707047E848818AC28A82
:10FAD0000905407841EA022108437047E348C0899C
:10FAE0007047E249C828C88184BFC820C8817047D0
:10FAF000DE48008A7047DD49C828088284BFC820D4
:10FB000008827047D94880897047D84AD84990817F
:10FB10000968098B814238BF91817047D348817B46
:10FB2000028A0906808941EA024108437047CF48AA
:10FB300080787047CD4988707047CC48008B7047FB
:10FB4000CA49C828088384BFC82008837047C748AB
:10FB5000408B7047C549B0F5C87F488384BF4FF4D8
:10FB6000C87048837047C1488178428B0906008B72
:10FB700041EA023108437047BC490A7810430870D3
:10FB80007047BA4800787047B8490020087070473D
:10FB900010B5044605F091FAB44AB6492CB9137869
:10FBA00091F800C013EA0C0F06D1401E844205D123
:10FBB00010784978084201D0012010BD002010BD06
:10FBC0002DE9F05FDFF8A4B200252E469BF8014036
:10FBD000BBF814A0BBF8169005F01FFA0746A4481E
:10FBE00020210068008BB0FBF7F8A34805F06AFA03
:10FBF0009BF80200012808BFBDE8F09FF5F7A2FDC1
:10FC000005281EBF002C0024002F98BFBDE8F09FE0
:10FC10007B1E9748026808FB04F081B29C420FBF2C
:10FC2000108B601C08FB00F080B28A4524BF504551
:10FC30002546894524BF48452646601CC4B2BC42BF
:10FC4000E9D3B54228BFBDE8F09F8B4ADBF820100E
:10FC5000012099B1002D08BFBDE8F09F791B491E16
:10FC6000BB1BC9B25B1E8B42C8BFBDE8F09F50549E
:10FC7000491EC9B28B42FADDBDE8F09FB54288BF8C
:10FC8000BDE8F09F5055691CCDB2B542FAD9BDE828
:10FC9000F09F2DE9F00376484FF47A734FF0020C91
:10FCA0000268724840F22634B2F8C610C18101825F
:10FCB0008381B2F8C430438280F801C0848240F26C
:10FCC0008554C482002484700183438392F86C10AD
:10FCD00011F0040F09D011F0010218BF0122C26116
:10FCE00011F0020118BF01210162D0F81C8001212E
:10FCF0006048042440221023082580262027B8F1DC
:10FD0000000F0CD00170847001718271037280F851
:10FD100001C0C57080F805C0C67147720BE080F85D
:10FD200000C0857080F804C0867107724170C4708D
:10FD30004171C2714372BDE8F00341E72DE9F0471C
:10FD400005F075F904464B4E90F8E804DFF81C8185
:10FD50000027A6F14A05C0B9B078F178727A084355
:10FD6000317A114340EA010905F05CF905F055F9D3
:10FD70000100384607D02A5C22EA09022A54401CB6
:10FD8000C0B28142F7D8A8F8037094F8EA04A0B989
:10FD90003079717940EA010905F044F905F03DF93F
:10FDA0000021002807D96A5C22EA09026A54491C2A
:10FDB000C9B28842F7D8A8F8057094F8EC04002876
:10FDC00018BFBDE8F087B079F17940EA010405F089
:10FDD00029F905F022F90021002898BFBDE8F08735
:10FDE0006A5CA2436A54491CC9B28842F8D8BDE88B
:10FDF000F08770B514460E46054605F00EF905F07D
:10FE000011F905F064F90023012D02D0022D0CD068
:10FE100016E0042C08BF012312D0052C08BF0423D0
:10FE20000ED0082C08BF41230AE0042C08BF02238F
:10FE300006D0052C08BF082302D0082C08BF822357
:10FE40002B21714300EB8101087B8A7B82422CBF0E
:10FE50000A4A70BD12F800C04CEA030C02F800C058
:10FE6000401C91F80EC0C0B2844509E05007011053
:10FE700094070110B2970110929701106897011032
:10FE8000E8D270BD2DE9FF4F83B09B46DDE9041237
:10FE900000F049FE049801900598009005F0C2F822
:10FEA000054605F0C4F80446FD484FF00109871CDB
:10FEB00001783A78407811447A78C9B2104494F8BD
:10FEC000E824C0B2012A0BD1002918BF002807D0AE
:10FED00085F8E894DDE9001005235A4600F053FD4B
:10FEE00094F8EA04012839D138787978DFF8B4A396
:10FEF0000144CEB2AAF14A0890B99AF8044005F03C
:10FF000091F805F08AF802004FF0000008D018F8C8
:10FF10000010A14308F80010401CC0B28242F6D87D
:10FF2000787890B99AF8054005F07CF805F075F8F6
:10FF300001004FF0000008D018F80020A24308F894
:10FF40000020401CC0B28142F6D83EB185F8EA9448
:10FF5000DDE9001004235A4600F015FDDDE9040137
:10FF600007B05A46BDE8F04F00F0F8BE2DE9F14F5A
:10FF7000CD488AB041780591B0F81490B0F8168059
:10FF800005F050F8044605F052F805F0A0F802908C
:10FF9000C6480026006890F8CE0080000490A07942
:10FFA0000190207A009094F84170002F88BF4FF0A4
:10FFB000010A5DD92B2006FB00F1029800EB8105B8
:10FFC000BA48B5F860100268B2F818B001FB0BF03F
:10FFD000118A90FBF1F081B2ADF81C10B5F8620007
:10FFE000B2F81AC0538A00FB0CF090FBF3F080B219
:10FFF000ADF80C0092F86C2012F0040F14BF2AEA3E
:020000021000EC
:10000000020302F001031BB1ACEB0000401E80B202
:1000100012F0020F03D0ABEB0101491E89B212F0BE
:10002000040F19BFADF81C00ADF80C10ADF81C1092
:10003000ADF80C00BDF81C00A5F89C00BDF80C0044
:10004000A5F89E009848807801280DD0F5F77AFB36
:1000500005281CBF0598002806D0BDF80C004845AF
:1000600024BF804585F892A0701CC6B2BE42A1D3C1
:10007000DFF8349299F80180B9F80E60B9F81050A1
:10008000B9F80C70B9F818A004F0CCFF029005F094
:100090001EF8069005F020F8029899F8021090F8E2
:1000A00041B0824801290068408B04BF554656463E
:1000B0000023BBF1000F72D9A0F1C801A0F10A0A18
:1000C000A0EB0609A0EB050C05912B2003FB00F12A
:1000D00006984FF0000E00EB8101B1F89C20B1F8BA
:1000E0009E0081F88FE0C82A27D8B8F1010F04BF1D
:1000F00091F892E0BEF1010F07D0B8421AD89642AB
:1001000063D3012081F88F0036E087420AD30A2E9C
:1001100005D8964201D3012029E0002027E00A2AD1
:10012000FBD8F8E70A2D02D89542F6D3F3E70A2A5E
:10013000F3D8F0E7AA42E4D947E0DDF814E07245CD
:1001400043DBB8F1020F04BF91F892E0BEF1010F5A
:1001500006D0B84227D89145D8BF0220D2DD34E07E
:10016000874217D30A2E12D89145D6DC022081F897
:100170008F0010F0FF0F28D091F8A500022819D0A9
:10018000032804BF91F86B00012813D01DE05245ED
:10019000ECDAC2E70A2D03D89445E7DDBDE719E0A4
:1001A0005245E3DAB9E79445DCBF022081F88F00BD
:1001B000E2DD0AE0029A012082F8E904062081F8D3
:1001C0008C0091F88F0081F89000581CC3B25B45F9
:1001D000FFF47BAF94F8E804002871D0324D2889F1
:1001E000401C80B22881B0F5167F84BF4FF4167092
:1001F00028816889401C80B268810499884229D38B
:1002000004F00BFF03004FF0000118BF284A1FD075
:10021000505C10F0100F1CBF20F010005054C0B202
:1002200010F0200F1CBF20F020005054C0B210F07E
:10023000040F1CBF40F010005054C0B210F0080F63
:100240001CBF40F020005054481CC1B29942DFD37B
:1002500000206881144E7078059004F0E3FE074694
:1002600004F035FF049004F037FF02900F48016856
:10027000D1F8C800069091F8CE000890488BB1786C
:10028000758A728B97F84190012908BF1546401B6B
:100290004FF0000B87B25E46B9F1000F0AE00FE0A5
:1002A00053070110B2970110500701109407011075
:1002B0006897011088BF4FF001087DD800F0A0B901
:1002C0000A9806900198059000980490F94847789C
:1002D00004F0A8FE054604F0FAFE064604F0FCFE13
:1002E00004F0EBFE0890F448002195F841500068B6
:1002F0000A460B46B0F81AC090F8CD000290002DC7
:100300002DD9DFF8B893ACF125084FF0010A4FF072
:10031000020B8E462B20584306EB800080F890E0BD
:1003200090F8A0C01CF0010F15D0B0F89CC0BCF133
:10033000250F06D880F890A099F80000012808D170
:1003400055E0C44507DB80F890B099F8000002281A
:100350004DD0501CC2B2581CC3B2AB42DAD3D84BFA
:100360004FF0000818780844597810F0FF00114445
:10037000C9B218BF002933D00144029881422FD35B
:10038000DDE905104FF00108049A00F066FBC94949
:100390000020002D4881014684BF0898A0F1010C7F
:1003A0001ED92B20484306EB8000D0F8A02012F085
:1003B000010F11D0437800E01CE0002B18BF63450B
:1003C0000AD190F89030BB4207BF90F89230012BD1
:1003D00042F40072C0F8A020481CC1B2A942E0D388
:1003E000B44884F8E88400210181418132E7481C47
:1003F000C1B2B0E72B2006FB00F1049800EB8102AC
:100400002B2192F8520092F88CC041430298BCF123
:10041000060F00EB8103B2F89C00B2F89E107AD070
:1004200092F8A5C0BCF1020F18BFBCF1030F09D0B0
:1004300092F8A00010F0010F6DD092F85000022841
:1004400078D0D8E04FF0000C82F890C0A84282BF6C
:1004500087424FF0020C82F88CC00AD892F850C044
:10046000BCF1020F02BF93F88CC0BCF1020F82F8FE
:100470008CC092F8A5C0BCF1030F04BF92F850A045
:10048000BAF1020F07D193F88CA0BAF1010F08BF9F
:1004900082F88C803FD092F88CA0BAF1020F18BF7E
:1004A000BAF1010F37D0BCF1020F0CD092F850C056
:1004B000BCF1020F04BF93F891C0BCF1000F02D051
:1004C000A84207D928E092F88FC0BCF1010F07D0ED
:1004D000A84202D882F8908008E0BCF1020F1AD03E
:1004E000B84218D34FF0020C82F890C092F890A056
:1004F000DDF814C0E24504BF92F892C0BCF1010FD0
:1005000060D092F8A5C0BCF1020F14D092F850C090
:10051000BCF1020F03D06EE08742E3D96BE093F8A1
:1005200091C0BCF1000F06D093F88CC0BCF1030F52
:1005300013D060E04FE0A2F89400A2F89610B2F851
:100540006000A2F89800B2F86200A2F89A000320B6
:1005500082F88C0082F891804DE0B3F894A0A0EB73
:100560000A0CB3F89600081A0CFB0CF100FB001003
:100570000699884226DCA2F894A0B3F89600A2F867
:100580009600B3F89800A2F89800B3F89A00A2F881
:100590009A0093F89100401CC0B282F8910008992B
:1005A00088423CBF032082F88C0024D3042082F8C8
:1005B0008C0092F8900004223146FFF71AFC4FF0AD
:1005C000010B18E082F88C80D2F8A00040F4806023
:1005D000C2F8A0000FE0B3F89400A2F89400B3F8BA
:1005E0009600A2F89600B3F89800A2F89800B3F825
:1005F0009A00A2F89A00701CC6B24E45FFF4FAAEFB
:1006000094F8EA044FF000084BEA000084F8EA048A
:100610000A9806900198059000984FF00209CDF8CD
:100620000080049004F0FEFC824604F050FD074672
:1006300004F052FD20489AF84150006890F8CE002E
:10064000460804F03AFD83469AF8E80401287DD173
:1006500018480089B04208D8DDE90510049A00F076
:10066000FCF914480021418141E00026002D84BF9F
:10067000ABF1020001903ED92B20704307EB8000C4
:10068000D0F8A01011F0010F2DD011F4806F2AD1F5
:100690004178012918D803780A4AD35C4A3292F883
:1006A00008C013EA0C0F0FD0107805223146FFF76F
:1006B000A0FB18E05007011094070110B297011039
:1006C0005507011068970110019A91420BDB0178E0
:1006D000FE48425C4A30417A0A4204D04078052202
:1006E0003146FFF786FB701CC6B2AE42C4D39AF8FF
:1006F000E80401284AD10020002D88BFABEB090394
:1007000016D92B21414307EB810191F8A520022A3C
:1007100018BF032A08D14978494505D39942BCBF7F
:1007200008F1010101F0FF08401CC0B2A842E8D363
:10073000B8F1000F1CBF0026002D27D9DFF89093D9
:10074000ABF101084FF0050A2B2000E01EE07043DA
:1007500007EB800090F8A01011F0010F12D0417843
:10076000002908BF99F8003004D0414508BF99F826
:10077000013007D133B180F88CA0052231461846EC
:10078000FFF737FB701CC6B2AE42DDD394F8EA1413
:100790000098084384F8EA040A9800F0D5FC94F81D
:1007A000EA144FF0000A084384F8EA04CDF800A0E8
:1007B000CDF804A0CDF808A004F034FC044604F001
:1007C00036FC814604F083FC804604F085FC074635
:1007D00094F84100002200282AD901264FF0030B8B
:1007E00002254FF00A0E0DF1FF302B21514308EB8B
:1007F00081014FF02B0C91F8523003FB0CF391F870
:10080000A5C007EB8303BCF1020F18BFBCF1030FB7
:1008100017D091F8A03013F0010F1CBF91F85110C0
:1008200001F800E0511CCAB294F841109142DCD8A2
:1008300084F8EBA40025EB46A648405D012836D09D
:1008400091E091F891C0BCF1000F12D091F88C307A
:10085000042B18BF092B06D0BCF1050F84BF91F8FB
:1008600051301E5402D891F851301D5481F86BB0AC
:10087000D8E791F88CC0BCF1010F18BFBCF1020F92
:10088000D0D191F850C0BCF1020F0CD193F891C0B7
:10089000BCF1000F07D0B3F898C0A1F860C0B3F85E
:1008A0009A30A1F8623091F851100D54BAE71BF854
:1008B000051021B10A2908BF0BF8050053E094F890
:1008C00041600A2E3CBF94F842000A284BD299F8A6
:1008D00041C00020BCF1000F88BF6B1C43D92B2105
:1008E000414308EB810207EB810191F851E09E45FD
:1008F00035D191F88CE0BEF1090F1FBF92F88C2022
:10090000062A91F8A01011F0010F28D02B21714375
:1009100008EB81062B21484307EB8001AC223046CF
:1009200004F04AFA94F84100401C84F8410094F81D
:100930004200401C84F8420094F8EB04401C84F808
:10094000EB04B6F89800A6F86000B6F89A00A6F88E
:10095000620086F891A0072086F88C0003E0401C16
:10096000C0B28445BBD8681CC5B20A2DFFF464AF81
:1009700056480099016201994162BDF8081001854D
:100980000BB0BDE8F08F2DE9F84F054600209846E2
:1009900016460C46009004F045FB04F08EFB07461B
:1009A00004F03BFB49494C4AB8F1040F45D0B8F17B
:1009B000050F3CD0B8F1080F1CBF1168B1F90E301B
:1009C00042D0B44288BFBDE8F88F9DF80090A7F1EF
:1009D0000108DFF8F8A09DF801C0BF1E35F914200A
:1009E00001199A42BCBF35F91110994205DA1AF87B
:1009F000041021EA09010AF8041008FB004189B239
:100A000007FB004235F9111092B29942BCBF35F98B
:100A10001210994205DA1AF8041021EA0C010AF8BA
:100A20000410611CCCB2B442D8D9BDE8F88FB1F83B
:100A30004C102823ADF80010C3E71268B1F84E102F
:100A400092F8CC20530805E01268B1F8501092F8E3
:100A5000CC205308ADF80010B3E72DE9F05F154640
:100A60000F46064604F0DEFA044604F030FB04F0BC
:100A700024FB804604F0D1FA8346174894F8E81422
:100A80000068012906BF90F8CC00420890F8CC20FD
:100A90003C46DFF838C0AF420CF14A0A9CBF9AF8D6
:100AA00002009AF808901CD836F9141091420BDD18
:100AB0001CF804100F2C41EA00030CF8043024BF8A
:100AC00043EA09010CF80410611C07E06897011063
:100AD000B29701108897011094070110CCB2AC4274
:100AE000E2D9A8F1010000FB0BF081B2AF423ABF9E
:100AF0009AF803309AF80940BDE8F09FC81936F912
:100B00001000904209DD1CF8070018430CF807009C
:100B10000F2F24BF20430CF80700781CC7B2AF4248
:100B2000ECD3BDE8F09F2DE9FF4F87B01E46884605
:100B300004F078FA04F07BFAFF4990F8E824096899
:100B4000012A0CBFB1F90E1091F8CC104627029182
:100B500004F0B3FA059004F060FA01900020834697
:100B6000044684460546034603900998B04269D876
:100B7000F24991F804A08A780492019A8979521E68
:100B80000092079A125C4AB338F91090029A914584
:100B900024DBEB4A125C12EA0A0F14D138B1DFF8F9
:100BA000A093814419F8019C19EA0A0F0BD1DDF8D2
:100BB0000090484509DADFF88893814499F801905C
:100BC00019EA0A0F01D0641CE4B2DDF8109012EAB1
:100BD000090F03D0039A521CD2B2039238F91020A5
:100BE000BA4204DB002B08BF05465B1CDBB2BA42ED
:100BF00001DBB04222D1062B2A4605EB030E0ED3B1
:100C0000964588BFCE4B18D913F8029049EA0109DE
:100C100003F80290521CD2B27245F5D30DE0724532
:100C200038BFC74B09D213F8029029EA010903F82B
:100C30000290521CD2B27245F5D30023401CC0B2C0
:100C4000B0429ED9002209981546B0427AD805993B
:100C5000491E00910199491E0591B84991F805A0D6
:100C6000CB780493CB79DDE9001901FB0901DDF8AC
:100C70001C9089B219F80190B9F1000F2ED038F903
:100C800011E0DDF80890CE4528DBDFF8B49219F8C2
:100C9000009019EA0A0F14D138B1DFF8A4E28644B3
:100CA0001EF801EC1EEA0A0F0BD1DDF814E07045C6
:100CB0000BDADFF88CE286449EF801E01EEA0A0FA8
:100CC00003D00CF1010C0CF0FF0CDDF810E019EA78
:100CD0000E0F1CBF0BF1010909F0FF0B38F91110C1
:100CE000B94204DB002D08BF02466D1CEDB2B942CB
:100CF00001DBB04222D1062D114602EB050E0ED3C8
:100D00008E4588BF8E4D18D915F8019049EA030920
:100D100005F80190491CC9B27145F5D30DE0714544
:100D200038BF874D09D215F8019029EA030905F863
:100D30000190491CC9B27145F5D30025401CC0B2D1
:100D4000B04290D97F480399017080F801B0801CAF
:100D5000047080F801C00BB0BDE8F08F2DE9F74FAB
:100D600092B0002400940194029403940494059496
:100D700006940794089409940A94824625460B9495
:100D80000C940D940E940F9404F04CF98146F4F7F2
:100D9000D9FC05287ED099F8E80401281FBF99F8EE
:100DA000EA04012899F8EC04012804D0002C04BFBF
:100DB00015B0BDE8F08FE84608AFDDF84CB0149EE2
:100DC00004F02BF9814604F078F910905A484FF05E
:100DD000020C5C460068B34590F8CC009CBFA9F1BA
:100DE0000102012116D80CFB09433AF91330834262
:100DF0000CDB08F80410002C1CBF08EB040303F8FC
:100E0000011C9442BCBF08EB04035970631CDCB2A4
:100E1000B442E8D91099C91ECAB2B3459CBFA9F122
:100E200001034FF0010C1BD802FB09B189B23AF95A
:100E3000111081420EDB07F80BC0BBF1000F1CBF85
:100E400007EB0B0101F801CC9B45BCBF07EB0B0185
:100E500081F801C00BF1010101F0FF0BB345E3D9AB
:100E6000CDF844D0DFF8E090DDE913480DF1200B18
:100E700099F8017004F0DBF804F01FF9109004F009
:100E8000CCF8064699F8020001287DD0F4F75AFC08
:100E9000052800E001E077D0BFE00027B8463E46D5
:100EA0003C46109704F0BEF804F007F9119004F0E6
:100EB000B4F8254A0021136A002B11BF0A46421AD2
:100EC000521E92B269B93AF912C0BCF1500F08DD56
:100ED00002EB000B3AF91BC0BCF1500FC8BF4FF03A
:100EE00001083AF912C0BCF1780F07DD02EB000CE3
:100EF0003AF91C20782AC4BF7A1CD7B2022F02D23A
:100F0000B8F1000F03D0012161F3070603E0491C8B
:100F1000C9B20529D0D34FF00008119AC446414602
:100F2000571E002B11BF07FB0012421A521E07FB6F
:100F3000002292B2C1B909E094070110B2970110E2
:100F40006897011053070110500701103AF912B0C9
:100F5000BBF1500F17DDA2EB000B3AF91BB0BBF150
:100F6000500FC8BF4FF001083AF912B0BBF1780F2B
:100F700009DDA2EB000B3AF91B20782AC4BF0CF163
:100F8000010202F0FF0C00E046E0BCF1020F02D2C9
:100F9000B8F1000F03D0012161F30F2603E0491CD3
:100FA000C9B20529BDD306F0FF08B8F1010F01D081
:100FB000310A1DD00022A0EB020C0721ACF1010781
:100FC000002B14BF00FB012C00FB017C1FFA8CFCE2
:100FD000491C3AF81CC0C9B2A4440FFA8CF4082981
:100FE000EED9511CCAB2012AE5D9B4F5AF7F01DCB4
:100FF000109850B1B8F1010F04BF012060F307054C
:10100000300A1CBF012060F30F25E8B2290AC8424C
:1010100014BF01240024BEE6002744459CBF10985D
:10102000A0F101094BD8FF4BA0199A7893F804C09E
:1010300042EA0C02A3F14A0C1CF804E012EA0E0F7B
:1010400016D01A78BA4204D1A3F12002125D012A07
:101050000ED000222AF814201199095D41B91CF81C
:10106000041093F802E011EA0E0F08BF2AF81020CE
:1010700009FB0640DA7893F805E080B242EA0E02F6
:10108000811B1CF804E089B212EA0E0F13D05A78C3
:10109000BA4203D1E44A125D012A0CD000222AF898
:1010A00010201BF8040030B91CF80400DB7818424B
:1010B00008BF2AF81120601CC4B24445B3D9E8B275
:1010C000012819D1D94800210C46D0F820C00020B1
:1010D000721A531EBCF1000F14BF06FB001206FB70
:1010E000003292B2401CC0B22AF812400728F1D355
:1010F000481CC1B20529EAD31098401E704387B23C
:10110000280A04BF15B0BDE8F08F0022C74807EBDE
:1011100006081546046A0020BB18A8EB020C002C38
:1011200012BF06FB103106FB10C1491E89B2401CDC
:10113000C0B22AF811500728F1D3501CC2B2052AB8
:10114000E9D315B0BDE8F08F2DE9F14F84B0002050
:10115000B64C074601906078039003F063FF0546A4
:1011600003F0B5FF029095F841B003F0A6FF277099
:101170004FF00009BBF1000F84BF401F009040F208
:10118000CB812B2009FB00F1029800EB810494F83D
:101190008C00042818BF062800F0B78194F8A50039
:1011A000022818BF032840F0B08160784FF0000893
:1011B0004246042806D823789D49CB5C4A31897978
:1011C0000B4209D10099884225DB23789849CB5CF2
:1011D0004A31C9790B421ED0237895490122C95C56
:1011E000904B93F804C011EA0C0F06D0042804D8E1
:1011F000187884F89000904655E093F805C011EAFD
:101200000C0F08D00099814205DC587884F89000D2
:101210004FF0010847E094F89010002908BF002A19
:1012200000F06481A27B237B94F80DC0D21AD3B264
:10123000E27BA2EB0C02B4F844C0D2B2BCF12D0F99
:1012400003D29A1A921D0C2A02D94FF0010803E02A
:1012500094F89120012A01D009BB0FE0714A13785C
:10126000994204BF09F1010363F30F2752789142B9
:1012700004BF09F1010262F31747EDE7B8F1000F6F
:101280000DD004289CBF6748007805D90099884292
:10129000A4BF6448407806DB84F8900003E0B8F10E
:1012A000000F00F02381049D03F007FF824603F046
:1012B000B4FEE1884CF6CD425143A2884CF6CD43B2
:1012C0005A43C2F3C74394F8A520C1F3C741022A89
:1012D00070D194F88C20022A18BF012A6AD14A1EC4
:1012E000032A68D86278002A65D001FB00321FFA11
:1012F00082FC022949D8012908BF664604D0022988
:1013000004BFACEB000296B2022B1DD3C21E934267
:1013100005EB460232F9043C29DC002B1CBFB2F974
:1013200004A0BAF1000F30D035F91620B2EB430F0C
:10133000D8BFB2EB4A0F28DD331835F91330D21A73
:101340006332C62A21D8E0E005EB4602B2F9043048
:10135000002B1CBF35F91620B2EB430F15DD3318F7
:1013600035F91330D21A6332C62A5AD90DE0002B50
:101370001CBF35F91620B2EB430F06DD331835F9E3
:101380001330D21A6332C62A4BD9491E624601294C
:1013900010DB121A92B235F912303BB135F91C60EC
:1013A00003EB8303F600B6EB430F3ADC491E09B2A8
:1013B0000129EEDA89E0AAF105029142A4BFAAF15F
:1013C00001028A427EDD01FB0032AAF1030C92B2D7
:1013D0008C455EDCAAF1020E714508BF164605D0A9
:1013E000614504BF02EB000C1FFA8CF6022B2BD3D5
:1013F000A0F1030C634505EB460339DC33F904EC3B
:10140000BEF1000F1CBFB3F904C0BCF1000F40D007
:1014100035F91630B3EB4E0FD8BFB3EB4C0F38DDB8
:1014200008E072E0B2970110929701105007011086
:1014300068970110A6EB000C35F91CC0A3EB0C0358
:101440006333C62B25D860E005EB4603B3F90430BF
:10145000002B1CBF35F916C0BCEB430F19DD331A46
:1014600035F91330ACEB03036333C62B4DD910E0D1
:1014700033F9043C002B1CBF35F916C0BCEB430FFD
:1014800007DD331A35F91330ACEB03036333C62B96
:101490003BD9AAF10206491C1346B14215DC0344AC
:1014A0009BB235F913C0BCF1000F08D035F912A07A
:1014B0000CEB8C0C4FEACA0ABAEB4C0F25DC491C2A
:1014C00009B200E001E0B142E9DD092084F88C00B6
:1014D00094F8900008224946FEF78BFC344994F8B2
:1014E00090000A78104308700120019094F8A5003C
:1014F000022804BF94F89000002806D1B8F1000F2C
:1015000004BF09F1010060F3070709F1010000F0D1
:10151000FF09CB453FF635AE0024BBF1000F39D9AA
:1015200007F0FF08C7F30726C7F307474FF0040982
:101530002B2004FB00F1029800EB810090F88C1046
:10154000042918BF092921D090F8A510022918BF35
:1015500003291BD190F89110012917D9B8F1000F78
:1015600018BF45461AD08DB190F8902003998A4251
:1015700004BF90F89210012908D080F88C90D0B266
:1015800004222146FEF735FC01200190601CC4B204
:101590005C45CDD3019805B0BDE8F08F002E18BF93
:1015A0003546E0D1002F18BF3D46DCD1EEE7000004
:1015B00050070110FE48FF490068C0EBC00000EB77
:1015C000800001EBC0007047FB48A0F10C014968A6
:1015D00000EB41007047F648F649006880F00100D2
:1015E000C0EBC00000EB800001EBC0007047F0488A
:1015F000F149406880F0010001EB400070474FF472
:101600008C7103F05FBD10B52621EC4803F05AFD44
:10161000E8480021C0F85612C0F85A12A0F85E122D
:1016200080F8601210BD70B5E14C00252560656042
:10163000F4F788F80528E24808BF0C30E560A060A0
:1016400070BDDB48016881F001010160416881F0F3
:101650000101416070472DE9F0410E46044603F058
:10166000DCFC054603F029FDD148D349406880F0F1
:10167000010001EB40004078002814BF0023BDE8C2
:10168000F08103FB05FC17220CEB0200521C36F81C
:10169000101024F810101F2AF6DD5B1C0F2BF0DD54
:1016A0000026002206FB05FC104617210CEB010367
:1016B00034F9133013F1070F03DBA3F10807112FDF
:1016C00001D21A44401C491C1F29EFDB0228A4BF89
:1016D00092FBF0F317210CDB0CEB010034F9102026
:1016E000D71D0F2F24BFD21A24F81020491C1F2900
:1016F000F2DB761C0F2ED4DDBDE8F081B14A00216B
:10170000A2F1260C135C0CF8031011547047A84981
:10171000A84A086880F00100C0EBC00000EB800020
:1017200002EBC00C48680C3180F0010001EB400274
:10173000002110780028D8BF704730B4032302245A
:10174000C1EBC1000CEB8000457E012D05D0107867
:10175000491C8842F4DC30BC7047457D022D08BF2F
:101760004375857B012D08BF8473F0E72DE9F05F99
:101770008F49904A086880F00100C0EBC00000EB80
:10178000800002EBC00748680C3180F0010001EBDB
:10179000400600F0AAFC317800250029D8BFBDE83A
:1017A000F09FA0F10108DFF814A24FF000090AF140
:1017B000260BC5EBC50007EB8004607E012813D122
:1017C000607988B110F8081011F0800F18BF84F804
:1017D000199009D100F080FCA17E681C0AF8010074
:1017E0006179A07E0BF8010030786D1CA842E0DC26
:1017F000BDE8F09F10B500F07AFC03F072FCFFF733
:10180000B5FFFFF784FF6A48016881F001010160BC
:10181000416881F001014160002010BDB0F9021063
:101820003F29CCBF3F220A4662F31743012262F3ED
:101830000703FA29C8BFFA2161F30F23022161F3DC
:101840001F63036170470A2262F3174162F30701C5
:1018500062F30F21022262F31F61016170472DE9DB
:10186000F34F8A46524983B000240868039FC0EBB7
:10187000C00000EB80024F4800EBC2064A6801F14D
:101880000C0000EB42000190886801680091D0F8DC
:10189000049030464FF48C7103F014FC03F0BDFB50
:1018A00000258046B9F1000F3CD9009805EB850171
:1018B00000EB41000168CBB2C1F30722C1F3074B33
:1018C0004FEA116E02FB083C0EFB08BB37F91CC047
:1018D00037F91B1090F809E00CEB010BF3451EDD06
:1018E00004EB0A010A291AD2C4EBC40E06EB8E0CD3
:1018F00001218CF8191006F82E308CF80120ACF874
:1019000002B04168CCF808108CF81A500089ACF885
:10191000170027488068816860468847641C6D1CF2
:101920004D45C2D301980026002C04702048006861
:10193000C0EBC00101EB81021E4980F00100C0EB49
:10194000C00000EB800001EBC20A01EBC00984BFBC
:101950004FF0000BDFF864801FD9C6EBC6000AEB1E
:101960008005AF7E18F8070000286DD0401E0221C8
:10197000C0B22971C0EBC00109EB81014A796A71DB
:10198000A871C87EE876701C08F807006A790D48CF
:10199000A97E8154761CA642DFD3054E054D3068E2
:1019A000C0EBC00101EB810105EBC1070CE00000B9
:1019B00074070110BC97011080070110EC99011009
:1019C000D47C0100129A011080F00100C0EBC0002D
:1019D00000EB8000002105EBC00C002C84BF4FF011
:1019E00001084FF0020909D9C1EBC10007EB8000E3
:1019F000427E012A3ED0491CA142F5D303F05DFB93
:101A00009148716800EB410730680026C0EBC001C7
:101A100080F00100C0EBC00000EB800005EBC009C6
:101A2000387801EB810105EBC10800284BDDC6EBDE
:101A3000C60008EB80052879022818BF002133D0A2
:101A4000687E01283BD136E000F06BFB002808BF20
:101A500085F819B09ED001212971687185F806B00A
:101A600085F81BB0701C08F807006A797748A97ED2
:101A700081548FE7827990F804A0C2EBC202B0F9DA
:101A800002300CEB8202BAF1020F14BF0022927DE9
:101A9000012A16BF022A027EC27D9342ACBF80F8A3
:101AA000148080F81490A6E7A879C0EBC00009EB79
:101AB0008000417DC4E7287D03F018FB6875387805
:101AC000761CB042B3DC039805B02146BDE8F04F68
:101AD000AFF300802DE9F05FDFF874818946064698
:101AE000D8F800105B4AC1EBC10000EB800002EBAC
:101AF000C00481F00100C0EBC00000EB80000127B2
:101B000002EBC00A03F089FA0546F3F71BFE05282D
:101B100004BF607E01281BD12078617801FB05029B
:101B2000491C01FB050106EB4200B0F90220B0F9A7
:101B300004001044133026280AD806EB4100B0F9FF
:101B40000210B0F9040008441330262898BF00277B
:101B500000253F488068D0E900B803F05EFA002114
:101B60000346B8F1000F30D901EB81000BEB4002C6
:101B70001068527A00F0FF0CC0F3072E0EFB03CC66
:101B8000C0F3074E000E00FB03E036F91CC036F927
:101B9000100060449042C8BF6D1C491C4145E3D30E
:101BA000062D12DD00F0A3FA03F09BFAFFF7DEFD2D
:101BB000FFF7ADFD2648016881F001010160416831
:101BC00081F001014160BDE8F09F0021B9F1000FF3
:101BD00098BFBDE8F09F03254FF0010C0226C1EB32
:101BE000C10004EB8000427D022A05D0032A04BF15
:101BF0000279022A07D022E00773002F14BF8573F1
:101C000080F80EC01BE08279C2EBC2020AEB8203AD
